:020000040000FA
:080000000002040000000000F2
:020000040000FA
:100400006F2521000E7F22000E01880000000000F1
:100410000C000700E0AE29000100200011000700D9
:10042000000020000000E000020032000000020096
:100430000000000042A30200000000000040DA00BB
:100440000000FE004440A900A04821000000E00098
:100450000300320000002000A00188004440A800F2
:100460000000060091018800800078000000EB0089
:1004700015003700E280400032A0B4009101BA00BC
:10048000E280400032A0B4009102BA00E280400055
:1004900032A0B4000002EB00472BDE00F507B200EB
:1004A000602CE10004003A000059EB008301E900F0
:1004B000FDFF3E00040037006128E100010032002A
:1004C0000082EB00040007001101BA000200E00006
:1004D000E8FF3A00000006003159BA008301E90044
:1004E0000C0032002159BA008301E90008003200F3
:1004F0000400E00003003A00E280400032A0B400B3
:10050000F5FF370011D9BA008301E900FAFF3A007C
:100510008100E800E180400032A0B4000000060045
:10052000E4B8040000000000ECB804000000000083
:10053000B0B8040000000000DEAF040000000000BE
:1005400052B0040000000000AEB004000000000043
:10055000BA64040000000000C06404000000000051
:10056000D06404000000000044BD0400000000004E
:1005700090BD0400000000009ABD040000000000CF
:10058000AABD040000000000BEBD04000000000081
:100590005CBD0400000000006A9804000000000038
:1005A00088980400000000009698040000000000F5
:1005B000A498040000000000B098040000000000AF
:1005C0002C990400000000004A990400000000007B
:1005D0005699040000000000DE9A040000000000AC
:1005E0006899040000000000AC99040000000000BD
:1005F000F099040000000000349A0400000000009C
:10060000789A040000000000C29804000000000076
:10061000969A040000000000A49A04000000000064
:100620000040DA000000FE00020AB900001BB90019
:100630000200B80081004200810043000000060073
:100640001004B100030035009001B10001003C002E
:100650001000050000000500800078001104B100C2
:10066000030035009101B10001003C000050A000E2
:10067000000006001004B100070035009001B10031
:10068000040034007000B100030035009001B10097
:1006900001003C0010000500000005006900E100B9
:1006A000040035006D00E100030034000002B100D9
:1006B0000100320000000500100005002002E200E9
:1006C00004003D002342AB00020032002302AB00D5
:1006D000FEFF32000040DA00FEFF37000A00FA0099
:1006E00080017800E20F500028003E00908E8000CC
:1006F000E10F500008003200802320000000E000DD
:10070000050032000423200025232000462320007A
:1007100080017800040037000422200025222000F8
:100720004622200083222000144090000004E000B4
:10073000040035008009EB00144090000074A00014
:1007400010429800154090000028A30003003A00D2
:10075000154090000024A000904298008001EB001A
:1007600007003700154090000008A300FDFF32008D
:1007700063C078000000FB00000B78008301E800F4
:10078000828F5100F7FF3A00080037003000200048
:10079000B0BF9F00C3BF9F00D1BF9F00E2BF9F00BB
:1007A0006A80570000C0DA006FB997000200780035
:1007B0000080FA00000006000A00FA001100200084
:1007C000B1BF9F00C0BF9F006A80570000C0DA0021
:1007D0004FB897000080FA00000006000A00FA00F7
:1007E00051002000B1BF9F00C0BF9F006A8057002A
:1007F00000C0DA005FB897000080FA000000060031
:100800000A00FA00881F7800800178000000E000EC
:1008100029003A00908E8000E10F5000080032005D
:10082000802320000000E0000500320004232000A7
:100830002523200067232000800178000400370072
:10084000042220002522200067222000832220008D
:10085000144090000004E000040035008009EB0023
:10086000144090000074A000104298000002EB00B9
:100870000C003700130A2000154478006140640022
:1008800002003A008301E900FBFF3A000402E8009D
:100890009541780061C061000500320017007800C2
:1008A0008058780004035100820F5200F1FF3A0093
:1008B000060051000800370020002000A0BF9F0064
:1008C000B3BF9F00C1BF9F00D2BF9F006C80570085
:1008D00000C0DA005FB897004F0478000080FA008B
:1008E00000000600889FBE0080047800A08E800073
:1008F0000000E00003003A00100007000000E000E4
:100900000A003500A08E80000900E00002003A00D5
:100910000004780006003700000478000900400059
:10092000060007000000E00001003D000084EB002D
:10093000080078004F04BE00000006008000780028
:100940000000E00004003A00601D2100A08E880035
:1009500001017800060037000081EB0060252100CE
:10096000808F500002003E00A18E88000001EB0045
:1009700002007800000006006022B8000602200095
:100980000000D0008180D2000482D2008582D20093
:100990000000A0000202520083825A0003003100CE
:1009A0000202420083824A000000A1000603E9001F
:1009B000F3FF3A0000000600EFFF07000400BE004E
:1009C00000000600889FBE008A9FBE008C1F780032
:1009D0000205BE000004BE000006EB00E00F500060
:1009E000E08F5800E00F5900E08F590007003D00EC
:1009F0006000B8006011B8000804500089845800F5
:100A00000A0559008B8559001C002000E00F520098
:100A1000E08F5A00E00F5B00E08F5B0002003D00BA
:100A20000F0007000C00A2000800BE000A01BE0073
:100A30001D0107000203BE000002BE000C00E00022
:100A400001003200060007000400BE000601BE00DF
:100A50004F0678004F05BE004F04BE0000000600A0
:100A60006000B8006011B800040250008582580090
:100A7000060359008783590000000600881F78008C
:100A8000000478005001BE004000BE000400400099
:100A9000858048000601490087814900009CBE000E
:100AA0000294BE000400E1000588E1000690E10028
:100AB0000798E10002003100680044001008E800D7
:100AC0004F04780000000600F4874700889FBE00AE
:100AD0008A9FBE008C9FBE008E1F78000205BE005C
:100AE0000004BE00D4B79F00E5B79F00F6B79F0093
:100AF00087BF9F000000EB00C0B79F00B0B79F000A
:100B0000A0B79F0090B79F0080B79F000D04200002
:100B1000BFB097004FB09700000140000000E00018
:100B20000F003D004F08DE0000007100C0B79F00BD
:100B30009E00070001003D0012002000A1000700F8
:100B400001003D0012002000A6000700B1000700D0
:100B5000B60007000F004000C8FF07002200370062
:100B60004F08DE0000067100CCB79F008F00070021
:100B700001003D00120020009200070001003D002E
:100B80001200200097000700A20007000FB2970094
:100B90009FB297002FB39700BFB39700A90007003B
:100BA0000000520081805A0002015B0083815B00DB
:100BB00080B79F0091B79F00A2B79F00B3B79F0077
:100BC0000007EB009F0007000020E10001A8E10002
:100BD00002B0E10003B8E100010031001E00200076
:100BE0000E005600C0B79F004FB297000400E0000F
:100BF0000700350010002000010020006011B8003F
:100C000008047000898470000A0571008B857100EA
:100C10008D06E900BEFF3A000400E00003003D003D
:100C2000820007000F00400094FF07004FA89700C4
:100C30000000E00004003A000FB497009FB4970052
:100C40002FB59700BFB59700940007004F077800B5
:100C50004F06BE004F05BE004F04BE004F01B1005D
:100C600000000600881F780018002000881F780008
:100C700095FF07008F87E9004F0478000000060009
:100C8000801FEB0090FF07008F87E900000006003F
:100C9000889FBE008A9FBE008C1F78006E000700F0
:100CA00007003D0073000700E00F5B00E08F5B0072
:100CB00007003D00320007000006EB00040037008B
:100CC0003400070002003D002A0007001C0020003D
:100CD00072000700E3FF07000203BE000002BE002F
:100CE0000C00E00001003200220007000400BE00FA
:100CF0000601BE004F0678004F05BE004F04BE003F
:100D000000000600889FBE008A9FBE008C1F7800EE
:100D10005100070005003D0056000700E00F5B0092
:100D2000E08F5B0006003D0004003700190007005B
:100D300003003D006000B8006011B800100007001B
:100D400056000700CEFF07000203BE000002BE00EF
:100D50000C00E00001003200060007000400BE00A5
:100D60000601BE004F0678004F05BE004F04BE00CE
:100D7000000006006000B8006011B80000003700F5
:100D800004025000858258000603590087835900E9
:100D9000000006000006EB00E00F5200E08F5A0052
:100DA000E00F5B00E08F5B00000006000180400068
:100DB00090B79F000001EB008FB097000100E000AA
:100DC000000006000200700090B79F000180400004
:100DD00080B79F000001EB00FFA897000100E00032
:100DE000000006000200700080B79F0001804000F4
:100DF0006FAA9700CF20DE0001007000F0AF9F00C7
:100E000004024200250007004F18DE0000027200B5
:100E100000000600E4AF9F000804440089844C00F1
:100E20000A054D008B854D00000006003FB297007B
:100E3000CFB297005FB39700EFB3970000FE2F008B
:100E4000000006003FB09700CFB097005FB1970059
:100E5000EFB19700000006000205BE000004BE00CE
:100E6000E00F5000E08F5800E00F5900E08F59006C
:100E7000000006006000B8006011B80008045000CF
:100E8000898458000A0559008B8559001C002000F0
:100E9000E00F5200E08F5A00000006000800BE007C
:100EA0000A01BE0000000600889FBE008A9FBE00A7
:100EB0008C9FBE000404B8000506B80089044600F3
:100EC00060854E000606B8000A054600E0854E0023
:100ED0000706B8008B054600040EB80089044600DA
:100EE0000A854E00E0854D00050EB8000A05460053
:100EF0008B854E00060EB8008B0546000416B80020
:100F00000A0546008B854E000516B8008B05460085
:100F1000041EB8008B0546000800BE000A01BE0092
:100F20004F06BE004F05BE004F04BE000000060085
:100F30000400FA00E0BF9F00E48157008129780097
:100F40000002EB000F0037006FB897009040780068
:100F50007FB89700104078000402E80080CF50006E
:100F6000040032008180FB000080FB000080500004
:100F7000070037006FB897000000E800E0BF9F004F
:100F80009309E800820F5200EFFF3A000000EB00E7
:100F90000080FA000000060010417800B1415100C5
:100FA00003003A000000E8000204E000FAFF3A0003
:100FB0000300FB00000006008001780000017800BB
:100FC00031407800005978000004E000FCFF3A004E
:100FD00003007800000006008001EB0002003700EB
:100FE000817178008301E800828F5100FCFF3A0094
:100FF000000006000000FA00CFB897006881570093
:10100000CC0007000080FA00000006008101780093
:101010000000E9000081EB00E50F500004003E00F5
:1010200080004000601B21006081780003B07800E0
:101030000200780000000600000178000000E900CE
:10104000E50F50000F003E0080004000601B2100B3
:10105000E08078000100E00002003A00100020006B
:1010600069030700E18F4000060032000000EB003A
:10107000E18F5000040032000200780001000100FE
:10108000000005000080EB000000060010002000BA
:10109000E9FF0700100020005B0307000C00FA00C6
:1010A000889FBE0000047800CFB09700F0FF2700B3
:1010B000D0BF9F008004EB0099BF9F0088BF9F00B6
:1010C000A8BF9F00200C2000B0BF9F007881570070
:1010D00070805700970007000FB897000948780004
:1010E0000FB8970008045000080078004F04BE00B5
:1010F0000080FA000000060080027800800178007D
:10110000010037008301E8001304E000FDFF3A000E
:101110000002EB00820F52000600320064C078002B
:10112000805978000402E8000004E0000200320068
:10113000F8FF37008049EB0005007800000006004A
:10114000810178000002EB000B003700E4407800DA
:101150000104E000030032000402E80093CF5000D5
:10116000040032008180FB001380FB0000805000EF
:10117000000006008301E800820F5200F3FF3A00EE
:10118000000005000C00FA00A0BF9F00C0BF9F0038
:101190000A000700B0BF9F00F0BF9F00100C2000A6
:1011A000D0BF9F0074815700EFB097006C8057004C
:1011B000450307000080FA00000006008000780068
:1011C0003004E000FEFF3A00010050000000E9009A
:1011D0000000060010417800814F510004003200E9
:1011E0000000E8000204E000FAFF3A000000EB0013
:1011F000000006008001EB000200370061F079007A
:101200008301E800828F5100FCFF3A0000000600D5
:10121000889FBE008A9FBE008000780000C2B30095
:101220000100370089007800810478003944780093
:10123000804F5400FBFF3200E94F5400F9FF3200A9
:10124000D0C2B300804F540004003A001944780023
:101250008184E8001AC0B300060037000045EB00A7
:10126000B0C2B300804F540002003A001944780025
:101270008184E8006022B8000A003700A200200044
:10128000030020000400BE00E7FC07000B414400FF
:101290000281FB000300200000024100818249001E
:1012A000394478000880FB000BFD2F000B00400044
:1012B000E90F5000F1FF36000A04E000020032009E
:1012C00060021200E0821A000400BE004F05BE005A
:1012D0004F04BE0000000600000378008002780082
:1012E000020278008001EB00080037000402E900E8
:1012F00063C07800805A78008301E8000004E000B1
:1013000002003A008000EB0006003700828F510097
:10131000F6FF3A00FBFF37000040EB0080F07A0058
:101320008100E800848F5000FBFF3A00060078003F
:1013300000000600FE874700889FBE008A9FBE000F
:101340008C9FBE008E1F7800F0B79F0001077800C9
:1013500082BF9F000000EB00A0B79F009F023700F4
:101360008006EB0050C2B30080CF5000090032006D
:101370000100FB00FFB09700F4030700E10F4000FD
:1013800096023200AFB097008100E800A1B79F003D
:10139000920237009E407800D0C2B30080CF500048
:1013A0000C00320007003C006D40500080CF500020
:1013B0000A0032006B40400080CF50000E003A001F
:1013C0000800370000C3B30080CF50000A003A0085
:1013D000060037000D30A000050037000D00A0000A
:1013E000030037000D10A000010037000D20A00001
:1013F0000E07E800E7FF37000D18A30001003200D8
:101400000D00A1000D38A300010032000D20A10045
:101410000100FB0002FD2F0002004000E90F500018
:101420000E003E000002EB00C4B79F00820178006E
:10143000CFB297006A28B9001E01FB0000014100ED
:1014400003014100C2B79F005E00FB0003004000A3
:10145000E90F50000B003E00F5FF37000006EB00DF
:10146000CCB79F00A0C2B30080CF500005003A0067
:101470000FB89700C000780080BF9F00C1B79F00E1
:101480000E07E8000001EB00B2B79F00E0C2B30016
:101490009E4F100018003A000DE0A0008E00E800FA
:1014A00064405000914F10000200320001077800A4
:1014B0000C0037000FBA9700C402780084BF9F0069
:1014C000B5B79F000E87E8000B0037003FB69700C6
:1014D0006A60B9000000410003004000B0B79F00FF
:1014E0000E07E8001E01FB0003FD2F000300410072
:1014F000E90F5000F5FF3600BE407800E1D79F00AD
:10150000C0C6B30080CF5000220032000F003C0064
:101510006940500080CF50007700320004003C004A
:101520000104E000310232006B4050000F00370030
:1015300040C6B30080CF50009300320065404000A9
:1015400080CF50008B003A008F00370030C7B300C7
:1015500080CF50001A00320007003C006440500069
:1015600080CF5000110032000040E80080CF5000D2
:1015700080003A000F00370050C7B30080CF500002
:10158000800032006340400080CF500079003A0074
:1015900009003700000028000D48A30001003A00B0
:1015A0000001200080867600D3FF37000D60A00088
:1015B000750037000D50A0000D70A00072003700BC
:1015C0008FB897004100780081BF9F000004780029
:1015D0000000E00001003A00681621008004EB00E2
:1015E000010037008104E800890078000880440089
:1015F0001004E000FBFF3A003FB197000200E0005A
:1016000003003200890F510001003100820478008C
:101610000002EB00E4AF9F00CFB29700898F520029
:101620000200360009805200E0AF9F004368DE00F0
:10163000E10660001B003A000D0678000900370043
:10164000FFB097000002200040030700E10F4000B8
:10165000030032002FB097000000E800A0B79F0001
:101660000C06E800EFA89700810F5600F4FF3A003F
:101670000081EB00E2AF9F000A003700880078008D
:101680003100FB0001047800FFB097002F03070032
:10169000E10F4000030032002FB297000402E8007F
:1016A000A4B79F000900E90080047800E10F400022
:1016B000F2FF3A000006EB000D00E0000A003A00DD
:1016C000C6013700FFB09700000220001F0307008B
:1016D000E10F400003003200AFB297008502E8003E
:1016E000A5B79F000C06E8006FA89700800F560072
:1016F000F4FF3A00B90137008FB897004100780035
:1017000081BF9F00CF80DE00010178008201780058
:101710000205BE000004BE000203BE000002BE00BF
:101720004822DE00482EDD0004027600E4D79F0048
:101730000D48A3000A0032000404E0000800320053
:10174000E14F42000600320071FD2F00018047008A
:101750000448780018409800290020000200370053
:10176000F0D79F001900200072FD2F00028447006F
:10177000A1FF370064FD2F000484470019002000FA
:101780009DFF37000D0CB3000D007800000CB20077
:1017900028003A000D00E00005003D008FBA9700D8
:1017A0004505BE004504BE0085BF9F0014003700FC
:1017B0000D48A3000B0032000FBE97004C00BE0086
:1017C0008CBF9F004F89DE00CF91DE000002BE007B
:1017D00002037800820378000605BE000404BE0000
:1017E000070037008FB897004100780081BF9F0045
:1017F00000047800CFC4DE00090578008A0578006F
:10180000E00F5400E08F5C00E00F5D00E08F5D00B2
:101810001F003D003D00B3006000B8006011B8003B
:1018200008045000898458000A0559008B85590026
:10183000170037000D00E00005003D000FB99700CC
:101840004205BE004204BE0082BF9F001000370068
:101850000D48A300070032000FBA97004400BE00F5
:1018600084BF9F006011B8000205BE000004BE00E6
:10187000070037008FBA97004500780085BF9F00AA
:1018800000047800090020000A0020000B0020005E
:101890003FB697000C00E00007003A00E00F54004C
:1018A000E08F5C00E00F5D00E08F5D0002003A0019
:1018B00010002000B0B79F008D007800010CB2002E
:1018C000E1B79F0000042000808F500030003200FC
:1018D00003003C000100E000080032004000370037
:1018E000000820006FB19700800F510014003200F3
:1018F000000C2000800F510039003A0014C0B300E2
:10190000650C21000B0037000400FB004300DD00E4
:10191000050040005001BE004000BE000040E10054
:1019200001C8E10002D0E10003D8E1002B0039003A
:101930000442E800F44F5200F3FF3A00270037005A
:1019400000012000010020006011B80014C0B300A5
:101950000040E10001C8E10002D0E10003D8E1004D
:101960001E003900450020000000D0008180D20018
:101970000281D2008381D2008502E900FAFF3A0099
:101980000442E800F04F5200F1FF3A001300370024
:1019900080002000010020006011B80014C0B300D6
:1019A0000040E10001C8E10002D0E10003D8E100FD
:1019B0000A0039003C0020000000D0008180D200E5
:1019C0000281D2008381D2000C06E900FAFF3A00BE
:1019D0000442E800F54F5200F1FF3A00E4D79F00BF
:1019E000EFD097000100FB003FB19700820F50003D
:1019F00002003D00E2D79F00040037003FB297008D
:101A0000800F520001003D00B0B79F00CFB2970099
:101A10000500E0000400320063806600020032002E
:101A20008502E900C5B79F000DE8A3000B00320056
:101A30004FB697003FB09700800F560003003C0060
:101A40008000EB00C1B79F00040037004FB1970042
:101A50003FB2970004015100C2B79F00EFD2970038
:101A60000500FB000006EB00DCAF9F00CFB0970045
:101A7000808F50000200340000805000D0AF9F00E3
:101A80000D28A30037003200E18066000D18A30086
:101A90000C003200D00220000100E00001003A00FA
:101AA0000080E900FFB0970028020700E10F400026
:101AB0000E0032002FB197000201E800A2B79F008C
:101AC0000A0037000100E00008003200FFB0970074
:101AD000000220001D020700E10F40000300320059
:101AE0002FB297000402E800A4B79F00DFAA970076
:101AF0000500E0000F0032000006EB00FFB0970089
:101B00000003200011020700E10F40000300320033
:101B10002FB097000000E800A0B79F000C06E80077
:101B2000DFA89700810F5600F4FF3A000001EB0098
:101B3000D2AF9F003FB29700C320DD00E00B210031
:101B40008080400091B79F004220DD00640050007B
:101B500080B79F006320B900F0AF9F00630650007C
:101B600084003700DFAA97000500E0001100320072
:101B7000688066000F003A0000067800FFB097000A
:101B800000022000F1010700E10F400003003200D5
:101B90002FB097000000E800A0B79F000C06E800F7
:101BA000DFA89700810F5600F4FF3A000001EB0018
:101BB000D2AF9F00E18066000D18A3000C00320038
:101BC000D00220000100E00001003A000080E9009E
:101BD000FFB09700DD010700E10F4000D5FF3200A4
:101BE0002FB297000402E800A4B79F00D1FF37008E
:101BF0000100E000CFFF3200FFB09700000220009C
:101C0000D2010700E10F4000CAFF3200AFB29700D7
:101C10008502E800A5B79F00C6FF3700000420003A
:101C2000EFB09700808F50003100320003003C007D
:101C30000100E000080032003E00370000082000EC
:101C40006FB19700800F510011003200000C20008E
:101C5000800F510037003A001FB097003002BE00DD
:101C60002003BE000800BE000A01BE00FDFB070005
:101C7000A4002000050020006033B80000FC07002D
:101C800004C3B30004424000E4D79F00290037009A
:101C9000D5162100D5B79F000D58A30002003A00C9
:101CA000E0172100D0B79F0014002000050020009D
:101CB0006033B8008FB097008100E9000500330061
:101CC0000402D0008582D2000683D2008783D2002E
:101CD000F9FF37000800BE000A01BE00E1FB070063
:101CE0006F0060005FB1970062407800100037001D
:101CF00014002000050020006033B8000C007800BC
:101D00000000E900050033000402D0008582D20003
:101D10000683D2008783D200F9FF37000800BE0097
:101D20000A01BE00CFFB0700674060000043B0001F
:101D3000E0D79F00EFD097000100FB00FFB09700B5
:101D400082010700E10F4000030032002FB197002D
:101D50000201E800A2B79F001FB29700680252007C
:101D600094B79F008FB29700E482520085B79F001E
:101D700063065600D0FF2F003FB197000090B900D6
:101D80007FAA97000000420063005000800F5600B9
:101D9000A2FF3A000D38A30010003200DFAA97001E
:101DA0000500E0000D0034000006EB00FFB09700D6
:101DB0000002200065010700E10F4000030032002F
:101DC0002FB097000000E800A0B79F000C06E800C5
:101DD000DFA89700810F5600F4FF3A00BE4078005C
:101DE000E1D79F000104E0005DFD3A002FB09700AD
:101DF0004F0778004F06BE004F05BE004F04BE00DF
:101E0000EF01B10000000600000478009601070011
:101E10000800780029FA0700889FBE0000047800B7
:101E20008144780000FD2F0000004400E90F5000BD
:101E300002003E00000178000D0037000800780025
:101E4000FFF907000000E0000300320008007800FE
:101E500001FA0700000478000800780005FA07007E
:101E60000000E0000700320090FA2F00000144005B
:101E70000980FB00800F510002003D000280FB0042
:101E800001003700F00F20004F04BE0000000600E4
:101E9000881F7800408E80008101070000047800D0
:101EA000FEF907000000E000FAFF3A00E10F4400ED
:101EB00003003200418E800008007800AC0107006A
:101EC0004F04780000000600EC874700889FBE00A2
:101ED0008A9FBE008C9FBE008E1F780081BF9F002E
:101EE00002077800408E88008046EB00040137002E
:101EF0008884FB0009007800E8F90700800078007A
:101F00000000E00002003200E1FF0700FC003700A3
:101F100050C2B300804F5400F0003A000FBD97004C
:101F200020C0B300C0EF9F00D1EF9F0081EF9F0062
:101F30000300370040C0B300C0EF9F000FBD970003
:101F40000FB99700B240780082BF9F008184FB00E8
:101F500090C6B30080CF50003500320017003E001D
:101F60006640500080CF5000620032000C003E00FE
:101F70007740500080CF50002800320006003E001D
:101F80000104E0009B003200A0C2B30080CF5000EB
:101F90006E003A001D00370080C5B3001600370000
:101FA00040C6B30080CF50002100320064404000A2
:101FB00080CF500065003A001200370030C7B300F0
:101FC00080CF50001E00320007003E0067405000E6
:101FD00080CF5000110032006340400080CF50009D
:101FE0005A003A001400370050C7B30080CF5000A9
:101FF0000F0032006340400080CF500053003A0091
:102000006500370020C0B300CBFF3700DFE8970042
:102010008140E800D1EF9F00C8FF37004FE99700EB
:1020200080C0B300E24F5100C3FF3A00C1FF370048
:10203000ACC0B300590037008CC0B3005700370064
:1020400093FF0700DFE897000104E00002003A0078
:102050004E017800D2B79F00408E8000100107002B
:1020600000047800E10F4000A20032008FEC9700DE
:10207000120037000A85E8008ABF9F00160037006B
:102080008FB897001100FB00800F5400F9FF320059
:102090005FE997000204E00003003A005FB0970098
:1020A00008587800D0B79F008944E9000A00320040
:1020B000408E8000FA000700000478000800E80065
:1020C000E10F5000040036000800780073F90700A3
:1020D0000000E000EAFF3200DFE897000104E000C2
:1020E00087003A008D46E8005FB19700014978000B
:1020F000830037005FE897000004E00003003A0027
:102100008D46E800CE007800D1B79F00408E800059
:10211000E3000700E10F4000760032005FE997001E
:102120000204E00003003A00DFB097008058780016
:10213000D1B79F000FE997000241E90082EF9F00AD
:102140004240A9006E003400F0FF37000180FB0020
:1021500008FD2F0008004000E90F50005F003E001E
:102160000A0078001F01070080EF9F0088007800B8
:10217000030037000FB897000000E80080BF9F0001
:102180000FB997001200FB0001004000E90F50005A
:10219000F8FF360069FF37000CC1B3003CFF0700B1
:1021A000408E8000BE000700000578000040EB0074
:1021B000E0EF9F00D0022000800F550005003A009C
:1021C000408E8000B60007000005780011C0B30003
:1021D000E1EF9F008C4078000A0078000EFF0700B6
:1021E000E14F40000A003A00418E80000A0078006A
:1021F000DF0007000D04E0004B003A00408E800035
:10220000300090000048A30043003200480037002F
:102210008FED97006044B8000C81FB0003002000A4
:102220000800BE0000F907000004BE008C407800E2
:102230000A007800F8FE07000080FB000100200083
:1022400008044000898448008B45E90007003200FB
:10225000408E800092000700000578008C407800D6
:10226000EDFE0700E14F4000EBFF3A008C407800A4
:102270000A007800E8FE0700E14F400003003A0042
:10228000418E80000A007800B90007006FE99700CE
:102290000204E0000200320060041400E0841C002C
:1022A0005FE897000004E00015003A008D46E80062
:1022B000CFE89700E4CF500003003A004E007800CA
:1022C0000888BE000E0037000E81E9000207780082
:1022D000120078000808780009003700408E80005E
:1022E0006F000700808F540005003200E10F4000AE
:1022F0000B003A000D04E0000D0032000A00370028
:102300008FB897003144780081BF9F000804E00037
:10231000F7FE3A00040037000000EB00050037002C
:10232000418E8000920007000D80FB000100370005
:102330000080EB004F0778004F06BE004F05BE003F
:102340004F04BE00CF00B10000000600889FBE0011
:102350000001780001047800B10090000118A3008A
:102360003D0032000198A30003003A0018009000DD
:102370000000E00038003A000190A000310498000D
:1023800082047800F90FB200180090000000E0000D
:1023900002003A0028009000000C7800EA8F5400F8
:1023A00006003A00380090000078A30003003A00CD
:1023B00088007800D0002000E4FF0700980090001B
:1023C00058009000808F50000B0032000100E800A0
:1023D000100498001800780009587800000C780064
:1023E00011C0B300601C210001487800EA8F54003E
:1023F0000600320019003700880078000940780094
:102400009C0007008004780014003700380090001A
:102410000088A3001100320018019000A80090006D
:1024200048009000ADF8070098009000810F500020
:1024300004003200380090000003B300300498001C
:102440008084EB000000EB0010049800280090004E
:10245000000C7800010037008084EB000900780050
:102460004F04BE0000000600881F7800508E8000D8
:102470000000E000010032000000010028192100E6
:1024800008007800BE0007006C044400601B2100B7
:10249000800F5400FAFF3A004F0478000000060055
:1024A000881F780000047800B00090000148A30065
:1024B00007003A000108A300050032000198A300BC
:1024C00008003200100090000000E000050032001B
:1024D000380090000040A000300498008080EB009D
:1024E000200037000190A1003104980018009000EE
:1024F0000000E000060034000000E900100498002D
:1025000018007800B080FB00000C7800060037004F
:10251000380090000068A300EDFF3A000800780042
:10252000CF00070080007800380090000078A300FA
:102530000C003A00FA8F500008003A002800900082
:102540000000E000E2FF3200180090000000E80008
:1025500010049800180CE900DDFF3700ED8F5000E3
:10256000E2FF3200010078004F047800000006000E
:1025700080017800E10F4000170032003100900028
:102580000008A300140032000098A30012003A00D3
:10259000210290000400E0000F00320011019000C1
:1025A00051009000800F51000B00320011007800A4
:1025B000840F500002003A008008E8000200370053
:1025C0000200E800900098001100E90080087800FF
:1025D00003487800010037008081EB000300780099
:1025E000000006000001780000C2B30001003700BF
:1025F0000201E8009240780080CF5000FCFF3200DA
:10260000E9CF5000FAFF3200D0C2B30080CF5000B3
:1026100003003A000201E80014C0B30005003700CF
:102620000042EB00B0C2B30080CF500001003A007E
:102630000201E8008000EB0005FD2F0004003700D8
:102640006A08B90000804100850040000201E800EE
:102650009201FB0005804100E90F5000F8FF3600B1
:102660000404E000010032008100EA00010078006B
:10267000000006000200FA00889FBE00A0FF9F0035
:1026800001047800B1009000810478000904B200D0
:10269000020032000000FB00360037000118A300E2
:1026A00005003A000103B3003104980019049800B2
:1026B0000080EB002F003700580090000000E00081
:1026C00006003A004800900012002000E680570003
:1026D00002F8070019049800240037002800900031
:1026E0000000E00008003A00201C210020049800AF
:1026F000000C78002000200050049800100498007E
:102700000130A0003104980018019000A80090004A
:1027100048009000F1F7070028009000000C7800B6
:102720000080EB001004980018007800AFF89700C4
:1027300001587800000C78002FF89700EA4F5000FD
:102740000A003A00380090000088A3000700320019
:1027500018019000A800900048009000DFF70700E3
:1027600019049800A8009000010C7800AFF89700B9
:102770000100FB004F04BE000080FA0000000600CC
:10278000889FBE008A1F7800000478003000900007
:102790006300600024003200080078007E0007001B
:1027A0003805900080EF2F0000006500300498008D
:1027B000280090000000E00004003200E8046500FA
:1027C00002003A00AD00070029049800480090007C
:1027D000F9F70700E10F400013003200B800900045
:1027E0000102B20010003A000AC8A300180032002B
:1027F000708E80000000E0001500320000017800BB
:1028000081047800012A200012289000880F5000CF
:10281000070032004205B0004905B000818F540026
:102820000B003200F8FF37000080EB000900370092
:1028300002007800E9F70700708E80000900400070
:102840008000EB001128980001007800010037009B
:102850000000EB004F0578004F04BE0000000600AA
:102860000200FA00889FBE008A1F780000047800EA
:102870000000EB0010049800380090008080EB000E
:102880000008A3003F003200601C21001004E0009B
:1028900010003200291921008A1921001A0078003D
:1028A0006C0545002010B20021102000810F50005F
:1028B00002003A000900780037000700EC84440069
:1028C000601B2100808F5400F4FF3A00601C21003F
:1028D0000048EB0048009000580190000200E00022
:1028E0000D003A001204980012002000E880570002
:1028F000C3F70700E10F500003003A000FF89700FC
:102900008080FB001F003700380090000040A000CE
:102910003004980012003700A8009000B8F70700B4
:10292000100498000000E00003003200E10F4000B6
:102930000D003A0003003700380090000040A0006E
:1029400002003700380090000003B3003004980004
:10295000A8009000010C78000000EB001004980023
:102960008080EB0007003700A8009000010C780081
:102970000000E9001004980001007800B080FB001E
:10298000000C7800010078004F0578004F04BE006D
:102990000080FA0000000600881F7800000478001C
:1029A000300090000008A30007003200800078008B
:1029B0000120B20004003A0011049800A800900021
:1029C000010C7800170037000018A300190032002E
:1029D0000098A30017003200A80090000100E0005A
:1029E00014003200180190000200E00011003200D3
:1029F0004800900039F7070098009000810F5000C0
:102A000003003200380090000003B3003004980047
:102A10000000EB001004980028009000000C7800E3
:102A2000380090000058A300020032000080EB0044
:102A3000010037000000EB004F04780000000600A2
:102A4000618E80000100E000030032001100780078
:102A5000608E88000300370020002000A1F70700E7
:102A600080007800E18F400002003A00906E26005E
:102A7000808E88000100780000000600618E8000D2
:0C2A800001087800608E8800000006004D
:020000040000FA
:0200000401F009
:04000C00FBFF0000F6
:020000040000FA
:0200000401F009
:04001000FDFF0000F0
:020000040000FA
:0200000401F009
:040014007FFF00006A
:020000040000FA
:1000080010030000B2A100007AA1000096A1000030
:10001800CEA10000EAA100001003000010030000B8
:100028001003000010030000100300009CBE000035
:10003800100300001003000010030000100300006C
:1000480022A20000100300001003000052B80000B4
:10005800100300001003000010030000100300004C
:10006800100300001003000010030000100300003C
:10007800100300001003000010030000100300002C
:1000880010030000100300001003000050B500002A
:100098007EB40000100300001003000010030000ED
:1000A80010030000100300001003000010030000FC
:1000B80010030000100300001003000010030000EC
:1000C80010030000100300001003000010030000DC
:1000D800100300001003000006A200001003000037
:1000E80010030000100300001003000010030000BC
:1000F80010030000100300001003000010030000AC
:10010800100300001003000010030000100300009B
:10011800100300001003000010030000100300008B
:10012800100300001003000010030000100300007B
:10013800100300001003000010030000100300006B
:10014800100300001003000010030000100300005B
:10015800100300001003000010030000100300004B
:10016800100300001003000010030000100300003B
:10017800100300001003000010030000100300002B
:10018800100300001003000010030000100300001B
:10019800100300001003000010030000100300000B
:1001A80010030000100300001003000010030000FB
:1001B80010030000100300001003000010030000EB
:1001C80010030000100300001003000010030000DB
:1001D80010030000100300001003000010030000CB
:1001E80010030000100300001003000010030000BB
:0801F8001003000010030000D9
:020000040000FA
:1002080010030000B2A100007AA1000096A100002E
:10021800CEA10000EAA100001003000010030000B6
:100228001003000010030000100300009CBE000033
:10023800100300001003000010030000100300006A
:1002480022A20000100300001003000052B80000B2
:10025800100300001003000010030000100300004A
:10026800100300001003000010030000100300003A
:10027800100300001003000010030000100300002A
:1002880010030000100300001003000050B5000028
:100298007EB40000100300001003000010030000EB
:1002A80010030000100300001003000010030000FA
:1002B80010030000100300001003000010030000EA
:1002C80010030000100300001003000010030000DA
:1002D800100300001003000006A200001003000035
:1002E80010030000100300001003000010030000BA
:1002F80010030000100300001003000010030000AA
:100308001003000010030000100300001003000099
:100318001003000010030000100300001003000089
:100328001003000010030000100300001003000079
:100338001003000010030000100300001003000069
:100348001003000010030000100300001003000059
:100358001003000010030000100300001003000049
:100368001003000010030000100300001003000039
:100378001003000010030000100300001003000029
:100388001003000010030000100300001003000019
:100398001003000010030000100300001003000009
:1003A80010030000100300001003000010030000F9
:1003B80010030000100300001003000010030000E9
:1003C80010030000100300001003000010030000D9
:1003D80010030000100300001003000010030000C9
:1003E80010030000100300001003000010030000B9
:0803F8001003000010030000D7
:020000040000FA
:102A8C0074650000787400002F7000006C61000009
:102A9C00696E00000074000065780000742F00005F
:102AAC00687400006D6C0000007400006578000014
:102ABC00742F0000786D00006C000000746500003D
:102ACC00787400002F63000073730000006900002D
:102ADC006D610000676500002F67000069660000EB
:102AEC00006900006D610000676500002F70000038
:102AFC006E670000006900006D61000067650000F2
:102B0C002F6A000070650000670000006170000013
:102B1C00706C00006963000061740000696F000054
:102B2C006E2F00006A610000766100002D760000B7
:102B3C006D00000061750000646900006F2F0000DB
:102B4C00782D000077610000766500000000000021
:102B5C0046950000519500005195000051950000DC
:102B6C005B950000649500006D9500007795000062
:102B7C00819500008C950000A0950000AD9500009B
:102B8C000D0A00000048000054540000502F0000B3
:102B9C00312E0000312000003230000030200000C7
:102BAC004F4B00000D0A0000436F00006E6E0000DA
:102BBC0065630000746900006F6E00003A2000002D
:102BCC00636C00006F730000650D00000A000000CC
:102BDC0048540000545000002F3100002E310000EA
:102BEC0020340000303000002042000061640000FE
:102BFC0020520000657100007565000073740000C0
:102C0C000D0A0000436F00006E6E0000656300004B
:102C1C00746900006F6E00003A200000636C0000C5
:102C2C006F730000650D00000A0D00000A340000EF
:102C3C00303000002042000061640000205200008F
:102C4C006571000075650000737400003A20000087
:102C5C00636100006E2700007420000068610000B2
:102C6C006E6400006C650000204300006F6E000075
:102C7C00746500006E7400002D4C0000656E000041
:102C8C0067740000680D00000A0000004854000042
:102C9C00545000002F3100002E3100002034000071
:102CAC0030310000205500006E610000757400008A
:102CBC00686F0000726900007A650000640D000006
:102CCC000A570000575700002D4100007574000092
:102CDC00686500006E740000696300006174000098
:102CEC00653A000020420000617300006963000037
:102CFC0020720000656100006C6D00003D22000038
:102D0C00507200006F740000656300007465000071
:102D1C00642200000D0A0000436F00006E6E00007C
:102D2C0065630000746900006F6E00003A200000BB
:102D3C00636C00006F730000650D00000A0D00004D
:102D4C000A34000030310000205500006E61000094
:102D5C0075740000686F0000726900007A650000ED
:102D6C00643A00002050000061730000737700008B
:102D7C006F72000064200000726500007175000025
:102D8C0069720000656400000D0A00000048000034
:102D9C0054540000502F0000312E00003120000050
:102DAC0034300000342000004E6F0000742000000E
:102DBC00666F0000756E0000640D00000A43000091
:102DCC006F6E00006E65000063740000696F000098
:102DDC006E3A0000206300006C6F00007365000009
:102DEC000D0A0000436F00006E740000656E000059
:102DFC00742D000054790000706500003A2000002A
:102E0C0074650000787400002F680000746D000079
:102E1C006C0D00000A0D00000A3400003034000074
:102E2C003A200000466900006C650000206E00002E
:102E3C006F740000206600006F7500006E64000067
:102E4C003C620000723E00005573000065200000DB
:102E5C003C6100002068000072650000663D0000C7
:102E6C00222F0000757000006C6F00006164000080
:102E7C00223E00004D50000046530000205500003B
:102E8C00706C00006F610000643C00002F6100005A
:102E9C003E200000746F000020700000726F000074
:102EAC0067720000616D0000207700006562000011
:102EBC002070000061670000657300000D0A0000BF
:102ECC000048000054540000502F0000312E000028
:102EDC003120000034310000342000005265000025
:102EEC007175000065730000742D000055520000D0
:102EFC0049200000546F00006F2000004C6F000050
:102F0C006E6700000D0A0000436F00006E6E00003B
:102F1C0065630000746900006F6E00003A200000C9
:102F2C00636C00006F730000650D00000A0D00005B
:102F3C000A3400003134000020520000657100009A
:102F4C0075650000737400002D5500005249000097
:102F5C00205400006F6F0000204C00006F6E0000CA
:102F6C00673A0000204200007566000066650000AC
:102F7C00722000006F76000065720000666C000025
:102F8C006F7700002064000065740000656300002A
:102F9C0074650000640D00000A0000004854000035
:102FAC00545000002F3100002E310000203500005D
:102FBC0030300000204900006E7400006572000083
:102FCC006E6100006C2000005365000072760000FA
:102FDC006572000020450000727200006F720000E4
:102FEC000D0A0000436F00006E6E00006563000068
:102FFC00746900006F6E00003A200000636C0000E2
:10300C006F730000650D00000A0D00000A3500000A
:10301C0030300000204900006E7400006572000022
:10302C006E6100006C200000536500007276000099
:10303C006572000020450000727200006F72000083
:10304C003A200000457800007065000063740000B1
:10305C0065640000206400006174000061200000C1
:10306C006E6F000074200000707200006573000029
:10307C00656E0000740D00000A000000485400004A
:10308C00545000002F3100002E310000203500007C
:10309C0030310000204E00006F7400002049000009
:1030AC006D7000006C6500006D6500006E740000B2
:1030BC00656400000D0A0000436F00006E6E000096
:1030CC0065630000746900006F6E00003A20000018
:1030DC00636C00006F730000650D00000A0D0000AA
:1030EC000A35000030310000204E00006F740000E3
:1030FC00204900006D7000006C6500006D650000DB
:10310C006E740000656400003A2000004F6E0000F1
:10311C006C7900002047000045540000206100003D
:10312C006E640000205000004F530000542000003B
:10313C0073750000707000006F7200007465000001
:10314C00640D00000A0000004854000054500000B8
:10315C002F3100002E3100002032000030300000F2
:10316C00204F00004B0D00000A4300006F6E000062
:10317C006E65000063740000696F00006E3A000019
:10318C00206300006C6F0000736500000D0A0000E6
:10319C00436F00006E740000656E0000742D00001B
:1031AC0054790000706500003A200000746500003E
:1031BC00787400002F680000746D00006C0D000026
:1031CC000A0D00000A3C0000687400006D6C0000E1
:1031DC003E3C0000626F0000647900002073000028
:1031EC00747900006C6500003D2200006D610000E8
:1031FC0072670000696E00003A3100003030000048
:10320C0070780000223E00003C6600006F720000E7
:10321C006D2000006D650000746800006F64000094
:10322C003D7000006F7300007420000061630000AB
:10323C00746900006F6E00003D2200002F750000C5
:10324C00706C00006F6100006422000020650000BB
:10325C006E63000074790000706500003D22000070
:10326C006D7500006C7400006970000061720000E4
:10327C00742F0000666F0000726D00002D6400005A
:10328C0061740000612200003E3C0000623E0000C0
:10329C004D50000046530000204900006D610000B5
:1032AC006765000020550000706C00006F61000025
:1032BC00643C00002F6200003E3C0000703E0000A9
:1032CC003C6900006E7000007574000020740000F2
:1032DC0079700000653D0000666900006C650000B7
:1032EC00206E0000616D0000653D0000692000004B
:1032FC00736900007A6500003D340000303E000028
:10330C00202600006E620000737000003B2000005D
:10331C003C6900006E7000007574000020740000A1
:10332C0079700000653D000073750000626D00004F
:10333C006974000020760000616C00007565000067
:10334C003D220000557000006C6F000061640000AD
:10335C00223E00003C2F0000666F0000726D0000E2
:10336C003E3C00002F6200006F640000793E0000BC
:10337C003C2F0000687400006D6C00003E000000E3
:10338C0048540000545000002F3100002E31000032
:10339C002032000030300000204F00004B0D0000A8
:1033AC000A4300006F6E00006E650000637400003D
:1033BC00696F00006E3A0000206300006C6F000023
:1033CC00736500000D0A0000436F00006E7400006E
:1033DC00656E0000742D00005479000070650000CB
:1033EC003A20000074650000787400002F6800001B
:1033FC00746D00006C0D00000A0D00000A3C00000A
:10340C00687400006D6C00003E3C0000626F0000B0
:10341C006479000020730000747900006C65000072
:10342C003D2200006D61000072670000696E0000B3
:10343C003A3100003030000070780000223E00006D
:10344C003C6200003E4D000050460000532000003E
:10345C00557000006461000074650000205300008A
:10346C0075630000636500007373000066750000EF
:10347C006C3C00002F6200003E3C0000703E0000DF
:10348C003C6100002068000072650000663D000091
:10349C00222F0000223E00005369000074650000DA
:1034AC00206D0000616900006E200000706100005A
:1034BC00676500003C2F0000613E00003C2F0000BF
:1034CC00626F0000647900003E3C00002F68000031
:1034DC00746D00006C3E0000004800005454000065
:1034EC00502F0000312E000031200000353000003C
:1034FC0030200000496E000074650000726E000000
:10350C00616C0000205300006572000076650000BD
:10351C007220000045720000726F0000720D0000F6
:10352C000A4300006F6E00006E65000063740000BB
:10353C00696F00006E3A0000206300006C6F0000A1
:10354C00736500000D0A0000436F00006E740000EC
:10355C00656E0000742D0000547900007065000049
:10356C003A20000074650000787400002F68000099
:10357C00746D00006C0D00000A0D00000A3C000088
:10358C00687400006D6C00003E3C0000626F00002F
:10359C006479000020730000747900006C650000F1
:1035AC003D2200006D61000072670000696E000032
:1035BC003A3100003030000070780000223E0000EC
:1035CC003C6200003E4D00005046000053200000BD
:1035DC00496D00006167000065200000436F00002A
:1035EC007272000075700000742000006F72000091
:1035FC0020570000726F00006E670000205600001C
:10360C0065720000736900006F6E00003C2F0000B3
:10361C00623E00003C7000003E3C00006120000057
:10362C0068720000656600003D2200002F750000E6
:10363C00706C00006F610000642200003E540000BA
:10364C00727900002061000067610000696E000063
:10365C003F3C00002F6100003E3C00002F62000048
:10366C006F640000793E00003C2F0000687400007D
:10367C006D6C00003E0000004854000054500000E7
:10368C002F3100002E3100002033000030320000BA
:10369C00204600006F7500006E6400000D0A0000EB
:1036AC00436F00006E6E00006563000074690000DB
:1036BC006F6E00003A200000636C00006F73000016
:1036CC00650D00000A4C00006F630000617400007F
:1036DC00696F00006E3A00002000000048540000A2
:1036EC00545000002F3100002E3100002034000017
:1036FC0030330000204600006F7200006269000049
:10370C0064640000656E00000D0A0000436F000049
:10371C006E6E000065630000746900006F6E00003F
:10372C003A200000636C00006F730000650D000010
:10373C000A0D00000A34000030330000204600005F
:10374C006F7200006269000064640000656E000026
:10375C003A200000535300004C200000526500003A
:10376C00717500006972000065640000202D000076
:10377C0020750000736500002048000054540000C0
:10378C00505300000D0A000000000000C995000015
:10379C00C9950000EE9500004C960000CD960000F7
:1037AC0067970000D497000044980000AA98000086
:1037BC00AD950000C6990000739A0000429B000072
:1037CC00749B0000436F00006F6B00006965000084
:1037DC003A00000041750000746800006F72000030
:1037EC00697A000061740000696F00006E3A000095
:1037FC00004300006F6E0000746500006E740000E2
:10380C002D4C0000656E000067740000683A0000E3
:10381C0000000000E89B0000F09B0000FF9B0000F4
:10382C007478000074000000687400006D000000E3
:10383C00687400006D6C0000006300006769000094
:10384C00007800006D6C00000063000073730000D2
:10385C000067000069660000007000006E670000E1
:10386C00006A000070670000006300006C610000DB
:10387C0000770000617600000000000000000000EE
:10388C0000000000169C00001A9C00001E9C00000A
:10389C00239C0000279C00002B9C00002F9C000008
:1038AC00339C0000379C00003B9C00003F9C0000B8
:1038BC00439C0000686500006164000065720000B4
:1038CC002E6900006E630000006600006F6F000040
:1038DC0074650000722E0000696E00006300000029
:1038EC0021440000454600000047000045540000FC
:1038FC00005000004F530000540000007570000091
:10390C006C6F0000616400000073000077690000B8
:10391C0074630000682E0000687400006D000000E5
:10392C000D0A00000D0A0000000D00000A0D000039
:10393C000A4D000050460000530200000100000038
:10394C000D0A00000D0A0000333000003420000086
:10395C005265000064690000726500006374000029
:10396C003A200000004300006F6E000074650000F8
:10397C006E7400002D54000079700000653A000050
:10398C0020000000436F00006E740000656E0000A4
:10399C00742D0000456E0000636F00006469000028
:1039AC006E6700003A200000677A00006970000022
:1039BC000D0A000000430000616300006865000010
:1039CC002D4300006F6E0000747200006F6C0000DD
:1039DC003A200000006E00006F2D000063610000B3
:1039EC0063680000650000006D610000782D000028
:1039FC0061670000653D00000036000030300000BB
:103A0C0000530000657400002D4300006F6F000030
:103A1C006B690000653A0000200000000000000007
:103A2C00000000000000000000000000000000008A
:103A3C00000000000000000000000000000000007A
:103A4C00000000000000000000000000000000006A
:103A5C00000000000000000000000000000000005A
:103A6C00000000000000000000000000000000004A
:103A7C00000000000000000000000000000000003A
:103A8C00000000000000000000000000000000002A
:103A9C00000000000000000000000000000000001A
:103AAC00000000000000000000000000000000000A
:103ABC0000000000000000000000000000000000FA
:103ACC0000000000000000000000000000000000EA
:103ADC0000000000000000000000000000000000DA
:103AEC0000000000000000000000000000000000CA
:103AFC0000000000000000000000000000000000BA
:103B0C0000000000000000000000000000000000A9
:103B1C000000000000000000000000000000000099
:103B2C000000000000000000000000000000000089
:103B3C000000000000000000000000000000000079
:103B4C000000000000000000000000000000000069
:103B5C000000000000000000000000000000000059
:103B6C000000000000000000000000000000000049
:103B7C000000000000000000000000000000000039
:103B8C000000000000000000000000000000000029
:103B9C000000000000000000000000000000000019
:103BAC000000000000000000000000004375000051
:103BBC0072720000656E00007420000053740000E7
:103BCC0065700000203D0000202500006C75000091
:103BDC000054000061720000676500007420000052
:103BEC005374000065700000203D0000202500008B
:103BFC006C750000004300007572000072650000D7
:103C0C006E740000205000006F72000074200000E1
:103C1C003D2000002575000000540000617200007A
:103C2C006765000074200000506F00007274000083
:103C3C00203D0000202500007500000049730000A5
:103C4C00204D00006F760000696E000067200000B8
:103C5C003D20000025750000004900007320000085
:103C6C00486F00006D6900006E670000203D000089
:103C7C00202500007500000049730000204800005A
:103C8C006F6D000065640000203D000020250000E1
:103C9C00750000004D610000676E00006574000047
:103CAC002031000020530000746100007465000096
:103CBC00203D000020250000750000004D61000033
:103CCC00676E000065740000203200002053000075
:103CDC007461000074650000203D00002025000088
:103CEC00750000004D610000676E000065740000F7
:103CFC00205000006F73000069740000696F0000B1
:103D0C006E2000003D200000256C000075000000B6
:103D1C000000000000000000000000000000000097
:103D2C000000000000000000000000000000000087
:103D3C000000000000000000000000000000000077
:103D4C000000000000000000000000000000000067
:103D5C000000000000000000000000000000000057
:103D6C000000000000000000000000000000000047
:103D7C000000000000000000000000000000000037
:103D8C000000000000000000000000000000000027
:103D9C000000000000000000000000000000000017
:103DAC000000000000000000000000000000000007
:103DBC0000000000000000000000000000000000F7
:103DCC0000000000000000000000000000000000E7
:103DDC0000000000000000000000000000000000D7
:103DEC0000000000000000000000000000000000C7
:103DFC0000000000000000000000000000000000B7
:103E0C0000000000000000000000000000000000A6
:103E1C000000000000000000000000000000000096
:103E2C000000000000000000000000000000000086
:103E3C000000000000000000000000000000000076
:103E4C000000000000000000000000000000000066
:103E5C000000000000000000000000000000000056
:103E6C000000000000000000000000000000000046
:103E7C000000000000000000000000000000000036
:103E8C000000000000000000000000000000000026
:103E9C000000000000000000000000000000000016
:103EAC004E690000636B00006E6100006D650000E0
:103EBC00203D000020250000730000004C45000050
:103ECC004420000042720000696700006874000022
:103EDC006E65000073730000203D0000202500007B
:103EEC00750000004D610000782000005374000044
:103EFC0065700000732000003D200000256C000060
:103F0C0075000000446500007669000063650000E0
:103F1C002054000079700000652000003D20000056
:103F2C0025730000004800006F6D00006520000044
:103F3C004F6E00002053000074610000727400008A
:103F4C00203D000020250000750000004D610000A0
:103F5C0078200000537000006565000064200000AC
:103F6C003D2000002575000000000000000000004E
:103F7C000000000000000000000000000000000035
:103F8C000000000000000000000000000000000025
:103F9C000000000000000000000000000000000015
:103FAC000000000000000000000000000000000005
:103FBC0000000000000000000000000000000000F5
:103FCC0000000000000000000000000000000000E5
:103FDC0000000000000000000000000000000000D5
:103FEC0000000000000000000000000000000000C5
:103FFC0000000000000000000000000000000000B5
:10400C0000000000000000000000000000000000A4
:10401C000000000000000000000000000000000094
:10402C000000000000000000000000000000000084
:10403C000000000000000000000000000000000074
:10404C000000000000000000000000000000000064
:10405C000000000000000000000000000000000054
:10406C000000000000000000000000000000000044
:10407C000000000000000000000000000000000034
:10408C000000000000000000000000000000000024
:10409C000000000000000000000000000000000014
:1040AC000000000000000000000000000000000004
:1040BC0000000000000000000000000000000000F4
:1040CC0000000000000000000000000000000000E4
:1040DC0000000000000000000000000000000000D4
:1040EC0000000000000000000000000000000000C4
:1040FC0000000000000000000000000000000000B4
:10410C0000000000000000000000000000000000A3
:10411C000000000000000000000000000000000093
:10412C000048000069670000682000005370000020
:10413C0065650000642000003D200000257500002E
:10414C000044000065660000617500006C7400009E
:10415C0020480000696700006820000053700000D0
:10416C0065650000642000003D20000025750000FE
:10417C00004C00006F7700002053000070650000B9
:10418C0065640000203D0000202500007500000043
:10419C004465000066610000756C0000742000002E
:1041AC004C6F000077200000537000006565000024
:1041BC00642000003D20000025750000004D00002B
:1041CC006F760000696E00006720000043750000E8
:1041DC0072720000656E0000742000003D2000002B
:1041EC002575000000440000656600006175000044
:1041FC006C740000204D00006F760000696E0000AA
:10420C00672000004375000072720000656E0000AC
:10421C00742000003D2000002575000000480000BF
:10422C006F6C0000646900006E67000020430000A2
:10423C0075720000726500006E740000203D000075
:10424C002025000075000000446500006661000038
:10425C00756C000074200000486F00006C64000056
:10426C00696E000067200000437500007272000048
:10427C00656E0000742000003D20000025750000D4
:10428C00004D0000617800002043000075720000B2
:10429C00726500006E740000203D000020250000B7
:1042AC0075000000705F000061700000705F00001E
:1042BC00636F00006E660000696700000073000009
:1042CC00726300002F480000756200002F48000048
:1042DC00756200002E63000000250000733A000098
:1042EC002569000020250000732000002D2D000002
:1042FC002061000073730000657200007469000097
:10430C006F6E000020660000616900006C650000A3
:10431C00640A000000000000000000000000000023
:10432C000000000000000000000000000000000081
:10433C000000000000000000000000000000000071
:10434C000000000000000000000000000000000061
:10435C000000000000000000000000000000000051
:10436C000000000000000000000000000000000041
:10437C000000000000000000000000000000000031
:10438C000000000000000000000000000000000021
:10439C000000000000000000000000000000000011
:1043AC000000000000000000000000000000000001
:1043BC0000000000000000000000000000000000F1
:1043CC0000000000000000000000000000000000E1
:1043DC0000000000000000000000000000000000D1
:1043EC0000000000000000000000000000000000C1
:1043FC0000000000000000000000000000000000B1
:10440C0000000000000000000000000000000000A0
:10441C000000000000000000000000000000000090
:10442C000000000000000000000000000000000080
:10443C000000000000000000000000000000000070
:10444C000000000000000000000000000000000060
:10445C000000000000000000000000000000000050
:10446C000000000000000000000000000000000040
:10447C000000000000000000000000000000000030
:10448C000000000000000000000000000000000020
:10449C000000000000000000000000000000000010
:1044AC000000000000460000697200006D770000FB
:1044BC0061720000652000005665000072730000F8
:1044CC00696F00006E2000003D2000002575000083
:1044DC002E250000752E00002575000000430000FD
:1044EC006F6D00006D6100006E64000020560000CE
:1044FC0065720000736900006F6E0000203D0000C3
:10450C0020250000752E0000257500002E250000CA
:10451C007500000032300000313700002F310000F0
:10452C00312F00003231000000520000656C000099
:10453C006561000073650000204400006174000098
:10454C00652000003D200000257300000053000092
:10455C0065720000696100006C2000004E7500005F
:10456C006D62000065720000203D000020250000F7
:10457C00750000005769000072650000642000009F
:10458C0049500000203D000020250000642E000052
:10459C00256400002E250000642E00002564000018
:1045AC0000000000000000000000000000000000FF
:1045BC0000000000000000000000000000000000EF
:1045CC0000000000000000000000000000000000DF
:1045DC0000000000000000000000000000000000CF
:1045EC0000000000000000000000000000000000BF
:1045FC0000000000000000000000000000000000AF
:10460C00000000000000000000000000000000009E
:10461C00000000000000000000000000000000008E
:10462C00000000000000000000000000000000007E
:10463C00000000000000000000000000000000006E
:10464C00000000000000000000000000000000005E
:10465C00000000000000000000000000000000004E
:10466C00000000000000000000000000000000003E
:10467C00000000000000000000000000000000002E
:10468C00000000000000000000000000000000001E
:10469C00000000000000000000000000000000000E
:1046AC0000000000000000000000000000000000FE
:1046BC0000000000000000000000000000000000EE
:1046CC0000000000000000000000000000000000DE
:1046DC0000000000000000000000000000000000CE
:1046EC0000000000000000000000000000000000BE
:1046FC0000000000000000000000000000000000AE
:10470C00000000000000000000000000000000009D
:10471C00000000000000000000000000000000008D
:10472C00000000000000000000000000000000007D
:10473C0000500000726900006D6100007279000089
:10474C00204400004E530000203D000020250000B6
:10475C00642E0000256400002E250000642E00004D
:10476C0025640000004E000065740000776F0000A7
:10477C00726B000020430000616200006C65000059
:10478C00204300006F6E00006E6500006374000033
:10479C0065640000203D000020250000640000003E
:1047AC0044480000435000002043000068610000B2
:1047BC006E67000065640000203D000020250000AD
:1047CC00640000004D4100004320000046720000D0
:1047DC006565000020520000782000003D2000009C
:1047EC0025640000004D00004143000020490000FA
:1047FC007320000054780000205200006561000016
:10480C0064790000203D00002025000064000000B9
:10481C0052650000636F00006E6E0000656300005F
:10482C0074200000436F0000756E000074200000BF
:10483C003D200000256400000000000054680000CA
:10484C006973000020760000657200007369000037
:10485C006F6E0000206F000066200000746800007E
:10486C006520000046690000726D00007761000051
:10487C0072650000206400006F650000732000006A
:10488C006E6F0000742000007375000070700000E3
:10489C006F7200007420000063680000616E0000FD
:1048AC00676900006E6700002074000061720000F0
:1048BC0067650000747300002077000068690000D1
:1048CC006C650000206D00006F760000696E0000C2
:1048DC00670000005468000065200000636F000052
:1048EC006D6D0000616E00006420000066610000C8
:1048FC00696C0000656400002062000065630000C4
:10490C00617500007365000020740000686500008C
:10491C002050000065720000736500007573000084
:10492C0020690000732000006E6F000074200000EE
:10493C00686F00006D6500006400000054680000A2
:10494C0065200000636F00006D6D0000616E00005B
:10495C006420000066610000696C00006564000062
:10496C002062000065630000617500007365000043
:10497C002074000068650000205000006572000083
:10498C00736500007573000020690000732000003F
:10499C0064690000736300006F6E00006E650000B8
:1049AC006374000065640000004500007272000032
:1049BC006F72000020740000657800007420000005
:1049CC006E6F0000742000006465000066690000D2
:1049DC006E65000064000000546800006174000003
:1049EC00206400006576000069630000652000000B
:1049FC007479000070650000206400006F65000091
:104A0C00732000006E6F00007420000065780000B9
:104A1C0069730000742E00000054000068650000EB
:104A2C00206300006F6D00006D6100006E6400007B
:104A3C002069000073200000696E000076610000A0
:104A4C006C69000064200000626500006361000076
:104A5C00757300006520000074680000652000007C
:104A6C006465000076690000636500002069000041
:104A7C0073200000686F00006D6900006E67000015
:104A8C000054000068650000206300006F6D00009A
:104A9C006D6100006E640000207200006563000010
:104AAC0065690000766500006420000077610000F5
:104ABC0073200000666F000072200000616E000021
:104ACC00206900006E760000616C000069640000D3
:104ADC002074000061720000676500007420000003
:104AEC0064650000766900006365000000540000F6
:104AFC0068650000207200006563000065690000B5
:104B0C00766500006420000069640000656E00009A
:104B1C00746900006669000065720000207700006F
:104B2C0061730000206E00006F74000020720000A2
:104B3C00656300006F6700006E6900007A65000015
:104B4C0064000000546800006520000072650000DD
:104B5C006365000069760000656400002063000056
:104B6C006F6D00006D6100006E640000206300003A
:104B7C006F6E000074610000696E000065640000D7
:104B8C00206900006E760000616C00006964000012
:104B9C002070000061720000616D000065740000FF
:104BAC00657200007300000054680000652000006E
:104BBC0072650000636500006976000065640000A2
:104BCC00206300006F6D00006D6100006E640000DA
:104BDC002077000061730000207400006F6F0000EC
:104BEC00206C00006F6E000067000000546800002D
:104BFC0065200000726500006365000069760000A6
:104C0C0065640000206300006F6D00006D610000A2
:104C1C006E6400002069000073200000666F0000C5
:104C2C00726D000061740000746500006420000067
:104C3C00696E0000636F0000727200006563000013
:104C4C00746C000079000000707200006F7400003A
:104C5C006563000074000000736E00006D7000004E
:104C6C0000610000646D0000696E0000006D0000C2
:104C7C0069630000726F00006368000069700000D7
:104C8C0000730000656E0000644300006D6400005A
:104C9C0000730000656C000065630000746F000019
:104CAC00722E0000687400006D000000707200002D
:104CBC006F74000065630000742F0000636F0000C8
:104CCC006E660000696700002E680000746D0000BD
:104CDC00006900007000000067770000007300009E
:104CEC0075620000006400006E730000310000006B
:104CFC00646E000073320000006D00006163000000
:104D0C00006800006F73000074000000646800000D
:104D1C0063700000002F0000707200006F740000C0
:104D2C0065630000742F000072650000626F000064
:104D3C006F7400002E680000746D00003F000000CE
:104D4C002F700000726F0000746500006374000027
:104D5C002F6300006F6E000066690000672E000074
:104D6C00687400006D0000004E6F0000762000009B
:104D7C0032310000203200003031000037200000BA
:104D8C00313100003A310000323A00003535000074
:104D9C0000760000352E000034320000006E00005A
:104DAC00616D0000650000006E6F00007420000053
:104DBC0073650000740000003C6200003E5500006A
:104DCC00706C00006F610000642000006120000026
:104DDC00466900006C6500003C2F0000623E00003C
:104DEC000063000068650000636B000065640000F0
:104DFC0000660000616900006C000000546800004F
:104E0C0065200000447900006E6100006D690000AF
:104E1C0063200000444E000053200000436C00004F
:104E2C00696500006E7400002069000073200000AA
:104E3C006E6F000074200000656E0000616200005F
:104E4C006C650000642E0000006E00006F6E0000A8
:104E5C0065000000626C00006F6300006B000000D6
:104E6C000000000000000000000000000000000036
:104E7C000000000000000000000000000000000026
:104E8C000000000000000000000000000000000016
:104E9C000000000000000000000000000000000006
:104EAC0000000000000000000000000000000000F6
:104EBC0000000000000000000000000000000000E6
:104ECC0000000000000000000000000000000000D6
:104EDC0000000000000000000000000000000000C6
:104EEC0000000000000000000000000000000000B6
:104EFC0000000000000000000000000000000000A6
:104F0C000000000000000000000000000000000095
:104F1C000000000000000000000000000000000085
:104F2C000000000000000000000000000000000075
:104F3C000000000000000000000000000000000065
:104F4C00000000004574000068200000536F000052
:104F5C00636B00006574000020440000697300005E
:104F6C00636F00006E6E000065630000742000002B
:104F7C00436F0000756E0000743A0000203D000085
:104F8C00202500007500000045740000682000001A
:104F9C00536F0000636B0000657400002043000039
:104FAC006F6E00006E65000063740000204300000B
:104FBC006F7500006E7400003A2000003D20000068
:104FCC0025750000004500007468000020420000B8
:104FDC00797400006573000020520000783A0000DC
:104FEC00203D0000202500006C7500000000000032
:104FFC0047450000544400004E4E0000004700009E
:10500C004554000053540000410000004745000087
:10501C005443000046470000004400004F48000085
:10502C00414C000054000000534500005444000063
:10503C004E4E0000004400004F4800004F4D000051
:10504C00450000005245000053450000545200003A
:10505C000053000045540000444500005600000079
:10506C0052450000424F00004F5400000053000016
:10507C00455400004D48000053000000534500000B
:10508C00544D00004C5300000053000045540000E8
:10509C004D4800004300000053450000544D0000F3
:1050AC004C43000000470000455400004D4F0000E9
:1050BC0053000000474F0000504F000052540000B6
:1050CC000052000054300000303000003500000069
:1050DC0053450000544C000045440000004E0000B5
:1050EC00696300006B6E0000616D000065200000BC
:1050FC003D20000000250000687500000025000020
:10510C007500000053450000540000003000000002
:10511C0073720000632F0000436C0000696500008F
:10512C006E740000436F00006E6E0000656300003B
:10513C00746900006F6E0000732F0000436C000058
:10514C00696500006E7400002E63000000250000ED
:10515C00733A000025690000202500007320000030
:10516C002D2D00002061000073730000657200009B
:10517C00746900006F6E0000206600006169000019
:10518C006C650000640A0000007000005F630000A2
:10519C006C690000656E0000742D00003E77000005
:1051AC0072690000746500000021000000450000D9
:1051BC00525200004F5200002049000044200000D1
:1051CC003D20000025640000004500005252000004
:1051DC004F5200002054000045580000542000009D
:1051EC003D20000025730000004500004E440000E7
:1051FC000021000000000000000000000000000082
:10520C000000000000000000000000000000000092
:10521C00503D00002575000000000000000000005B
:10522C000000000000000000000000000021000051
:10523C000033000000450000523D00003300000028
:10524C00455200003D340000004C00003D2500009C
:10525C0075000000455200003D250000750000005F
:10526C004D3D000025750000005300004E3D000030
:10527C0025750000005600003D250000752E00002D
:10528C002575000025750000004800000000000096
:10529C00474500005443000046470000004700000B
:1052AC0045540000444200004700000052450000F5
:1052BC00424F00004F5400000052000045530000C4
:1052CC0045540000480000004745000054450000CC
:1052DC0044490000005300004554000044530000B2
:1052EC004E000000257500000053000045540000DE
:1052FC000000000008000000C80000002C010000A5
:10530C0008000000C80000002C010000080000008C
:10531C00C80000002C0100000A0000000001000081
:10532C00800000000A000000000100008000000066
:10533C000A00000000010000800000000D0A0000BF
:10534C0044480000435000002F5000006F770000CD
:10535C006572000020650000766500006E74000028
:10536C00206F00006363000075720000726500001E
:10537C006400000050650000727300006575000049
:10538C00730000004D500000465300000201000065
:04539C00000000000D
:020000040000FA
:1053A0000000FA0080407800BED0BF00814F50005E
:1053B00017003200E24F400008003200E2C1B300A3
:1053C0000440BC00E088200000014100C0802000B3
:1053D0000E00090030197800E201B10001007800E8
:1053E000BEF0B700E2CF4000090032000140780073
:1053F000E2C1B3000440BC00E0882000000141008D
:10540000C08020000E00090032187800E201B100CF
:105410000080FA00000006000000FA0011002000E1
:10542000E54F500009003E00DDFF070021418000EC
:10543000000021000080600002003A008000780037
:10544000020037002588A900110020000100780023
:105450000080FA00000006000000FA008000EB0067
:10546000E54F500006003E00CDFF07008000EB0036
:1054700010418000E70F500001003A0011002000A9
:10548000010078000080FA00000006000000FA0029
:10549000E54F500012003E00C1FF070022C8BF00C8
:1054A000E74F500002003200EB4F50000C003A0072
:1054B00091408000A040800001015000808F50008A
:1054C00005003900604080000E08B5000200400071
:1054D0000000E900030037000200E9000100370086
:1054E0000000EB000080FA00000006000000FA0057
:1054F000889FBE00804478000000EB00E5CF540098
:1055000009003E0009407800A5FF070068408000C0
:1055100070408000080450000804E9000940780049
:10552000DAFF0700000054004F04BE000080FA00BC
:10553000000006000000FA008000EB00E54F50007C
:105540000D003E0096FF0700B2408000C140800081
:10555000810F510002003900810051000600370020
:1055600080408000810050007040800000005100A9
:10557000808040008100E800010078000080FA008F
:10558000000006000000FA00889FBE0080447800FA
:105590000000EB00E5CF540008003E000940780011
:1055A0007FFF0700784080008040800008045000A2
:1055B00009407800DFFF0700000054004F04BE00E0
:1055C0000080FA00000006000000FA00881F780042
:1055D00000047800100078000C8D0200000000002C
:1055E000000C7800180090000C8D020000000000F4
:1055F0001004980028009000B8009000228D02004E
:105600000000000020049800310498004800900039
:10561000D8009000228D0200000000004004980095
:1056200051049800780090000C8D020000000000EA
:1056300070049800080890000C8D02000000000023
:10564000000C9800180890000C8D0200000000006B
:10565000100C98004F0478000080FA00000006004B
:105660000200FA00889FBE00C000200052B902006C
:10567000000000003252020000000000000FB200E3
:105680004280DE00F44450003200320071002000FD
:105690000000EB005C520200000000002A0037000E
:1056A00032520200000000000004E0002900320035
:1056B000E14F500024003200E24F500016003A0043
:1056C000E2CF540023003600000FEB0032520200FC
:1056D00000000000E44F500006003A003252020081
:1056E0000000000010479800325202000000000045
:1056F000004F78009E00780070212000808F5000BD
:1057000014003600D039B000808F500012003E00E7
:105710000100780010003700E1CF54000D00360082
:1057200032520200000000000044780080CF540094
:10573000080039008080FB000000EB005C52020092
:105740000000000088C454008944E900E1CF44000F
:10575000D3FF3A00802120004F04BE000080FA00F1
:10576000000006000000FA00889FBE008A1F780033
:105770000005780002047800840478000304E00047
:1057800015003200E1CF51002A003A000104E00088
:1057900008003200E1CF500026003A0004017800F2
:1057A000880078000A007800FA0802000000000073
:1057B00020003700E10F4500030032000A007800A6
:1057C0004E590200000000000800BE001C530200F9
:1057D00000000000170037000104E0000C00320058
:1057E000E1CF500013003A00E10F41000300320006
:1057F00002007800145902000000000089007800BF
:105800000A0078005C520200000000000900370026
:1058100004017800880078000A007800C056020071
:1058200000000000AC560200000000000000E00094
:10583000FCFF32004F0578004F04BE000080FA00E4
:10584000000006000000FA00BFD0BF00E10B2100FD
:10585000914078000104E10018003200E24F40005E
:105860000B003200E2C1B3000440BC007C034100E5
:10587000E588200062807A008002B1008402200066
:1058800013C0B30062862000E6C07A00B5FF0700AF
:10589000BED0BF00BFF0B70082FD2F006140800086
:1058A000010141008402200083822000934178009E
:1058B00011C0B30060862000AAFF07000080FA0034
:1058C000000006000000FA00DEFF0700B043800081
:1058D000304188006040800090408800A0408800EF
:1058E00070408000B0408800C04088004000200028
:1058F0002468AB0001003A00D0002000104188006D
:105900002408A9002428A9002448A9002488A90063
:1059100024A8A90024C8A90024E8A9002508A900F2
:105920002528A9002548A9002568A9002588A800E0
:105930008808A9008828A9008868A9008888A90083
:1059400060408000904388007C89020000000000D5
:10595000504388007C8902000000000060438800FA
:1059600086A8EF0010002000C04388000080FA00E5
:10597000000006000000FA008000EB00E54F500038
:1059800009003E0086FE0700AEFF070000802000F1
:10599000C18720000900090031587800A043800029
:1059A0005040880001802000010078000080FA004B
:1059B000000006000000FA00889FBE008A9FBE001B
:1059C000C010E20007003A00E28902000000000077
:1059D000F27F200002006000024020000200400030
:1059E00000868800C20320008000EB00A082200017
:1059F000EC0702000000000049F920000005EB0060
:105A000018982A000A40780065FE07000800E800A0
:105A10009000780063004400100178001804E00052
:105A200008003A000280400000804400AB022000E1
:105A30008085450000ED2100808F55000200360072
:105A4000FDFF3700FFFF37002868EF0080022000CD
:105A50000900400060408800010040000000E800AC
:105A6000704088000200400080408800D000200084
:105A7000104188002468A90072FF070078F8970099
:105A80008DE8B7008FFF07000A05E80066044400B0
:105A9000E60F5500020032008B047800D9FF370072
:105AA0004F05BE004F04BE000080FA000000060053
:105AB0002600FA00889FBE008A9FBE008C1F7800D7
:105AC00000447800014578005EFF07000808A30045
:105AD000020032002568A8000804A10024A8A9003B
:105AE00024C8A90024E8A9002528A9002548A90060
:105AF0002508A900BC5B0200000000000000E000D7
:105B0000FCFF3200E60064008004EB0056003A001F
:105B10009040800092438000820F500002003A00C3
:105B20008104780045003700C3438000820F500095
:105B30001300360002005000830F500001003600B1
:105B40000300780059448000890F500002003E0095
:105B500080047800010037002548A8000902780079
:105B600083822000934178008040EB00909D2000CC
:105B7000FCFE0700090078007228B4002F003700EF
:105B80007140800002825000040F980080004200A3
:105B90006040800000805000830F500001003600FC
:105BA0000300780059448000890F500002003E0035
:105BB00080047800010037002548A800890F5200B2
:105BC00001003600090F98000E0A90008382200021
:105BD000934178008040EB00909D2000E1FE07009B
:105BE0000E08900000825400040F98000900320053
:105BF00062408000904380000E08B500919D200017
:105C00000100400083822000934178008040EB0037
:105C1000D4FE0700904380008080440091438800B8
:105C200072408000828F5000040039006040800084
:105C30000000510000805000904388002568AB00B0
:105C400007003200C0438000808F540004003200FF
:105C500050448000808F5400010032000804A000EE
:105C60000900E00002003A00630064001600320000
:105C7000090078007828B5000900E0000100320032
:105C80000834A0000A08A300050032008C68EF0069
:105C9000D1122300314388001100200041438800C5
:105CA00034BE020000000000324380004343800005
:105CB0000001410081814900D2408800E340880012
:105CC0002488A8002B003700224180008A80FB0036
:105CD0000118A3000E0032008240E800E780600057
:105CE00080FF2F000000610001007000204188004B
:105CF000504380006143800061005000E080580004
:105D000050438800614388001900200019003700C3
:105D10007000610002003A0080047800150037002E
:105D20000108A3000A003A008CC8BF000800320036
:105D30000040E9008CE8B700304380004143800018
:105D40008100D1000080D3003043880041438800A7
:105D500034BE020000000000324380004343800054
:105D60000001410081814900D2408800E340880061
:105D70008004EB00B1438000110F9800A043800025
:105D8000200F98005243800063438000320F980038
:105D9000430F98007043800081438000500F9800AB
:105DA000610F98007E089000F1FF23000100600061
:105DB00001FF2F0001006000700F9800785F9800CD
:105DC0000000EB002017980009014100E081490024
:105DD00052438800634388008880FB000100D100A3
:105DE00061006000804578000004E000130032008C
:105DF0000148A30003003A006000B800500F98006B
:105E0000610F98008828AB00070032003E08900020
:105E1000CE08900061005000E0805800300F9800DC
:105E2000410F98000500370061014100E081490001
:105E300052438800634388008828A8000808A3000C
:105E4000010032008808A800B2408000C1408000F4
:105E5000810F510005003900704080001008B50026
:105E60008100510001005000020037000280500004
:105E70000000E900001798003A5B020000000000F3
:105E800080007800000F7800F0032000808F500021
:105E900002003E00000FEB000200370000FC2F0064
:105EA000008F40009E007800720647000E109000A0
:105EB000810F500001003600011798000C00780097
:105EC000C1FD070074854400F2F02F007E089000A9
:105ED000820060000105B300710F98000B04E00020
:105EE0000A0032007885440020C0B30020479800A3
:105EF00040C0B30030479800208021002007980060
:105F0000028060000006B300700F980001BC200002
:105F1000914078008180FB00C1CBBF004800DD00CC
:105F20000101700021BC2000914078008180FB00BD
:105F3000C3CBBF004800DD0081017000660447004C
:105F4000028CBE00E0438000F143800050079800BF
:105F5000610798000040EB00604F980069C0B300F3
:105F6000794F98000A0F98000A0078000C8D020003
:105F700000000000000F9800C10020000800780019
:105F8000468D0200000000000080EA001017980013
:105F9000109B20004E590200000000000A0178000A
:105FA00089407800C087200088B902000000000006
:105FB000410120000C0078001C530200000000008A
:105FC0000B04E00004003200410020000E80E800D5
:105FD0001C53020000000000509C200014590200D5
:105FE000000000000A0078003258020000000000A3
:105FF000000F7800509D20004E5902000000000064
:10600000210020000E0078001C5302000000000058
:1060100088590200000000004F0678004F05BE00BE
:106020004F04BE000080FA00000006000000FA00E5
:10603000889FBE008A9FBE00010478000205780098
:1060400083447800E54F500054003E00D4FC070024
:106050000800E00001003A001800200060408000C5
:106060001008B5008005E9000A0444008B0F5400B5
:106070004A003E00F3FD07006380640001003A001F
:106080003940B300088055008981FB000318A30044
:1060900002003A000A017800040037000308A30058
:1060A000010032000000D100000145006040800086
:1060B000000041000004E800B1408000324480004C
:1060C000E10F410009003200D04380000000410090
:1060D0008080400080408000808F500003003600A8
:1060E0000E08B500008040008000E900C04080003C
:1060F000810F50000200390005003600704080001A
:10610000800F5400040036000328A30023003A0047
:10611000C8408800B8408800C0408000808F500090
:10612000110031000328A3000F00320072408000EC
:1061300002825000838220009341780083407800DF
:106140000800780087FD0700B1408000C040800053
:10615000808F500004003100080078000E08B50060
:1061600000805000B0408800784088006040800087
:1061700090438800A04088009040880011002000D3
:1061800010418000E70F500005003A0000C1B30045
:1061900047FE070011002000010037008000EB00DF
:1061A000010078004F05BE004F04BE000080FA00D9
:1061B000000006000000FA00881F78000044780004
:1061C000DCFC07000000E000070032000840780017
:1061D00073FC0700B0408000C040880011C0B300CD
:1061E00000C1B30032FE07004F0478000080FA00BF
:1061F000000006000000FA00E54F500009003E00D4
:1062000067FC07008FFD07009140800090438000ED
:10621000808F50000300320011C0B30000C1B300F2
:1062200023FE07000080FA00000006000000FA00CC
:10623000E54F500036003E0059FC0700B04080009A
:10624000C040880010418000E50F50002F00320050
:1062500006003E00E10F50000D0032002B00390017
:10626000E30F500026003E0028003700EB0F5000DF
:106270001500320003003E00E70F500020003E00F2
:1062800006003700EE0F50001D003A0019003700DD
:10629000387F0200000000001C00370011C0B3006E
:1062A00010C1B30002FE07007808E20004003200CB
:1062B0009140800090438000808F5000F7FF3A00AB
:1062C000800020000C00370011C0B30010C1B300E3
:1062D000F7FD07007808E2000400320091408000DA
:1062E00090438000808F5000F7FF3A00C0002000EC
:1062F00001003700D0002000104188000400370062
:106300008040EB0040C1B300E9FD07006DFD0700D0
:106310000080FA00000006000000FA00881F7800E4
:1063200000447800E54F500004003E001CFC0700CC
:106330002468A90008407800BCFF07004F047800DB
:106340000080FA00000006000400FA00889FBE00EA
:106350008A9FBE008C1F7800008FBE000244780028
:1063600003057800844578008004EB000946780036
:10637000094078000AFC070010418000ED0F500032
:1063800060003A002FFD07000B4078008D48E300C5
:106390005C003A0080212000504488000804E0009E
:1063A00006003A00BA4388002468A8004000200094
:1063B000104188003A4188005000370000C02F008B
:1063C000C010B40081F82000810F50000200360098
:1063D000004020000086880000868000B0438800CE
:1063E0000000E80000868800AA43880034BE02004E
:1063F00000000000D0408800E14088002488A80008
:10640000E34F54001500320003003E00E14F5400FA
:106410003A00390003003700E44F540037003A00D7
:106420001E0037001E00BE00E0438800F1438800D4
:106430000814A2000880FB000000E9004F00DE0005
:106440004200DD00414480000120A10080807000F6
:10645000414488002228EF00280037001E009000E9
:106460001E0040000A004000B143800001006800A7
:10647000304188001E00BE00E0438800F1438800E0
:106480008C68EF0081092000314388006828EF0004
:106490002000200010418800180037001E017800FD
:1064A000224090000080FB00B2409000C808DD0050
:1064B000808070009281FB00124090004800DD0057
:1064C00003007000808040008A804000B04380005C
:1064D0008080680031418800C087200009000900E1
:1064E00032587800A200B10050002000104188000E
:1064F00011C0B30020C0B3006DFD07000C80FB008D
:10650000040037008904E800E68F540097FF3A0042
:10651000E00F20004F0678004F05BE004F04BE007C
:106520000080FA00000006002E00FA00889FBE00DE
:106530008A9FBE008C9FBE00800578008204780090
:106540001082FB00104090004800DD000401700044
:106550002B4290000482FB003B4090004800DD008D
:1065600084017000028FBE001101BE002207980056
:10657000330798000040EB00004F980060C0B30064
:10658000104F980059079800090078000C8D020000
:106590000000000050079800C10020000E007800A5
:1065A000468D020000000000000478000900780019
:1065B00032580200000000008880EA00808F5000FE
:1065C0003B033A000000EB0052B90200000000005B
:1065D0006C04470041012000080078005C52020072
:1065E0000000000008007800F7FB07004E0890004C
:1065F0004400DE006F4060004200DD007440500047
:106600000080FB0000865400F40156001317980028
:10661000FE0190000300E000250332002B409000B3
:106620000080FB00BB409000C808DD008080700047
:106630001B81FB001B4090004800DD000200700041
:10664000808040009880400003856800E9CFB30057
:106650000004EB000840780051FB07001041800067
:10666000ED0F50002100320031418000E40F500056
:1066700005003A007E009000808F50001B003A0019
:1066800088447800190037008A8F500017003A00BC
:106690006CFC0700FE009000B0438000808F50002B
:1066A00012003A00EC004700A0438000910F100058
:1066B0000E003A009B80FB001B4090004800DD006C
:1066C00001017000AB4090008180FB003B409000D6
:1066D0004800DD0081017000E0438000F14380004C
:1066E000800F5100818F5900E40232000804E80055
:1066F000E60F5400D7FF3A006C044700E2CF440095
:106700000F0032000940780025FB07004DFC070010
:106710003A418800C4872000090009003B5A7800EC
:10672000AB00B10018047800A8438800FE02900076
:10673000B54388006640800096438800CF0237004A
:106740004E0890000098A300D90232006208E200CF
:10675000D7023A007E039000980278008004EB0094
:10676000A4832000140078000000E000170032002D
:10677000860F500011003A0054B89700850F500062
:106780000E003A009B80FB001B4090004800DD009B
:1067900001017000AB4090008180FB003B40900005
:1067A0004800DD008101700004B8970094B897009C
:1067B000820F5000838F58008F0232008904E80056
:1067C00074024200E38F5400E6FF3A000004EB003D
:1067D00008407800F2FA07002468AB000500320098
:1067E00018FC0700B14380007E009000808F5000AD
:1067F000880232000804E800E60F5400AC023200C0
:10680000F3FF370034BE02000000000042782D0084
:10681000730120000001410081814900D2408800BD
:10682000E340880014418000E40F5200030032006E
:10683000E50F520047003A00160037000880FB00C1
:10684000E400600006003A000048A30006003200A1
:106850005A4388006B4388000440780094FC07008A
:1068600018FC0700920237000018A300FCFF32005A
:106870002E149000BE14900061044400E0844C008B
:10688000784388008943880075FB070050448800DE
:106890002A0037008880FB000128A30084023A0008
:1068A0004408DE0061006000004678000004E0005B
:1068B000050032005843800069438000880F55006E
:1068C000898F5D008D003A000118A3007802320024
:1068D0002E109000BE10900061004000E080480043
:1068E0007043880081438800DE089000C14388001F
:1068F0005BFB0700504488000C04E0000F003200EE
:1069000011C0B30000C1B30069FC07007000200093
:106910001041880034BE02000000000042782D00C3
:10692000730120000001410081814900D2408800AC
:10693000E34088002488A9005D02370011C0B3003D
:1069400020C1B3005AFC07006000200010418800FD
:10695000570237000883FB0061016300521798005B
:10696000026F9800AE6A90000504E00003003A0050
:106970009E14900009179800020037007306560015
:106980000C1798000884FB00681798000818A300EB
:10699000030032000E1090000000E800001798007D
:1069A000B2408000C1408000810F510005003900D5
:1069B000704080001008B5008100510001065000B1
:1069C00002003700028050000006E900704380009A
:1069D000814380002E149000BE14900000015400EA
:1069E00081815C00820678008E1490000900E0002E
:1069F0001F0032000C00E00028003200E00F5100C0
:106A0000E08F5900040035006160B800820F50002B
:106A1000838F58000A003E008E129000050041004E
:106A2000E08049004240A9000700340005005600FC
:106A3000CF80DE00800F5100818F590002003C00A2
:106A400015002000010037008002EB006160B800F3
:106A5000800F5100818F59000E003D000E149000F0
:106A6000088046004240A90010003C0009003700A1
:106A7000E00F5100E08F59000C0032000700350094
:106A80006160B800820F5000838F580007003E00FD
:106A9000020037000500E00004003A00EE14900008
:106AA0000928A30002023A00F001370066006300E3
:106AB0006BFF3A006E1090000048A300FC0132000A
:106AC000EB0F520005003E00E70F520015003100A9
:106AD000E60F5200D2003A0003003700EC0F5200DC
:106AE000CF003A00C6003700584380006943800059
:106AF000880F5500898F5D00080032005A438800D6
:106B00006B43880011C0B30040C0B300E8FB07002E
:106B10005843880069438800E50137007000200071
:106B20001041880097438000924080008700510008
:106B300003003B00604080000E08B50080804000EC
:106B4000524380006343800001004100E08049001F
:106B50000000550081805D004240A900090034001A
:106B60008808AB0003003200E10F5000E08F5800AE
:106B7000020032008040EB00BD0137006105550086
:106B8000E0855D00A640800006805300CF80DE00D7
:106B90000002510081825900868F530002003900A3
:106BA0000400BE0004003700604080000E08B500FD
:106BB00000005200E0805A000001550081815D0014
:106BC0004240A9002F0034006140800079408000DD
:106BD000018454006140B800800F5100818F59003A
:106BE00028003E008868A9008888A9002508A90017
:106BF000A040800002024000A44088009143800031
:106C0000808F500004003900848F50000D00310047
:106C1000010052000400370008804000840F50003B
:106C2000080031000000520052438000634380009E
:106C300000004100E0804900504388006143880023
:106C40009443880071408000810F52000400390095
:106C5000604080000080500000005200A04088008A
:106C60009243800071408000810F51001C00390068
:106C70006040800000805000000051009043880078
:106C800017003700870F5300150032004044800082
:106C90000038A300110032000048A3000E003200AB
:106CA000544388006543880090438000860F50005D
:106CB00007003100604080000E08B500CF80DE0084
:106CC0000000520081805A005043880061438800D0
:106CD000964388002548A8008888A8008868A800EE
:106CE000A140800090408000808F500015003A0045
:106CF0002568AB000A003A0034BE02000000000024
:106D000042782D007301200000014100818149007B
:106D1000D2408800E34088002488A9000900370099
:106D200050438000614380008A0F50008B8F5800D1
:106D300004003A008808AB00020032002488A90051
:106D40002568A900504380008A0050005E0890002A
:106D5000010050007808E20003003A000000E00063
:106D6000010032002528A800C0438800104180009F
:106D7000E80F500013003A00504380006143800048
:106D80008A0F50008B8F580025003A008808AB000E
:106D90002300320034BE02000000000022BC2E009E
:106DA000B30020000001410081814900D2408800E9
:106DB000E34088002488A80090002000104188004B
:106DC00017003700E90F500008003A00DE1090006D
:106DD0000100E00012003A005A4388006B4388002B
:106DE000AE68900040C1B3009CFE3700EA0F50002F
:106DF0000B003A00504380006143800004003700DC
:106E0000524380006343800061004100E0804900FC
:106E10008A0F50008B8F580025013A0090FE3700F2
:106E2000EE1490000902B20021013A0010418000E6
:106E3000EB0F50001E013200EA0F50001C0132001F
:106E4000EC0F50001A0132009E1190000300E00088
:106E50009E0032000D8441000D00E0004C003C001B
:106E60004E0890004200DE00C003B2000D0050004A
:106E700052B90200000000008C0F540001003E00D7
:106E80000806780070438000814380000C004000B9
:106E9000E08048007043880081438800B54080004E
:106EA000824080000C804200818220009140780066
:106EB000820F500013003600050451000804E8005A
:106EC00008027800894178000081EB000500780015
:106ED00024FA0700080456008182200091407800BF
:106EE0007040800008027800894178000081EB0042
:106EF0001CFA07007040800000044400B84088007D
:106F0000070037000C027800894178000081EB000F
:106F10000500780013FA07000C0078001628B4006A
:106F200030448000E10F4000680032008C005000C7
:106F300031448800D04380000081400012003300BB
:106F40000100E00061003C0070438000814380004C
:106F500002004000E08048007043880081438800C0
:106F6000B040800080004100B14088008040800037
:106F7000808F5000040036000E08B50000804000ED
:106F80000000E900B040880086A8EF004F003700FD
:106F90008C0F5400020036000D0656001C17980096
:106FA0004E0890004200DE00C003B20052B9020059
:106FB00000000000B34080008D82410082408000CC
:106FC0009E10900001804200820F50001900360090
:106FD0008182200091407800030051000D00500094
:106FE0000004E8000B0033000802780089417800B3
:106FF0000081EB0005007800DAF9070081822000AB
:1070000091407800704080001E11900008025100ED
:1070100005003700020078000E08B500008042002D
:107020000000E9001E129000894178000081EB0009
:107030000600370081822000914078001E129000E7
:10704000894178000081EB0005007800C5F9070050
:1070500030448000E10F400004003A003D448800C5
:107060009E119000D3438800180037001E12900034
:107070000D044200D1438000808F56000C00310087
:1070800081004000810F540002003E00800F540038
:10709000030031009E129000D543880002003700A3
:1070A0000D805000D04388003D4488000700370021
:1070B00081004000810F540004003600818F56008B
:1070C00002003E0000005400D04388000E139000E0
:1070D0000600E0001400320010418000E70F50006D
:1070E00002003200B8408000C840880024E8AB00AD
:1070F0000500320011C0B30000C1B3006CFA0700F4
:10710000D0F907000800370024E8A80024C8AB0025
:1071100005003A0024C8A8004EBE0200000000008E
:10712000D003B000004188008E6C90000904E0009C
:107130005F003200704380008143800061014000A5
:10714000E08148000E1390002E129000BE129000B5
:1071500006004200E0804A00800F5100818F5900F4
:1071600053003A0072438800834388001041800036
:10717000E70F50000E00320003003E00E60F500003
:107180003A003A0005003700E80F50000F003200C7
:10719000E90F500035003A0014003700C00020000D
:1071A0001041880011C0B30010C1B3003100370096
:1071B000B0002000104188004EBE02000000000018
:1071C000A007B0000041880028003700504380002D
:1071D000614380008A0F50008B8F580003003200FB
:1071E000A000200010418800200037008040EB0004
:1071F00000C1B30099FD37004EBE02000000000040
:107200007449B90072014100A482200000317A0063
:1072100027003700744CB900AA8220000A004400FD
:10722000090009003B587800A000B100AB00B10094
:107230006A004400EE04900009307D000A0044001A
:107240000E0990009E09900062009800730098005B
:107250007000440001307D004EBE020000000000BE
:107260007204440000347D001100370011C0B300E7
:1072700000C1B3000EFA07000D0037001E5C90003D
:107280002E0D9000BE0D90000E0A90009E0A9000F8
:1072900024179800351798002408A9002428A9006D
:1072A0002448A9002488AB005EFD3A0055FD370054
:1072B000DC54020000000000100020004F06BE0059
:1072C0004F05BE004F04BE000080FA00000006001B
:1072D0000400FA00889FBE008A9FBE008C1F7800C1
:1072E0000006EB008C4578000C4078002CF8070075
:1072F0002041800001602000010060003100320068
:10730000BC5B0200000000000000E0002D00320025
:10731000204180004A00DE006105600009C1B30021
:107320002A00370047F907007440B900800178004F
:10733000A282200002004000C1872000090009004D
:10734000B0587800A000B100EA804100E100790067
:10735000A1438800EC80410082804000160020009C
:107360000700200031024300A1824B0074438800D3
:1073700085438800E1438000F74380008780400018
:10738000A243800082804000B24380008280680077
:107390003141880061002000114188006202140020
:1073A0007422B900E18320000181410013C0B300C1
:1073B00083407800EBF807006228EF0029C1B30092
:1073C000310037008044EB000005EB0024A8AB003F
:1073D00007003200F84080004EBE020000000000AE
:1073E000000454004240A90001003C0009C1B30060
:1073F00024C8AB0007003200084180004EBE0200E6
:1074000000000000000454004240A90001003C00BC
:1074100009C1B30010418000EB0F500009003A0091
:10742000084180004EBE020000000000000454002D
:107430004240A90003003C00C00020001041880029
:1074400019C1B30010418000E40F50000C003A0055
:10745000324180000004EB00A1832000110078007D
:107460000000E00006003200820F5000ADFF320045
:107470000804E800F4804000E30F5400F7FF3A00EE
:107480000904E0000400320011C0B3008AC05000BB
:107490000940780086F907002488AB0026003A00EE
:1074A00010418000E70F5000EB003A0034BE0200AC
:1074B00000000000D2408000E34080000200500045
:1074C00083805800E4003300214180006780600021
:1074D000E60F50000B003A00430CDE0061446400EC
:1074E0000B40780051FB07000B4078004FFB070072
:1074F0000804E000D8003A00E000200010418800B5
:10750000D5003700CFF8070021C0B30000C1B30099
:1075100067F9070034BE02000000000042782D0029
:10752000730120000001410081814900D2408800A0
:10753000E3408800C800370034BE020000000000AD
:10754000D2408000E3408000020050008380580059
:10755000C1003300BBF8070010418000010020008B
:10756000EC0F5000E08F580093003E0000600100D7
:107570000C00370015003700390037004000370095
:107580008D0037005E003700690037007200370059
:107590007A0037008C0037007D0037006E0037001E
:1075A00080003700287F0200000000000000E0009B
:1075B000810032001100200011418800E04380006A
:1075C000567F0200000000007B0037000E007800AC
:1075D00022800200000000000000E000760032007F
:1075E000387F020000000000000478000000E00086
:1075F000110032001E00BE00E0438800F143880005
:107600002000200010418800E04380007E08B40084
:10761000A143800001004000B143800001006800E8
:10762000304188008C68EF008109200031438800D8
:107630006828EF006000370034BE02000000000040
:1076400042782D0073012000000141008181490032
:10765000D2408800E3408800184188005600370077
:107660004EBE020000000000F0408800C0872000ED
:10767000D6A50200000000003000200019003700ED
:1076800001882000C0872000A2A4020000000000A2
:107690000000E00015003A004EBE020000000000AD
:1076A000F24080000200500032438000820F500000
:1076B000410036008CC8BF00E54F500008003E0076
:1076C0000040E8008CE8B700304380004143800070
:1076D000000040008180480030438800414388001A
:1076E00020002000104188003300370050002000A7
:1076F000104188000004EB0029C0B300500037009F
:1077000029C0B300C088200012C0B300904F110000
:1077100077003600090078008CE8B700444B2C0055
:107720003443880044002000444388007000370040
:10773000C088200015C0B30090CF1200670036004B
:1077400020418000680060001F003A0029C0B3009B
:10775000000478001E003700C088200026C0B30057
:10776000904F13005F003600800020001041880019
:1077700019C1B3000004EB0015003700C0882000D9
:1077800027C0B30090CF1300580036000E0037001A
:10779000C088200021C0B30090CF100051003600F7
:1077A00009003700C088200022C0B300904F1100AC
:1077B0004E003600040037000004EB000904E0002E
:1077C00003003A002400370049C1B300180020002C
:1077D0000A00E0001A0032008C68EC0030438000A0
:1077E0004143800000004000818048003043880011
:1077F0004143880090438000A34080000301500073
:10780000830F500003003100604080000E08B50077
:10781000000141005043800061438000020050009D
:10782000E0805800504388006143880002007800DF
:107830007828B400934388008040EB0001003700B3
:1078400011C0B3000940780099F807000800E00073
:10785000010032001BF807000C06E800E60F560096
:10786000A0FE3A008004EB007448B90000047800E0
:1078700070004000AA82200060007D000000E0004F
:107880001D0032004EBE02000000000072014400E4
:1078900062017D000200500072722000820F5000D1
:1078A0000A003600628214007422B900E2832000CC
:1078B000020144000A00440013C0B3008340780072
:1078C000A8F707006228EF008904E9008904E800AE
:1078D000E28F540008003E00E3FF370029C1B300E7
:1078E0000300370009C1B3000100370019C1B3001C
:1078F0000004EB00B8FF37004F0678004F05BE00CC
:107900004F04BE000080FA00000006003000FA00BC
:10791000889FBE008A9FBE008C9FBE0000447800F6
:1079200051179800820578000305780084047800D8
:1079300065179800E54F500097003E000200E000F8
:107940009500320096F6070008407800F9F6070027
:107950000A0650008B0F56009A0039000900E0001B
:1079600003003200890F5600010036000906780036
:10797000C04080000001450081408000810F51001F
:1079800004003600010078000E08B5000000410038
:107990000001E900028050000000E8003017980064
:1079A0005E1090000017980030447800001798008F
:1079B000EE1090000100E00006003200F0C9B300B4
:1079C00000404400F94F500002003E0000CEB300DA
:1079D000004444008B0478001A179800421798005E
:1079E0000E1590008006EB0002C2B30042679800BB
:1079F0003E109000FF0F500001003E0040679800CD
:107A00004E6190000280FB008C0F50000100360098
:107A10004C679800CE6090000183FB00060278005E
:107A200083822000934178004E11900011C0B30072
:107A30000E007800761798004AF707007E13900032
:107A40004E11900006014100421798003E10900030
:107A5000060050003017980004003A007140800082
:107A6000411798000081EB00321798008003EB006B
:107A700003CEB3006E1090000000E00023003A0037
:107A800000017800390037000081FB008E004100C2
:107A900011427800F5C9B30005404200F94F50008B
:107AA00001003E0083484200914F540009003A0013
:107AB0008904E9003A0032003A4478000540440065
:107AC0001D002000F94F50000F003E000344440009
:107AD0000D0037000D00E00002003A008B04780032
:107AE00009003700DE109000114478000540440082
:107AF000F94F500001003E00034444008B0478001D
:107B00000E1590008006EB008703E8000740780020
:107B10004E61900082CF5300DBFF39001700370021
:107B20008080FB000E804000904F540005003A001A
:107B30008904E9001E0032003A4478001D0020004C
:107B4000090037000D00E00002003A008B047800C5
:107B5000050037005E109000104478008B04780018
:107B60000E1590008006EB000201E800024078004C
:107B7000CE609000814F5100E9FF390006065600A3
:107B8000890F56000F0039001E11900006014100B8
:107B90001217980094FF37000000EB000A0037002E
:107BA0009E1090000B805000020040000300370040
:107BB0001E1190000B005100010040000000E80081
:107BC000010037000080EB004F06BE004F05BE00ED
:107BD0004F04BE000080FA00000006000200FA0018
:107BE000014F780084027800030278008201780057
:107BF000120020008E00780044FF07000080FA0089
:107C0000000006000000FA00889FBE008A9FBE00A8
:107C1000004478008105780082047800030578002C
:107C2000E54F50002B003E000200E000290032002A
:107C3000DBF50700084078003EF60700800078007A
:107C400009004500810F5000010036008A84500071
:107C5000C04080000001450081408000810F51003C
:107C600004003600010078000E08B5000000410055
:107C70000001E900028050000004E80028C8BF00AD
:107C8000888F540005003E0009027800804178008A
:107C900011C0B3000B0078000B0037000802780019
:107CA0008041780011C0B3000B007800ADF60700EA
:107CB00072408000088045000882540083822000C2
:107CC0009341780011C0B300A6F6070009017800BF
:107CD000010037000001EB00020078004F05BE00F4
:107CE0004F04BE000080FA00000006000200FA0007
:107CF00081017800120020008E007800C1FF07008B
:107D00001E80FB000080FA00000006000000FA0060
:107D1000889FBE008A9FBE000045780081047800DD
:107D20000204780003F60700800578000000E000F8
:107D3000320032000A40780099F507008B0F54009A
:107D4000010036000B047800C240800081408000B2
:107D5000080041000005EB00810F50000E003600C6
:107D6000028050000005E8000900E0000700320032
:107D70000A027800838220009341780011C0B3008A
:107D80000900780077F607008A8444000A0454004A
:107D900070408000C04088000900E0000700320009
:107DA000C24080000802780083822000934178005E
:107DB00011C0B300090078006AF6070008007800D7
:107DC0001828B4000A04440008805500880F5000A9
:107DD00002003E002548A8000700370024A8AB0099
:107DE00005003A0024A8A8004EBE020000000000D2
:107DF000A007B000F0408800080078004F05BE00E2
:107E00004F04BE000080FA00000006000000FA00E7
:107E1000889FBE008A1F78008044780001057800A2
:107E2000C4F50700000478000000E00016003200EE
:107E3000094078005AF507000A00E0000700320008
:107E4000C24080001400200083822000934178000B
:107E5000844078000A00780042F60700C1408000A4
:107E60008100E800C140880080408000808F500081
:107E70000200360070408000C0408800E10F5400CE
:107E800003003A002548A8000800780009003700E0
:107E90001000200024A8AB0006003A0024A8A80087
:107EA0004EBE020000000000A007B000F0408800B5
:107EB000100020004F0578004F04BE000080FA003B
:107EC000000006000000FA00889FBE008A9FBE00E6
:107ED0008C9FBE00004578008105780082067800FE
:107EE0000000EB00E54F550042003E000A407800DC
:107EF0002BF507000A40780064F50700800478003D
:107F00000000E00004003A000A407800B9F80700D9
:107F100009007800370037008D0F5000020036004E
:107F20000D04780001003700000478002508AB003C
:107F300008003A00604080000E08B5000000D10043
:107F4000808F540003003E000A407800A9F8070023
:107F50002508A800954080007140800008804200FC
:107F60000006EB00810F50000C0039000586500020
:107F700081822000914078000C02780013C0B30089
:107F80000B01780005007800F6F507008C854500A8
:107F90000C045400604080009040880081822000E2
:107FA00091407800904080000802780013C0B30030
:107FB0000B017800EBF50700080078001228B400E8
:107FC0008D8F540003003E000A40780089F80700B6
:107FD0000700370024A8AB0005003A0024A8A80039
:107FE0004EBE02000000000078004000F040880013
:107FF0000C0044004F06BE004F05BE004F04BE00FB
:108000000080FA00000006000000FA00889FBE0011
:10801000804478000104780001007800DE08020046
:108020000000000000017800880078000940780016
:10803000A4FF0700000044004F04BE000080FA00C7
:10804000000006000200FA00889FBE00804478000D
:10805000014F7800E54F500033003E00D0F4070098
:108060000940780009F50700000478000000E000EE
:108070002D003200E10F500002003A000940780064
:108080005CF807002508AB0008003A00604080005B
:108090000E08B5000000D100800F540003003E0020
:1080A0000940780053F807002508A80081822000C5
:1080B00091407800904080001400200084417800B6
:1080C0000E017800A7F50700914080008100E800CC
:1080D0009140880070408000808F5000020039007D
:1080E0006040800090408800E10F540004003A0096
:1080F000094078003FF80700080078000B003700BF
:108100001000200024A8AB0008003A0024A8A80012
:108110004EBE02000000000078004000F0408800E1
:1081200010002000010037000000EB004F04BE00EB
:108130000080FA00000006000000FA00B8CABF0084
:108140000080FB004200DD00E1C7B300C2AB2000AD
:108150006040790022400200000000000080FA0028
:10816000000006000000FA00889FBE00B86AEF0019
:10817000210037000084FB00A9AB20004244DD0051
:10818000090044000008EB0084C0B3000305200090
:108190000041EB006000B800A431020000000000C4
:1081A0000884E80000F47C00D6EAEF00D7EAEF008C
:1081B00082AB2000124178000281FB006909200097
:1081C0000991B90000ED2100020040004E59020063
:1081D00000000000000478008900780020AC200036
:1081E0001C53020000000000080078004E590200F5
:1081F00000000000B86AEC00B8CABF00E14F5000B0
:10820000DCFF3600B86AEF004F04BE000080FA00C1
:10821000000006000000FA00889FBE008A9FBE0092
:1082200000457800B8CABF00804F55001E003200DC
:108230000080FB00680920000880B9000BED2100D8
:10824000008045004E5902000000000080047800C4
:108250008800780020AC20001C53020000000000C1
:10826000090078004E590200000000000A80FB005F
:108270000880B90000804500145902000000000089
:10828000800478008800780020AC20005C52020056
:1082900000000000090078001459020000000000EE
:1082A0000A007800B8EAB7004F05BE004F04BE00D0
:1082B0000080FA00000006000200FA00889FBE005D
:1082C0008A1F780000047800DE0802000000000029
:1082D00080017800080178002300370082047800CC
:1082E000B94078000305E900D0C3B30080CF500047
:1082F000030032007740500080CF500002003A0067
:10830000005CEB0016003700B0C2B30080CF500015
:1083100002003A006B4050000E00370050C2B3001C
:1083200080CF50000D003A00E10F550010003600DC
:10833000994478001947980022409000004F780037
:10834000E3044100638551001E0078003A8C02006E
:1083500000000000005C780001003700015C78003C
:108360008A017800090178000300E000DBFF3A0091
:10837000005CEB0008007800004CEB004F05780033
:108380004F04BE000080FA00000006000000FA0062
:10839000889FBE000004BE001600370088007800E9
:1083A00009007800CC070200000000000000E00097
:1083B00006003A0009007800DE0802000000000014
:1083C000000044000000E8000D00370008007800BD
:1083D000DE08020000000000000044000004E80085
:1083E00008007800DE0802000000000000004400E1
:1083F0000004E8001804E000E8FF3A000000EB0089
:108400004F04BE000080FA00000006000200FA00DF
:10841000889FBE008A9FBE008C9FBE0083AB200059
:1084200093417800ABAB2000004F78000106780044
:10843000820678000004E0000B0032000380FB009D
:108440004200DD000080E8000002EB0084017800BB
:10845000040178009E40780060C07D00EE3D02007F
:1084600000000000060037000380FB004200DD0032
:108470000080E80060C07D009A2A02000000000031
:10848000000578002B002000E10F40006C00320056
:10849000E18F560012003E000C00E0001200320096
:1084A0001856800029568000B8CABF000080FB0023
:1084B0004200DD000A0178008000EB00C3AB200021
:1084C00060C07900863E02000000000000045400F5
:1084D000E0845C0018568800295688003600370072
:1084E0000C00E00010003A00185680002956800069
:1084F000B8CABF000080FB004200DD000A0178001E
:108500008000EB00C3AB200060C07900863E020013
:108510000000000000045400E0845C00185688004D
:1085200029568800340037000D81E900ABAB2000EC
:1085300083AB2000934178001856800029568000B4
:10854000820F50001E0036000380FB004200DD0059
:108550000080E8008C00780060C07D00863E02004C
:108560000000000000045400E0845C0018568800FD
:10857000295688000D0155000281E800B8CABF00E5
:108580000080FB004200DD000080E8008000EB007E
:1085900060C07D00863E0200000000000000540024
:1085A000E0805C0010568800215688008D0046004F
:1085B0000040EB00E0F89F001B0020000F00370098
:1085C0000380FB004200DD000080E8000A01780023
:1085D0008C00780060C07D00863E02000000000034
:1085E00000005400E0805C0010568800215688008E
:1085F0000040EB0000757E008005EB001E40780017
:108600000004E0000E003200185680002956800059
:10861000B8CABF000080FB004200DD008000EB0014
:10862000C2AB200060407900063F0200000000005D
:1086300000045400E0845C00185688002956880025
:108640000B0078004F06BE004F05BE004F04BE0071
:108650000080FA00000006000000FA00889FBE00BB
:10866000000478000101780080007800D0C3B300D6
:1086700066FF0700800478000800E0000400320074
:108680001804E00002003200080078000AFF07002A
:10869000090078004F04BE000080FA0000000600C8
:1086A0000000FA00889FBE008A9FBE008C1F7800E1
:1086B000000578000106780001017800800078004C
:1086C00060C2B30051FF070080057800E20F500040
:1086D00012003A001856800029568000B8CABF0020
:1086E0000080FB004200DD00C1AB200060C07800CC
:1086F0009A2A02000000000001002000800F5400B0
:10870000818F5C0005003A000C0178008A00780037
:108710000040EB003DFF0700800578000A00E00004
:10872000040032001A04E000020032000A0078005F
:10873000E1FE07000B0078004F0678004F05BE00F1
:108740004F04BE000080FA00000006004000FA005E
:10875000889FBE008A1F7800000178007056800054
:1087600081568000E00F5000E08F580010003A0062
:1087700002007800A67A0200000000008044780021
:10878000E14F40003D0032003C7E0200000000004E
:108790007056880011003700094078000479020003
:1087A00000000000CE2AEF00D02AEF00330037008F
:1087B00070568000487A0200000000008044780073
:1087C000E14F40002D00320082568000030020005F
:1087D000210020002E7C020000000000B8CABF006B
:1087E0000080FB004200DD00C1AB200060C07800CB
:1087F000462A02000000000000057800160037003D
:108800000A01780000042000800F550001003600A6
:10881000000178008E00780009407800A2790200FB
:1088200000000000000478000000E000DAFF3200E1
:10883000B8CABF000080FB004200DD0008017800DC
:108840008E007800C3AB200060C07900623F020058
:1088500000000000080555000A00E000E8FF3A00AB
:1088600009407800207E0200000000008056880049
:108870000940780004790200000000004F057800EC
:108880004F04BE000080FA00000006000000FA005D
:10889000E70F5000E08F58001400320007003E0040
:1088A000E00F5000E08F58000B003200E20F500044
:1088B000E08F580016003A0009003700E80F50001A
:1088C000E08F58000C003200E90F5000E08F580094
:1088D0000F003A000B00370000C6290001003700E6
:1088E000B0C6290099FF0700120037001E6B020076
:1088F000000000000F003700626B02000000000063
:108900000C0037008C6B02000000000009003700EB
:10891000B8CABF000080FB004200DD00420020001A
:1089200061C72900C3AB200060C07900623F02002C
:10893000000000000080FA00000006009600FA0027
:10894000889FBE008A9FBE008C9FBE000000EB0087
:10895000208F9800CDAB2000CE5491001D407800B0
:10896000E24F4000B40632000C2A02000000000072
:108970000000E0001E0032004E50910025FE07006E
:10898000A8AB2000B8CABF000080FB004200DD0099
:10899000080040000008EB00D6CABF00E14F4000CD
:1089A000030032000479020000000000D6EAEF0064
:1089B000D7CABF00E14F4000030032000479020033
:1089C00000000000D7EAEF00B8CABF000080FB003B
:1089D0004200DD000080E80043C0B3000001EB006E
:1089E0001100200060407C001630020000000000F2
:1089F0007DB897000000E00005003A001D407800B7
:108A00009A2A0200000000000000E0008A063200FE
:108A100009407800FFFD0700B8CABF000081FB00D5
:108A2000C210DD00A0AB2000610078000100200032
:108A3000EB0F5000E08F58007F063E000060010001
:108A4000180037003F00370079013700E302370094
:108A5000060337000F0337004B0437006804370064
:108A600013053700BE0537004106370056063700AC
:108A70000180FB004200DD000080E80022002000B1
:108A80008000EB0060407E00863E02000000000097
:108A9000B8CABF000080FB004200DD0031002000AA
:108AA00098013700A9AB20004210DD000080E800EB
:108AB00060C07C009A2A0200000000000000E00074
:108AC0005D063200E0AD200090568800B8CABF00B5
:108AD0000080FB004200DD001800200008B07C0090
:108AE000D9EAEF00D86AEF0034BE020000000000AF
:108AF000229D2400B306200000014100818149002D
:108B00005256880063568800CEAAEF00D0AAEF0024
:108B1000C22AEF00C42AEF00566BEF00B8CABF00AC
:108B20000080FB004200DD000080E80053C0B3007D
:108B30000001EB008800780060C07C001630020065
:108B400000000000A9AB2000B8CABF000080FB00F5
:108B50004200DD000080E8000002EB0084017800A4
:108B600004017800A1C0B30060C07C00EE3D0200AB
:108B700000000000E10F40001D003A00B8CABF002D
:108B80000080FB004200DD000080E80060C07C0047
:108B9000C22A020000000000000178001800200036
:108BA0000000E00008003A0050002000D056880085
:108BB000B8CABF000080FB004200DD007100200049
:108BC00001B07C000204780034BE02000000000006
:108BD0005256800063568000020050008380580087
:108BE0004240A90012063400A8AB2000BF023700A3
:108BF00034BE020000000000229D2400B3062000C5
:108C00000001410081814900525688006356880066
:108C1000B8CABF000080FB004200DD000080E80011
:108C20000002EB00840178000401780001C2B30067
:108C300060C07C00EE3D020000000000E50F500027
:108C400001003600500020000001E800B8CABF0053
:108C50000080FB004200DD000080E800E1AD200064
:108C600060C07C00863E0200000000003200200050
:108C7000B1C72900E0AD2000980702000000000005
:108C80000000E0000F00320042002000F1C7290080
:108C9000E0AD200098070200000000000000E000A6
:108CA00002003A001000200006003700710020008A
:108CB000D1568800B8CABF000080FB004200DD002A
:108CC00027003700D0568800A9AB2000B8CABF00E3
:108CD0000080FB004200DD000080E8000002EB00A5
:108CE000840178000401780001C2B30060C07C00F8
:108CF000EE3D02000000000000047800B8CABF008A
:108D00000080FB004200DD000080E8000002EB0074
:108D10008801780004017800F1C3B30060C07C00D2
:108D2000EE3D02000000000000017800880F5000B6
:108D3000010036000801780081AB200091407800E6
:108D4000B0062000800F51000700360050002000C0
:108D5000D05688000180FB004200DD007100200039
:108D600001B07C002CFF37000180FB004200DD00D9
:108D70000080E800E1AD200060C07C00863E02007B
:108D8000000000007C0040002BAC20000B004000E5
:108D90000048EB00E0AD200047FD0700ECAD2000EF
:108DA0000C007800DE0802000000000000047800DB
:108DB0007200200041C82900F0AD20009807020091
:108DC000000000000000E0000E003A00F0AD2000BE
:108DD000D864020000000000D9EAB700800020003B
:108DE000DA0AE2000100320090002000D05688002C
:108DF000B8CABF000080FB004200DD002200200056
:108E00006B0337007B0044000B054000F9C2B30040
:108E10009ACF140004003200F0AD2000A67A0200C0
:108E200000000000D6EAB70060AD200080C0EB0073
:108E300090CF10000E003A009ACF140003003200C9
:108E40007C00440009F07D000804E8000C004400A8
:108E5000B1C82900DC070200000000006A044400D9
:108E6000F0AD2000A67A020000000000D6EAB700AC
:108E7000D0AD200000004400E2AD2000E1C2B3000C
:108E80000300370090CF1000030032000000E9001B
:108E9000820F5000FBFF3A000004E800DC2AEF00DC
:108EA000090037008000400080C42900E1007800FC
:108EB00008007800C48C0200000000000004E000FC
:108EC00004003200DC2AEC00E0568000EA0F50007B
:108ED000F4FF3600F0AD2000D8640200000000006E
:108EE000D9EAB700D6CABF00E14F40000B003200FC
:108EF0008A7D0200000000000018A3000700320075
:108F0000D6CABF003C7E0200000000000000E8005E
:108F1000487A020000000000D7EAB700A9AB2000A1
:108F2000B8CABF000080FB004200DD000080E800FE
:108F30000002EB00840178000401780001C2B30054
:108F400060C07C00EE3D02000000000000047800DC
:108F50000000E0001C00320010C0B300D8EAB700E7
:108F6000B8CABF000080FB004200DD000080E800BE
:108F70008E00E80060C07C00063F02000000000098
:108F80000801E90081AB20009140780050072000E3
:108F9000800F51006DFF3E00985680000180FB005D
:108FA0004200DD000080E800E1AD200060C07C00F0
:108FB000863E0200000000000004440060C2B300CE
:108FC000005C780098568800A8AB2000B8CABF00A3
:108FD0000080FB004200DD000080E8000002EB00A2
:108FE0008401780004017800A1C0B30060407C00D7
:108FF000EE3D0200000000000001E800B8CABF001A
:109000000080FB004200DD000080E8008000EB00F3
:1090100060407C00863E020000000000B8CABF002D
:109020000080FB004200DD002100200001307C00B8
:1090300018002000ACAB2000B8CABF000080FB00C5
:109040004200DD000080E8000002EB0084017800AF
:1090500004017800A1C0B30060407E00EE3D020034
:109060000000000000057800E10F400027003A00F2
:10907000B8CABF000080FB004200DD000080E800AD
:1090800060407E00C22A020000000000000178005B
:109090000000E00008003A0050002000D056880090
:1090A000B8CABF000080FB004200DD007100200054
:1090B00001307E000204780034BE0200000000008F
:1090C0005256800063568000020050008380580092
:1090D0004240A900D6043400B8CABF000080FB009B
:1090E0004200DD000080E80060407E001631020092
:1090F00000000000B8CABF000080FB004200DD0095
:10910000B100200001307E0043FE370034BE020073
:1091100000000000229D2400B30620000001410051
:1091200081814900525688006356880081AB200037
:1091300091407800E10F55004DFE32000180FB00A8
:109140004200DD000080E8000002EB008A017800A8
:1091500004017800A1C3B30060407E00EE3D020030
:1091600000000000800578008084E80081AB2000CA
:1091700091407800F08F54000A0036000A01E800A0
:109180000180FB004200DD000080E8008000EB0071
:1091900060407E00863E0200000000000004EB00FC
:1091A000A4FF37007C0447000180FB004200DD0083
:1091B0000080E800090178008800780060407E00A7
:1091C000863E0200000000000B00E800080040009E
:1091D0000048EB00890555000004EB0009C1290097
:1091E000990078007C004700CC07020000000000D6
:1091F000800078000000E000E9003A000804E00088
:1092000069003A00A8AB2000B8CABF000080FB008C
:109210004200DD000080E800810278000102780051
:109220008101780022002000615C290060407C0000
:10923000863C0200000000008004780040B5200059
:109240009156800001005000808F54005300390077
:1092500050002000D0568800B8CABF000080FB0034
:109260004200DD007100200001307C00BD003700AD
:10927000ABAB2000B8CABF000080FB004200DD009D
:109280000080E8000002EB0084017800040178000F
:10929000B1C3B30060C07D00EE3D020000000000DD
:1092A000000478009A56800009017800808F5400ED
:1092B0000100360000017800B8CABF000080FB0042
:1092C0004200DD000080E8008A00780060C07D0078
:1092D000863E0200000000000000450061C2B300AD
:1092E0000158780090568800890F54001D00310005
:1092F000B8CABF000080FB004200DD000080E8002B
:109300008000EB0060C07D0005003700B8CABF00D8
:109310000080FB004200DD000080E80060407C002F
:10932000063F020000000000A8AB2000B8CABF0042
:109330000080FB004200DD000080E8000002EB003E
:10934000840178000401780001C2B30060407C0011
:10935000EE3D020000000000800078000000E00008
:10936000EAFF320086AB2000164378000683FB003C
:109370004233DD008002EB000502780085017800B1
:1093800022002000615C2900C0AB2000664078000C
:10939000863C020000000000800478000900E00024
:1093A000B3FF3A006F003700E14F540046003A0027
:1093B000D94AE2006B003500A8AB2000B8CABF0054
:1093C0000080FB004200DD000080E8006200200019
:1093D0008000EB0060407C00863E02000000000040
:1093E000B8CABF000080FB004200DD000080E8003A
:1093F0008002EB0005027800850178002200200041
:10940000615C290060407C00863C02000000000096
:1094100063044000C80FB20040022000800F5400D7
:109420000100360000047800C90220008E84440048
:1094300011003700B8CABF000080FB004200DD0009
:109440004200200089007800C3AB200060C0790092
:10945000863E020000000000330020000901780071
:109460004100200009007800468B02000000000047
:1094700064045400E38444000800E000EDFF3A0077
:10948000884C7800C10220008E804000A2C3B30047
:10949000400520000E004000914F110003003200F3
:1094A0008100E800808F5000FBFF3A008058EB00FD
:1094B000C00220000E004000046502000000000011
:1094C000D9EAB70027003700E24F540025003A00E0
:1094D000A9AB2000B8CABF000080FB004200DD003D
:1094E0000080E8008002EB0005027800850178002A
:1094F00022002000615C290060C07C00863C0200E4
:109500000000000000017800E90F5000050036005F
:1095100020002000D0568800C22AEF00C42AEF00A5
:10952000100037000E84E800B8CABF000080FB00BE
:109530004200DD000080E8008800780060C07C0008
:10954000863E020000000000080040000048EB00DA
:10955000080078000809020000000000105688008A
:109560002156880085AB2000954278008582FB005B
:10957000C22ADD000002EB008401780004017800BB
:10958000A1C0B300C0AB200065407800EE3D0200F2
:10959000000000008005780018002000050037005A
:1095A0000804E8008984E800E30F54000CFF3A0047
:1095B0000004EB000B01E800B8CABF000080FB000C
:1095C0004200DD008000EB00C3AB200060C07900EA
:1095D000863E02000000000096FE3700D94AE200F5
:1095E0000700350030002000D05688004211DD0011
:1095F00071002000A0AB20000131780006FD37008B
:10960000905680000048EB00E0AD20002AFB0700E8
:1096100090568800ABAB200081AB200091407800D1
:10962000D0568000E80F500005003A000180FB0092
:109630004200DD007100200001B07D00F6FC370023
:109640000180FB004200DD008B0040004000200054
:1096500080087800D84AE20002003A00500020005A
:1096600080087800D86AEF00EBFC37002C65020018
:1096700000000000E20F50006F033200B8CABF00C4
:109680000080FB004200DD00A2AB20005100200062
:1096900001307900A8AB2000B8CABF000080FB00F1
:1096A0004200DD000080E80060407C009A2A020051
:1096B000000000006101B8007056800081568000F3
:1096C000800F5100818F590014003A0034BE02000F
:1096D00000000000525680006356800002005000D7
:1096E000838058004240A9000C003400B8CABF0073
:1096F0000080FB004200DD000080E80060407C004C
:109700001631020000000000B8CABF000080FB0054
:109710004200DD00B100200029033700D15680004F
:10972000E18F50000400320069805000E20F5000C9
:10973000050036000E0137007465020000000000CD
:1097400010479800CF003700EA8F50008E0032009B
:10975000EB8F500065003200E98F5000C5003A00E1
:10976000A9AB2000B8CABF000080FB004200DD00AA
:109770000080E8008002EB00050278008501780097
:109780004200200061C9290060C07C00863C0200C4
:10979000000000000001780081AB200091407800BB
:1097A000E10F40003B0032000180FB004200DD0081
:1097B0000080E8008000EB0060C07C00863E020074
:1097C0000000000012568000235680000001510066
:1097D000E08159001256880023568800B8CABF009D
:1097E0000080FB004200DD000080E80060C07C00DB
:1097F0009A2A020000000000E90F50009D00360088
:109800006C044700B8CABF000080FB004200DD00C6
:109810000080E800A20020008800780060C07C0082
:10982000863E020000000000125680002356800091
:1098300000015100E081590012568800235688002B
:10984000A2002000B1C92900080078009807020092
:10985000000000000000E0000A003A00A000200024
:10986000D0568800EE7C020000000000D6EAB70067
:1098700062002000F00047009E7E02000000000011
:1098800002003700B0002000D056880020002000E1
:10989000790037000180FB004200DD000080E80015
:1098A00060C07C009A2A02000000000064015000A1
:1098B000B8CABF000080FB004200DD000080E80065
:1098C0008000EB0060C07C00863E020000000000CB
:1098D000125680002356800000015100E08159009B
:1098E0001256880023568800620037001856800000
:1098F00029568000AAAB2000B8CABF000080FB0038
:109900004200DD000080E80060407D009A2A0200ED
:109910000000000000045400E0845C001856880039
:1099200029568800B8CABF000080FB004200DD0055
:109930000080E80060407D00DA3002000000000096
:10994000C0F92F00F1FF2F0012568000235680002F
:109950000200400083804800C2F92F00F3FF270077
:10996000820F5000838F580042003600B8CABF00F3
:109970000080FB004200DD007100200001307D000E
:109980000000EB003C003700B8CABF000080FB00BD
:109990004200DD00C1AB200060C078009A2A0200BE
:1099A00000000000800478001256800023568000DA
:1099B00001002000820F5000838F58001B003600EA
:1099C000820478001900370009017800F08F5400F4
:1099D00001003600020120006C044700B8CABF0035
:1099E0000080FB004200DD0088007800C3AB20004F
:1099F00060C07900863E020000000000000178008F
:109A0000105680002156800002005000E08058006F
:109A1000105688002156880082845400D6CABF00A0
:109A2000880078009E7E0200000000000900E0002F
:109A3000E5FF3A001056800021568000E00F5000EC
:109A4000E08F58000B003A00100020007E7E0200DC
:109A500000000000B8CABF000080FB004200DD002B
:109A6000A2AB2000710020000130790009007800CD
:109A70000100370010002000104798000004E000AB
:109A8000470032001E409000E24F50000C003A00A8
:109A9000B8CABF000080FB004200DD00C1AB20005F
:109AA00060C078009A2A0200000000000000E9006F
:109AB0000100200070568800815688005E02370041
:109AC000E14F50002A003A00A8AB2000B8CABF00FE
:109AD0000080FB004200DD000080E80060407C0068
:109AE0009A2A020000000000010020007056880041
:109AF0008156880034BE020000000000229D240030
:109B0000B3062000000141008181490052568800BF
:109B100063568800125680002356800070568000DD
:109B200081568000800F5100818F59000900360056
:109B3000B8CABF000080FB004200DD000080E800E2
:109B400060407C00C22A0200000000000000E0002B
:109B500039023A0060002000D0568800B8CABF0021
:109B60000080FB004200DD0071002000140237007D
:109B7000B8CABF000080FB004200DD00A2AB20009D
:109B8000610020000130790060AD200080C1EB0051
:109B900090CF110009003A0040002000D056880004
:109BA000B8CABF000080FB004200DD007200200048
:109BB000A1AB200002B0780097FB3700C22AEF006B
:109BC000C42AEF00D7CABF00E14F400003003A00AB
:109BD000C6AAEF00C8AAEF000300370061AC20005E
:109BE000847B020000000000B8CABF000080FB00B8
:109BF0004200DD00A2AB200071002000013079009E
:109C0000A8AB2000B8CABF000080FB004200DD0006
:109C10000080E80023C0B3000001EB001100200029
:109C200060407C001630020000000000D05680002A
:109C300000004000C1BC2900E0807800B8CABF0025
:109C40000080FB004200DD000080E80060407C00F6
:109C50000440020000000000D0568000EC0F5000CD
:109C600020003A00B8CABF000080FB004200DD00BF
:109C70000080E800E1AD200060407C00044002006C
:109C800000000000B8CABF000080FB004200DD00F9
:109C90000080E80061CA290060407C0004400200A6
:109CA00000000000B8CABF000080FB004200DD00D9
:109CB0000080E800E1AD200060407C00044002002C
:109CC00000000000B8CABF000080FB004200DD00B9
:109CD0000080E800615C290060407C0004400200D4
:109CE00000000000D0568000E10F50000600360052
:109CF000B8CABF000080FB004200DD00B1002000B8
:109D000001307C00CC013700E0568000EB0F5000A2
:109D10001B003200B8CABF000080FB004200DD001B
:109D20000080E80091CB290060407C0004400200E4
:109D300000000000E056800000004000E15A2900C9
:109D4000E0807800B8CABF000080FB004200DD0060
:109D50000080E80060407C00044002000000000039
:109D6000B8CABF000080FB004200DD000080E800B0
:109D7000615C290060407C0004400200000000009B
:109D8000D6CABF008A7D0200000000000008A300C0
:109D900008003200B8CABF000080FB004200DD00AE
:109DA0000080E80081CC290060407C000440020073
:109DB00000000000B8CABF000080FB004200DD00C8
:109DC0000080E80011CE290060407C0004400200C1
:109DD00000000000D0568000E10F50000500320066
:109DE0003056800041568000E10F4000E08F48006F
:109DF00006003200B8CABF000080FB004200DD0050
:109E00000080E80011CF29000D003700B8CABF005C
:109E10000080FB004200DD000080E800A1CF2900A7
:109E200060407C000440020000000000B8CABF008F
:109E30000080FB004200DD000080E80031D02900F6
:109E400060407C000440020000000000A8AB20003D
:109E5000B8CABF000080FB004200DD000080E800BF
:109E6000615C290060407C000440020000000000AA
:109E700081AB200091407800D84AE2000400320013
:109E80000180FB004200DD00810020004C01370012
:109E90000180FB004200DD000080E800615C2900D9
:109EA00060407C00044002000000000040013700D8
:109EB000E0AD2000A0568800980037000180FB002C
:109EC0004200DD000080E80071D0290060C07D0004
:109ED00004400200000000003B00370000C2B30055
:109EE00080CF500005003A00B8CABF000080FB00D8
:109EF0004200DD00B1C2B3002F003700F0C2B30052
:109F000080CF50000B00360060CCB30000C0400092
:109F1000E64F50000700360050CAB30000C04000B2
:109F2000E54F500003003600A0C7B30080CF5000BB
:109F30001E003600A8AB2000B8CABF000080FB009E
:109F40004200DD000080E80051C2B30060407C00A8
:109F500022400200000000001E4090009A8C020087
:109F60000000000080407800B8CABF000080FB00FD
:109F70004200DD000080E80060407C0022400200DA
:109F8000000000001E409000B08C020000000000A5
:109F900080407800B8CABF000080FB004200DD00AE
:109FA0000080E80060407C0005003700B8CABF00B0
:109FB0000080FB004200DD00C2AB20006040790061
:109FC0002240020000000000A0568000B04078004F
:109FD00011479800A05688000104E000BFFF3A0036
:109FE000B8CABF000080FB004200DD00D1C3B3004F
:109FF0003700370000C2B30080CF500005003A00A0
:10A00000B8CABF000080FB004200DD00B1C2B3004F
:10A010002F003700F0C2B30080CF50000B00360095
:10A0200060CCB30000C04000E64F5000070036008F
:10A0300050CAB30000C04000E54F50000300360096
:10A04000A0C7B30080CF50001E003600A8AB200090
:10A05000B8CABF000080FB004200DD000080E800BD
:10A0600051C2B30060407C002240020000000000AA
:10A070001E4090009A8C0200000000008040780092
:10A08000B8CABF000080FB004200DD000080E8008D
:10A0900060407C0022400200000000001E40900052
:10A0A000B08C02000000000080407800B8CABF00F9
:10A0B0000080FB004200DD000080E80060407C0082
:10A0C00005003700B8CABF000080FB004200DD0079
:10A0D000C2AB200060407900224002000000000076
:10A0E000A0568000B040780011479800A056880024
:10A0F0000104E000BFFF3A00B8CABF000080FB00C7
:10A100004200DD00615C2900C2AB200060407900A4
:10A110000440020000000000D86AED00ABAB200054
:10A1200081AB200091407800D84AE20063FF3A00FA
:10A130000180FB004200DD000080E800615C290036
:10A1400060C07D000440020000000000B8CABF00EB
:10A150000080FB004200DD009100200001B07D0086
:10A16000B8CABF000080FB004200DD00C1AB200088
:10A1700060C07800462A02000000000014568000EB
:10A18000255680003256800043568000040151005D
:10A190008581590001002000800F5100818F5900F6
:10A1A000010036000001BE00820478000200420077
:10A1B000E0804A0010568800215688001A003700B7
:10A1C0008900780002042000828F540001003600CC
:10A1D00082007800ABAB20004A0520000E05450048
:10A1E000D6CABF00010178008A007800A279020077
:10A1F00000000000000478000000E000460032008B
:10A20000B8CABF000080FB004200DD000080E8000B
:10A21000080178008A00780060C07D00623F02007B
:10A2200000000000888454000900E000E4FF3A00C8
:10A230001256800023568000305680004156800020
:10A24000800F5100818F59003E003A00B8CABF000C
:10A250000080FB004200DD00A2AB2000A100200036
:10A2600001307900CE2AEF00D02AEF00D6CABF0015
:10A27000890078002079020000000000D6CABF00E3
:10A280008E00780020790200000000000000E0004D
:10A290000900320010568000215680006100400005
:10A2A000E08048001056880021568800E0C7B300BF
:10A2B0009E4F1000F1FF3A00125680002356800096
:10A2C00061014100E0814900125688002356880050
:10A2D000D7CABF00A1AC2000847B020000000000B0
:10A2E000D7CABF0061AC2000847B020000000000E0
:10A2F000000478000000E00012003A00C6AAEF0057
:10A30000C8AAEF00D7CABF0004790200000000000D
:10A31000D7EAEF000C003700D6CABF00047902006C
:10A3200000000000D6EAEF00B8CABF000080FB00C2
:10A330004200DD00B100200001B07D0018002000C7
:10A34000010037000004EB00B8CABF000080FB002A
:10A350004200DD00C1AB200060C07800462A020048
:10A36000000000000000E00031003A003200370039
:10A37000A8AB20004210DD000080E80060407C00B7
:10A38000462A020000000000EF0F50002A003600AD
:10A3900050568000615680003CF9070070568000DE
:10A3A00081568000E00F5000E08F580022003A00F4
:10A3B000B8CABF000080FB004200DD009100200011
:10A3C00001307C0094F93700D6CABF00E14F40004D
:10A3D000030032000479020000000000D6EAEF001A
:10A3E000D7CABF00E14F40000300320004790200E9
:10A3F00000000000D7EAEF00A8AB2000B8CABF00F9
:10A400000080FB004200DD000080E80060407C002E
:10A410001631020000000000B8CABF000080FB0037
:10A420004200DD00080040000008EB000200370099
:10A430000800E00078F93200AE8990008301E8005E
:10A44000238F9800E4864600E28F510042F93A00DB
:10A450004F06BE004F05BE004F04BE000080FA004C
:10A46000000006000000FA00CD22A90041E2A90088
:10A470004342A80041E2A80000A023004012880047
:10A4800040C2BF000018A300FDFF3A0040C2BF0059
:10A490000008A300FAFF320041E2A9004342A900EC
:10A4A00041E2A80040128000CD22A8000080FB00FD
:10A4B0000080FA00000006000200FA0000017800A7
:10A4C000CD22A900A0032000401288000200E00075
:10A4D000010032000201E90040C2BF000018A300E1
:10A4E000FDFF3A0040C2BF000008A300FAFF32009F
:10A4F00040128000004F78000002EB00E18F500016
:10A500003000360041E2A9004342A80041E2A80021
:10A510004822EF000482E80040C2BF000018A300F8
:10A52000FDFF3A0040C2BF000008A300FAFF32005E
:10A53000431280000200E000040032004818DE00F0
:10A54000104198000281E80003497800048050001F
:10A55000E10F5000EEFF3E0041E2A9004342A90096
:10A5600041E2A800170037004822EF000402E8008B
:10A570000200E0000A0032000201E80040C2BF0011
:10A580000018A300FDFF3A0040C2BF000008A3006E
:10A59000FAFF3200401280000049780009003700BD
:10A5A00040C2BF000018A300FDFF3A0040C2BF0038
:10A5B0000008A300FAFF320040128000004F78002C
:10A5C0000001EB00810F5200E7FF3900CD22A80007
:10A5D000040078000080FA00000006000200FA0083
:10A5E000CD22A90041E2A9004342A80041E2A8000F
:10A5F0000080FB0001A027000100700040128800CD
:10A6000040C2BF000018A300FDFF3A0040C2BF00D7
:10A610000008A300FAFF320041E2A9004342A9006A
:10A6200041E2A80040128000004F7800CD22A8002F
:10A630000080FA00000006000200FA0080017800A5
:10A6400001027800CD22A900A00720004012880056
:10A6500040C2BF000018A300FDFF3A0040C2BF0087
:10A660000008A300FAFF320040128000004F78007B
:10A67000E10F520002003E008000EB003B0037007B
:10A680001380FB004800DD00F20FB20000017100F2
:10A69000134090000080FB0001F02F0001016100D9
:10A6A000000171008381E80041E2A9004342A80053
:10A6B00041E2A800421288000482E900E10F520042
:10A6C000120036001380FB004800DD00F20FB200DC
:10A6D00000017100134090000080FB000101610047
:10A6E000000171008381E80040C2BF000018A30090
:10A6F000FDFF3A0040C2BF000008A300FAFF32008D
:10A7000040128000004F7800EAFF370040C2BF00CF
:10A710000018A300FDFF3A0040C2BF000008A300DC
:10A72000FAFF320040128000004F780041E2A90099
:10A730004342A90041E2A800CFFF370063C0780080
:10A740000080FB004012880040C2BF000018A30038
:10A75000FDFF3A0040C2BF000008A300FAFF32002C
:10A7600040128000004F78008100E800848F500084
:10A77000F2FF3A00CD22A8000080FA000000060097
:10A780000000FA0000017800CD22A9008180FB00C2
:10A790004112880040C2BF000018A300FDFF3A002C
:10A7A00040C2BF000008A300FAFF32004012800040
:10A7B0004822EF0040C2BF000018A300FDFF3A008E
:10A7C00040C2BF000008A300FAFF32004012800020
:10A7D0004822EF0040C2BF000018A300FDFF3A006E
:10A7E00040C2BF000008A300FAFF32004012800000
:10A7F000CD22A80000497800020078000080FA000D
:10A80000000006000200FA00CD22A9000064A000AA
:10A810000080FB004012880040C2BF000018A30067
:10A82000FDFF3A0040C2BF000008A300FAFF32005B
:10A8300040128000004F78000180FB004012880029
:10A8400040C2BF000018A300FDFF3A0040C2BF0095
:10A850000008A300FAFF320040128000004F780089
:10A860000000000000000000CD22A8000080FA00D7
:10A87000000006000000FA00881F780001848000B4
:10A880008100400074844000109A2000800F540022
:10A890000200360020672F000084400088407800C6
:10A8A0000040EB00D7FF0700C840DE0010C0B30037
:10A8B000D4FF07004F0478000080FA000000060073
:10A8C0000200FA00889FBE000004780081447800EE
:10A8D000020F780031CAB30020C0B300C9FF0700DF
:10A8E00091C0B30030C0B300C6FF0700009B20003A
:10A8F0001E0F40009E40780060C0B300C1FF0700FB
:10A900009E40900070C0B300BEFF070061002000B1
:10A910000800780048FF070061002000D0BE20003A
:10A9200045FF070080C0B3002CFF070061C0B300E3
:10A930000904E00001003A008940780001407800F5
:10A9400026FF07004F04BE000080FA00000006004A
:10A950000200FA00CD22A9000074A0000080FB00D4
:10A960004012880040C2BF000018A300FDFF3A005B
:10A9700040C2BF000008A300FAFF3200401280006E
:10A98000004F78000180FB004012880040C2BF00E9
:10A990000018A300FDFF3A0040C2BF000008A3005A
:10A9A000FAFF320040128000004F7800CD22A8004C
:10A9B0000080FA00000006000000FA00881F7800FE
:10A9C0007E10E20011003A0010002000F0838800A1
:10A9D000188480000804E900109A2000800F5400B9
:10A9E000010036000004780001C4B300E0C1B300E8
:10A9F000D7FF070088407800C0C0B30081FF070080
:10AA0000C840DE00D0C0B3007EFF07004F047800CE
:10AA10000080FA00000006000200FA00CD22A90022
:10AA20000080FB00000AB3004012880040C2BF0053
:10AA30000018A300FDFF3A0040C2BF000008A300B9
:10AA4000FAFF320040128000004F78000180FB00C6
:10AA50004012880040C2BF000018A300FDFF3A006A
:10AA600040C2BF000008A300FAFF3200401280007D
:10AA7000004F7800CD22A8000080FA0000000600F8
:10AA80000200FA00000F780031C0B300F0C1B3003B
:10AA9000E1FF07009E409000F0C1B300ACFF07004B
:10AAA0000080FA00000006000000FA00881F78000D
:10AAB0000044780050312000F1FF07008840780002
:10AAC00050C1B3004FFF07000000EB00ECFF070090
:10AAD0004F0478000080FA00000006000400FA002D
:10AAE000881F780000447800010F78004021200082
:10AAF000E3FF07008840780040C1B30041FF070032
:10AB00009E40780060C1B3003EFF07009E40900069
:10AB100070C1B3003BFF0700A0302000D8FF070042
:10AB2000A1C0B3000E80E80015FF07002E40900082
:10AB30000008A300FAFF3A000000EB00D0FF070076
:10AB40004F0478000080FA00000006000400FA00BC
:10AB5000889FBE00800478000144780040212000D6
:10AB6000C7FF07008840780040C1B30025FF0700F9
:10AB700011C0B30020C1B30022FF0700A0302000A5
:10AB8000BFFF0700A1C0B3000E007800FCFE070065
:10AB90001E40780061446000FAFF3A004021200026
:10ABA000B7FF07008840780020C1B30015FF0700F9
:10ABB00081C1B3000E00E800F1FE07001E409000C6
:10ABC0000080FB0001F02F00010464000004740009
:10ABD00091C1B3000E80E800E9FE07002E4090000E
:10ABE0004800DD00F80FB200000474000000EB0024
:10ABF000A3FF0700880C7800090078004F04BE000E
:10AC00000080FA00000006000200FA0011C0B30044
:10AC10000E007800CDFF07001E0078004200DE0025
:10AC2000610060000080FA00000006000000FA00E9
:10AC300000017800CD22A9008180FB00411288002C
:10AC400040C2BF000018A300FDFF3A0040C2BF0091
:10AC50000008A300FAFF3200401280004822EF00F3
:10AC600040C2BF000018A300FDFF3A0040C2BF0071
:10AC70000008A300FAFF320040128000CD22A80095
:10AC800000497800020078000080FA000000060009
:10AC90000200FA00881F78005031200078FF07007A
:10ACA00051C1B3000E007800E0FF07001E84FB00D6
:10ACB0000000EB0072FF0700080078004F047800E6
:10ACC0000080FA00000006000200FA0001C2B30092
:10ACD000E0C1B30050FF0700D1C1B3000E007800FF
:10ACE000D2FF07009E40780061C06000FAFF32008A
:10ACF00041C0B300F0C1B30015FF07000080FA00A7
:10AD0000000006000200FA0041C0B300F0C1B30029
:10AD100041FF0700D1C1B3000E007800C3FF070058
:10AD20009E40780064C06000FAFF3A00F1C1B300B1
:10AD30000E00E800BDFF07001E4090000038A30091
:10AD4000FAFF3A0001C2B300E0C1B30000FF070000
:10AD50000080FA00000006000200FA00F1C1B30012
:10AD60000E007800B1FF07001E80FB004500DE00EA
:10AD70000000A200610060000080FA0000000600F0
:10AD80001000FA00889FBE008A9FBE008C9FBE0004
:10AD9000000F780011079800220798000005EB00CB
:10ADA0008A0578000080EB009E0F10000200320040
:10ADB0008A0678000C00370021C0B3006600470007
:10ADC0009AFF07006E4090000080FB00000F7800A3
:10ADD00031C0B3006700470094FF07007E40900039
:10ADE000104798001D0020000006EB001E00900098
:10ADF000E10F40000C003A008040EB006800470083
:10AE00008AFF07000E4890000080FB0010079800A2
:10AE100011C0B3006900470084FF07001E4890007E
:10AE2000304798001C002000AE049000E18F5400D1
:10AE30003F003E000C00E0000C003A008C4078001F
:10AE40006A00470079FF07002E4890000085FB004C
:10AE500011C0B3006B00470074FF07003E4890002C
:10AE60004800DD00FA0FB200000575000D00E0009B
:10AE70000C003A0021C0B3006C0047006BFF0700D4
:10AE80004E4890008085FB0031C0B3006D00470044
:10AE900066FF07005E4890004800DD00FB0FB2002F
:10AEA00080857500AE4090000040EB0055FE070025
:10AEB000BE40900010C0B30052FE07009E407800D4
:10AEC00020C0B3004FFE07009E40900030C0B3008A
:10AED0004CFE07000004EB000300370061FD070093
:10AEE000BEFD07000804E800890F5400FBFF3A008C
:10AEF0000C00E00006003A008A4078000C40780020
:10AF000040FE0700C850DE0010C0B3003DFE070041
:10AF10000D00E0004E003A008B40780020C0B300E6
:10AF200038FE0700C858DE0030C0B30047003700C5
:10AF30000D00E000080032001E84440088407800C4
:10AF400020C0B3002FFE07004844DE008840780090
:10AF500030C0B3002BFE07001E049000088544009B
:10AF60008A04E90029079800F1C1B3006E00470088
:10AF70002EFF07006E4890000058A300FAFF3A0029
:10AF8000AE40900000C1B3001EFE0700BE4090001E
:10AF900010C1B3001BFE07009E40780040C1B30003
:10AFA00018FE07009E40900050C1B30015FE070038
:10AFB000109A2000800F540005003E00808F54003E
:10AFC00003003600D0652F000000450020079800E0
:10AFD000640547009A40780020C1B30009FE0700CD
:10AFE000E50447009940780030C1B30005FE070032
:10AFF00001C1B300F0C1B30087FE070001C2B30076
:10B00000F0C1B30052FE07000C00E0001000320057
:10B010002E0190008200E80021079800109A20007D
:10B02000800F540004003E00808F50000200360064
:10B0300000005100200798009A4078000040EB0083
:10B04000F0FD07009940780010C0B300EDFD070047
:10B050004F06BE004F05BE004F04BE000080FA0040
:10B06000000006001A00FA00889FBE008A9FBE00FA
:10B070008C9FBE00800578008040EB007600470082
:10B08000EAFE07006E5090000080FB0001F02F00E8
:10B09000010565000005750011C0B3007700470089
:10B0A000E2FE07007E509000005F98004800DD003F
:10B0B000FA0FB200000575006066B800190037008D
:10B0C0008B007800F48F550001003600410120000C
:10B0D0000E047800011C780008007800F6FC0700D8
:10B0E0009E00780081855500618060000300320079
:10B0F0000040EB0080707C001E0FE8009E0078008E
:10B10000080178000400370032007800000646008D
:10B11000E0864E008180E9000100E000FAFF3A007D
:10B12000010F78000B00E000E5FF3A000C04BE00C0
:10B130008A4078000B407800B2FD07008E589000DE
:10B1400010C0B300AFFD07006148B8000C0040001C
:10B15000E0804800010040000080EA004F06BE0089
:10B160004F05BE004F04BE000080FA00000006003C
:10B170000200FA00889FBE008A9FBE008105780009
:10B18000018480008100400074844000109A2000F7
:10B19000800F54000200360020672F00008440001A
:10B1A0008040EB000E007800A0FE07000E00780043
:10B1B0003081FB0001F02F000105650002057500DC
:10B1C00011C0B30099FE07009E4490004848DD007E
:10B1D000FA0FB20000057500884078000040EB00CF
:10B1E00088FD0700C840DE0010C0B30085FD0700E1
:10B1F0000B0078009BFF0700000478008A4078006D
:10B200000040EB007FFD07008940780010C0B300CC
:10B210007CFD0700080078004F05BE004F04BE000B
:10B220000080FA00000006000400FA00881F780081
:10B230000E017800001978008040EB0002007800D1
:10B240007AFE07002E4090000080FB0001F02F00E6
:10B25000010464000004740011C0B30063004700DF
:10B2600072FE07003E4090004800DD000884FB00AD
:10B27000000474009E4078000040EB0061FD070070
:10B280009E40900010C0B3005EFD070008007800EB
:10B290004F0478000080FA00000006000400FA0065
:10B2A000881F78000E0178000019780021C0B300D3
:10B2B000020078005DFE07002E4090000080FB0039
:10B2C00001F02F00010464000004740031C0B300D9
:10B2D0006300470055FE07003E4090004800DD0037
:10B2E0000884FB00000474009E40780020C0B30076
:10B2F00044FD07009E40900030C0B30041FD0700B0
:10B30000080078004F0478000080FA000000060072
:10B310001000FA00889FBE008A9FBE008C9FBE006E
:10B3200001C8B300F0C1B30089FD070001C8B30034
:10B33000F0C1B300B8FD0700A1C0B300C0C1B300A5
:10B34000B5FD070081C0B300F0C1B30080FD070068
:10B350007CD0BF0065405000E14F500072003E00BD
:10B360000004EB00C1C1B300680047002FFE0700D6
:10B370000E4890006A00600004003A000804E800EB
:10B38000803E2000800F5400F6FF3A00C1C1B30098
:10B390006900470025FE07001E4890000018A30022
:10B3A00003003A00703E2000800F54005E0036001B
:10B3B00081C0B300F0C1B30097FD07008040EB00EF
:10B3C0006A00470019FE07002E4890000080FB002D
:10B3D00008F02F00888464008084740011C0B300DA
:10B3E0006B00470011FE0700BE4D90004858DD007D
:10B3F000F90FB2008084740061C0B3006C00470094
:10B400000AFE07004E4890000080FB00080464001C
:10B410000004740071C0B3006D00470003FE070014
:10B420005E4890004800DD00F80FB2000004740090
:10B430000804E80008467800884078000040EB00E7
:10B44000F0FC07004844DE0008457800884078009A
:10B4500010C0B300EBFC07008E06780081002000CE
:10B460000E00780014FC070008C1B300C1C1B3008E
:10B470006E004700EDFD07006E4890000018A30025
:10B48000230032001E00900000D8A30020003200EC
:10B4900001C8B300F0C1B3002DFD070001C8B3001F
:10B4A000F0C1B3005CFD0700A1C0B300C0C1B30090
:10B4B00059FD070081C0B300F0C1B30024FD0700AF
:10B4C000C1C1B3006F004700D8FD07007E4890005F
:10B4D0006A006000FAFF320081C0B300F0C1B3001F
:10B4E0004DFD07008C4078000040EB00C5FC0700D4
:10B4F0008A40780010C0B300C2FC07008100200021
:10B500000D007800ECFB07000844E900D7FF3A0083
:10B51000894078000040EB00BAFC07008B407800BF
:10B5200010C0B300B7FC07004F06BE004F05BE00B9
:10B530004F04BE000080FA00000006001600FA006A
:10B54000889FBE008A1F780000057800810478007B
:10B55000901120004AFD070091C1B300740047001C
:10B56000B2FD07004E5490000000EB0044FD0700C0
:10B570000000EB000804E0003A0032007E10E20018
:10B5800003003A000CFD07000000EB003500370017
:10B590001084800000848800010821009140780018
:10B5A0000040EB0097FC0700110821009140780053
:10B5B00010C0B30093FC0700410120000E0078008A
:10B5C000BDFB07001E0890000C8D0200000000006B
:10B5D000100F98009E017800109A2000808F510073
:10B5E0000D003E009E40780061C060000A003A00F5
:10B5F0002E019000000128000000610006003A00C2
:10B600009E009000E05E2000808F500002003E000F
:10B610000278A30001003A000000FE0013848800B5
:10B620006C00470005000900305D78006A00B10039
:10B630006000B10080CCEB003E509000E84F50001D
:10B6400006003A002E5090000004E0000200320094
:10B65000E64F500001003A00804C78007E30EF0049
:10B66000100020004F0578004F04BE000080FA0053
:10B67000000006000600FA00889FBE008A1F7800BE
:10B6800090112000FEFC070091C1B3000E0078006D
:10B6900066FD07001E447800E0002000F8FC07006B
:10B6A000E1C0B3000E00E80060FD07001E409000FE
:10B6B0000080FB000AF02F008A84640080847400FC
:10B6C000F1C0B3000E80E80058FD07002E40900046
:10B6D0004800DD00F90FB200808474009011200052
:10B6E000E7FC070091C1B300630047004FFD07006E
:10B6F0003E409000884F5000E3FF3A00C000200019
:10B70000DFFC0700C1C0B3006400470047FD07002D
:10B710004E4090000080FB000A04640000047400A6
:10B72000D1C0B3006500470040FD07005E409000B7
:10B730004800DD00F80FB20000047400888F540048
:10B740000400360088805400109A20000100500048
:10B7500005003700109A2000888F54000200320044
:10B76000090054000000E9004F0578004F04BE00B6
:10B770000080FA00000006000200FA00F1C1B300E8
:10B780000E00780029FD07001E80FB004300DE004C
:10B790000000A200610060000080FA0000000600C6
:10B7A0000400FA00889FBE00CD22A800C922A9008B
:10B7B0004022EF00F0002000101288004422EF0029
:10B7C0004302A80042A2A80041E2A80001C2B300BF
:10B7D000E0C1B30090FC070010002000E8C30200A5
:10B7E00000000000CD22A900F00F200040128800C8
:10B7F00040C2BF000018A300FDFF3A0040C2BF00D6
:10B800000008A300FAFF320040128000004F7800C9
:10B81000CD22A80010002000E8C3020000000000B4
:10B82000D1C1B3000E80E80000FD07002E4090005B
:10B830000080FB000038A300E4FF3A000080EA002B
:10B84000E1046000E1FF3A0018002000F88388005E
:10B85000198488008940780080C0B300E9FB0700A4
:10B860008940780090C0B300E6FB070011CAB3001E
:10B87000C0C0B300E3FB070091C0B300D0C0B30069
:10B88000E0FB070011CAB300A0C0B300DDFB070056
:10B8900091C0B300B0C0B300DAFB070021CAB30007
:10B8A00040C0B300D7FB070091C0B30050C0B30045
:10B8B000D4FB070021CAB30020C0B300D1FB0700AE
:10B8C00091C0B30030C0B300CEFB07000940780040
:10B8D00042FB07000020200069FC0700D1C0B30034
:10B8E00009407800C7FB070021C3B30020C0B300A4
:10B8F000C4FB070021C1B30040C0B300C1FB070077
:10B9000001C4B30030C0B300BEFB0700F1C3B300F5
:10B9100090C0B300BBFB070021C1B30060C0B300FF
:10B92000B8FB0700C1C0B30070C0B300B5FB07008F
:10B93000E1CEB300A0C0B300B2FB070051C0B3001A
:10B94000B0C0B300AFFB0700403020004CFC070044
:10B95000D1BE20009140780040C0B300A9FB070091
:10B96000E1BE20009140780050C0B300A5FB070065
:10B97000F1BE20009140780020C0B300A1FB070079
:10B9800001BF20009140780030C0B3009DFB07004C
:10B9900011BF2000914078000940780099FB070012
:10B9A00021BF2000914078000840780095FB0700F7
:10B9B0008940780050C1B30092FB070021C1B30059
:10B9C0006300470099FC07003E4090007CF0B70000
:10B9D0000110200000C1B30040FC070021472300F4
:10B9E00040C1B3003DFC07008900780009407800A1
:10B9F0003AFC07000900780021FC070041C0B300B1
:10BA0000F0C1B300D2FB07004F04BE000080FA0073
:10BA1000000006000000FA00BA10E20003003A003D
:10BA200010002000D0858800C2EFEF00C2CFBF0019
:10BA3000E14F400003003200488E02000000000089
:10BA4000C2EFEF0020002000607E8800CE2FEF00C4
:10BA500010002000207E8800C66FEF00C68FA8006F
:10BA6000C62FA8000080FA00000006000000FA00BF
:10BA7000C2CFBF00E14F400003003200488E0200F9
:10BA800000000000C2EFEF00C42FEF000080FA00BA
:10BA9000000006000000FA00C40FE20006003A00B1
:10BAA00020002000607E8800CE2FEF0010002000D4
:10BAB000207E8800C60FA9000080FA000000060062
:10BAC0000000FA00207E80000000E000010032004B
:10BAD000100020000080FA00000006000000FA00BC
:10BAE000307E8000610060000080FA0000000600E7
:10BAF0000000FA00307E8000620060000200320028
:10BB0000C62FA900100020000080FA0000000600E7
:10BB10000000FA00307E80004300DE00610060001B
:10BB20000080FA00000006000000FA00C07E8000DD
:10BB3000D17E8000C0EBB7004801DE000200780033
:10BB4000C1EBB70001007800C2EBB7004808DE0087
:10BB5000C3EBB7000080FA00000006000800FA00FE
:10BB6000881F78000040EB00104798000E80E80026
:10BB70006C910200000000002E409000E24F500047
:10BB8000E0003A00C00120003E90020000000000EA
:10BB9000D8BE20000E80E8006C910200000000007A
:10BBA0002E409000984F5000ED003A000804E80045
:10BBB00030BF2000800F5400F6FF3A00C64FAB00A4
:10BBC00008003A00000120003E9002000000000042
:10BBD0004100200080FD2000949102000000000040
:10BBE000EC0FA800000F20003E90020000000000B3
:10BBF0000E84E800080078006C910200000000004C
:10BC00000000E000BF003200AE40900030C3B3003F
:10BC100080CF50008A00320007003E00E3CF500082
:10BC200031003200E6CF50004E003200E1CF50002C
:10BC3000AA003A001700370060C3B30080CF50005D
:10BC40006C003200E1CF4000AE0032000040E9005D
:10BC500080CF5000A1003A00080078006C910200EB
:10BC6000000000002E409000E14F5000BC003A0060
:10BC70000E00E8006C91020000000000C64FAB000F
:10BC8000DBFF32001E409000E24F5000D8FF3A0028
:10BC9000B3003700080078006C910200000000003B
:10BCA0002E409000E44F5000AD003A00C64FAB006C
:10BCB00007003200004478000E80E8006C9102001A
:10BCC000000000000844E900C9FF3200FAFF370015
:10BCD0004100200000FE20009491020000000000BE
:10BCE000EC4FA800C2FF37000E0078006C910200F4
:10BCF0000000000030C0B3009E4F100098003600D6
:10BD0000C64FAB000700320048C0B3000E80E80009
:10BD10006C910200000000000844E90006003200B7
:10BD2000FAFF370041002000C0FD2000949102007E
:10BD300000000000EC2FA8009E40780064CF500067
:10BD4000030037000E80E8006C9102000000000044
:10BD50001E40E900004F7800E14F4000F9FF3A0033
:10BD6000A3FF37000E0078006C9102000000000075
:10BD700034C0B3009E4F120079003600C64FAB00AE
:10BD800017003A004100200040FE2000949102007C
:10BD900000000000EC6FA8009E40780064C05000D6
:10BDA000004F7800E34F50000D003600C64FAB0047
:10BDB0000B003A004100200080FE20009491020018
:10BDC00000000000EC8FA8001E427800644F520073
:10BDD000030037000E80E8006C91020000000000B4
:10BDE0001E40E900004F7800E14F4000F9FF3A00A3
:10BDF0007FFF3700080078006C910200000000000F
:10BE00002E409000E44F500055003A006700470074
:10BE10006C91020000000000660047006C91020077
:10BE200000000000650047006C9102000000000067
:10BE3000640047006C910200000000006CFF3700B6
:10BE4000080078006C910200000000002E40900075
:10BE5000E44F500042003A00C64FAB0008003200E9
:10BE60000044EB000E80E8006C910200000000002E
:10BE70000844E800E44F54005DFF3200F9FF37004A
:10BE800030FD20006C9102000000000020FD200029
:10BE90006C9102000000000010FD20006C91020077
:10BEA0000000000000FD20006C9102000000000076
:10BEB000807E8000917E8000C509DE004B0ADD0097
:10BEC0004501DE000201720002005000838058002C
:10BED000807E8800917E880045FF37000E00780044
:10BEE000010037000E80E8006C91020000000000A5
:10BEF0001E40E900004F7800E14F4000F9FF3A0092
:10BF00003BFF37001E409000E24F500006003A0011
:10BF10002E009000BE009000A07E8800B17E8800B8
:10BF2000C64FA80009003700A27E8000B37E8000C3
:10BF30002E009000BE009000800F5100818F5900AC
:10BF4000020032000040EB0010479800C29102004E
:10BF5000000000001E4090000080FB00030037003E
:10BF6000C2910200000000000000EB004F047800C6
:10BF70000080FA00000006000000FA00889FBE0062
:10BF80008A1F7800804478000105780010C0B30053
:10BF9000809002000000000010C0B30080900200FA
:10BFA0000000000060C0B3008090020000000000AC
:10BFB0000040EB00809002000000000020C1B300B0
:10BFC000809002000000000030C2B30080900200A8
:10BFD0000000000040C3B300809002000000000099
:10BFE00060C5B30080900200000000000040EB003C
:10BFF00080900200000000000040EB0080900200F2
:10C00000000000000040EB00C68FAB0001003A00CA
:10C0100000C8B30080900200000000000040EB0068
:10C020008090020000000000E3CF540007003A00B7
:10C030000A00E000050032004100200080FD2000E1
:10C04000AA900200000000000C0037000040EB0046
:10C0500080900200000000000040EB008090020091
:10C06000000000000040EB00809002000000000093
:10C070000040EB0080900200000000000044EB0054
:10C080000040EB0080900200000000000844E8003F
:10C09000EC4F5400FAFF3A0061002000D0BE2000AF
:10C0A000AA90020000000000A8CCB3000040EB0002
:10C0B00080900200000000000844E900FBFF3A0005
:10C0C00030C6B300809002000000000020C8B3001A
:10C0D000809002000000000030C5B3008090020094
:10C0E0000000000030C6B300809002000000000095
:10C0F00050C3B300809002000000000010C0B300E5
:10C10000809002000000000009407800809002004A
:10C1100000000000E1CF540002003A00C64FA90021
:10C1200016003700E3CF540014003A000A00E00084
:10C1300012003A0060C3B3008090020000000000CB
:10C1400040C0B3008090020000000000D7CFBF00C5
:10C150008090020000000000D6CFBF008090020057
:10C1600000000000D5CFBF0080900200000000005A
:10C17000D4CFBF00809002000000000070C3B30065
:10C18000809002000000000040C0B30080900200D8
:10C190000000000010C0B30080900200000000000A
:10C1A00030C0B300809002000000000060C0B30007
:10C1B0008090020000000000C0C0B3008090020028
:10C1C00000000000E3CF540003003A000A00E00042
:10C1D0000800320011003700E1CF54000F003A0090
:10C1E000C07E8000D17E8000E00F5000E08F5800BC
:10C1F0000A00320020C3B30080900200000000005B
:10C2000040C0B30080900200000000004100200008
:10C2100080FD2000AA90020000000000C0C0B30012
:10C2200080900200000000000004EB00C2BD20006E
:10C2300001C2B30068407900814F50000300320012
:10C240000804E800EF0F5400FAFF3A0008407800B5
:10C25000809002000000000088007800C0BD20002F
:10C26000AA9002000000000000C0EB0001003700AF
:10C270000040EB008090020000000000417580004B
:10C28000B0122000808F5000F9FF360001BC200062
:10C29000914078008180FB00C1CBBF004800DD00E9
:10C2A0000104700021BC2000914078008180FB00D7
:10C2B000C3CBBF004800DD00810470000A00E0002D
:10C2C00006003A000005FD00C0EBB700C1EBB70067
:10C2D000C2EBB700C3EBB7000005FD00F49002000D
:10C2E0000000000008007800C0EBB7004840DE0006
:10C2F000C1EBB70009007800C2EBB7004848DE0088
:10C30000C3EBB7004F0578004F04BE000080FA0071
:10C31000000006000000FA00889FBE008A9FBE0051
:10C320008C9FBE00207E8000010020006100500034
:10C33000E0805800EB0F5000E08F58007A013E007B
:10C34000006001000B003700150037005700370070
:10C350006200370092003700F700370022013700F3
:10C360004A01370020013700480137001E0137001D
:10C370004601370034042000430420000041EB0054
:10C380006000B800828E020000000000C2EFB7001B
:10C39000E14F40006401320020002000207E880030
:10C3A000C0032000807E8800D22FEF00EC6FEF00EA
:10C3B000C60FA900C64FA9000456020000000000E5
:10C3C0000000E00058013200C2CFBF0052900200CE
:10C3D00000000000B1122000810F50005201360011
:10C3E000317E80004408DE000080EA0061006000C9
:10C3F0004400DD000140A10080807000317E880093
:10C40000C2CFBF0082C1B3000440BC00C0EA20001C
:10C4100000004100A2002000F10F2000EC07020004
:10C42000000000008000EB0010C0B300D2FE070047
:10C4300034BE0200000000000006BE00607E8000E6
:10C44000717E80006011B800A42526002500200020
:10C450006033B800E2040200000000000205BE00E4
:10C460000004BE007C8902000000000001002000E2
:10C470000200200003002000A42526002500200043
:10C480006033B800400602000000000008044000CD
:10C49000898448000C0444008D844C00487E880048
:10C4A000597E8800300020001E013700C2CFBF0037
:10C4B0004C91020000000000910F2000810F5000FD
:10C4C0003D003600C66FA800A4FD0700E24F5000F3
:10C4D00015013A0040002000207E8800C2CFBF0036
:10C4E000529002000000000011102000810F500047
:10C4F0000D013600C2CFBF0082C1B3000440BC00B2
:10C50000C0EA200000004100A20020008180E90074
:10C51000EC070200000000008000EB0030C0B30018
:10C5200095FE070034BE0200000000000006BE00B9
:10C53000607E8000717E80006011B800A425260016
:10C54000250020006033B800E20402000000000073
:10C550000205BE000004BE007C890200000000004D
:10C56000010020000200200003002000A425260076
:10C57000250020006033B8004006020000000000E3
:10C5800008044000898448000C0444008D844C0059
:10C59000487E8800597E880050002000E100370066
:10C5A000C2CFBF004C91020000000000910F20009C
:10C5B000810F500013003E0034BE02000000000056
:10C5C000427E8000537E800002005000838058002D
:10C5D0004240A900D4003400607E8000717E80005B
:10C5E000F2032000820F5000E08F5800CC003E0084
:10C5F0000000400081804800607E8800717E8800D5
:10C60000C700370055FD0700E54F5000B5003A0060
:10C61000C2CFBF00488E020000000000C2EFEF0052
:10C6200034BE020000000000407E8800517E880079
:10C6300060002000207E8800C62FA800C60FA8003A
:10C64000637F80000308A3000A003200C07E8000E0
:10C65000D17E8000C0EBB7004801DE000200780008
:10C66000C1EBB70001007800C2EBB7004808DE005C
:10C67000C3EBB7000328A3000A003200007F80004C
:10C68000117F8000C4EBB7004801DE000200780093
:10C69000C5EBB70001007800C6EBB7004808DE0024
:10C6A000C7EBB7000318A3000A003200E07E800049
:10C6B000F17E8000C8EBB7004801DE000200780080
:10C6C000C9EBB70001007800CAEBB7004808DE00EC
:10C6D000CBEBB7000338A30008003200207F8000B6
:10C6E000CCEBB7004800DE00CDEBB700307F800018
:10C6F000CEEBB7004800DE00CFEBB700D06BEF0009
:10C70000D16BEF00D26BEF00D36BEF000348A300B7
:10C7100085003200407F8000D0EBB7004800DE008B
:10C72000D1EBB700507F8000D2EBB7004800DE00AD
:10C73000D3EBB7007C00370034BE020000000000DD
:10C74000487E8000597E8000080050008980580093
:10C750009225260023002000820F5000838F58006E
:10C76000710036003200200003002000607E80004F
:10C77000717E80001403020000000000827E8000B1
:10C78000937E8000800F5100818F59000B0036008E
:10C79000A0252600210020000800400089804800D4
:10C7A000407E8800517E880061005100E080590081
:10C7B000807E8800917E88005B0037003404200072
:10C7C000430420000041EB006000B800828E0200AC
:10C7D00000000000C2EFB700E14F400052003200FD
:10C7E00070002000207E8800C2CFBF00529002005F
:10C7F0000000000011102000810F50004A00360098
:10C800001100200030C0B300DBFD0700C64FA900B7
:10C8100034BE0200000000000006BE00607E800002
:10C82000717E80006011B800A4252600250020003C
:10C830006033B800E2040200000000000205BE0000
:10C840000004BE007C8902000000000001002000FE
:10C850000200200003002000A4252600250020005F
:10C860006033B800400602000000000008044000E9
:10C87000898448000C0444008D844C00487E880064
:10C88000597E8800C42FEC0027003700C2CFBF00BC
:10C890004C91020000000000910F2000810F500019
:10C8A0000D003E0034BE020000000000427E800009
:10C8B000537E800002005000838058004240A9004F
:10C8C00019003400C40FEC00207E8800EC0F5000EB
:10C8D0001500360012003700A0FC0700E54F50009D
:10C8E00003003200E64F50000F003A000C00370002
:10C8F000C2CFBF00488E020000000000C2EFEF0070
:10C9000034BE020000000000407E8800517E880096
:10C9100060002000207E8800C62FA800020037009B
:10C9200020002000207E88004F06BE004F05BE007C
:10C930004F04BE000080FA00000006000000FA006C
:10C94000E0508800D05088000080FA000000060007
:10C950000000FA0042A2200001AB2000E0A120006C
:10C96000C8BB02000000000000AB20000080FA00FD
:10C97000000006000000FA000080FA000000060037
:10C980000000FA000000EB00AA50E20002003200B2
:10C99000AA70EF00100020000080FA0000000600DE
:10C9A0000000FA0040A220000080FA00000006000B
:10C9B0000000FA00881F7800000478007200200050
:10C9C000A1622A0098070200000000000000E000B9
:10C9D000080032004200200021632A00080078008D
:10C9E0009807020000000000010820000000E0009D
:10C9F00001003A008000EB00010078004F0478004D
:10CA00000080FA00000006000000FA00881F78008D
:10CA10000104780071632A00CC07020000000000C6
:10CA20000000E00007003A00D1632A000800780007
:10CA3000CC07020000000000010820000000E00018
:10CA4000010032008000EB00010078004F04780004
:10CA50000080FA00000006000000FA00889FBE0077
:10CA600071642A00E0AD2000C64102000000000011
:10CA7000000478000000E00017003200C0C3B300DB
:10CA8000984F100014003A008004EB00E8C07C00CE
:10CA9000E0A1200064BC0200000000000000E000F3
:10CAA00006003200E20F5000060032008904E80060
:10CAB000FE8F540008003200F4FF3700AAF0B700E0
:10CAC0000500370010C0B300AAF0B700E0A12000B5
:10CAD000D6BB0200000000000000EB004F04BE00C7
:10CAE0000080FA00000006004A00FA00889FBE009D
:10CAF0008A9FBE000E84E800D6CABF004201200013
:10CB000088007800D87D020000000000920020001C
:10CB1000F1642A0008007800980702000000000075
:10CB20000000E00003003A00400120000000E9009E
:10CB3000FEFF3A0022012000C1652A000E80E800B5
:10CB400098070200000000000002EB000000E00077
:10CB5000FA003A001856800029568000ABAB20003E
:10CB6000B8CABF000080FB004200DD000080E80082
:10CB700060C07D009A2A02000000000000057800D5
:10CB8000B8CABF000080FB004200DD000080E80062
:10CB900060C07D00C22A02000000000000004500C5
:10CBA00001002000800F5400818F5C00DA003E00FD
:10CBB000B8CABF000080FB004200DD000080E80032
:10CBC00060C07D009A2A0200000000006101B800E8
:10CBD000140020001056800021568000800F510064
:10CBE000818F5900D50039003303200076014700BA
:10CBF0006000200001002000C0A70200000000002B
:10CC00001E2090000060A100A500370061002000F8
:10CC1000E0AD20002C430200000000000000E00016
:10CC2000BD003A000107200040AE20005043020042
:10CC3000000000000000E000B7003A00E8AD20006E
:10CC4000F1662A0008007800CC070200000000000E
:10CC50000000E0000C003A007604470088007800ED
:10CC600040AE20008E8A0200000000000000E000BC
:10CC7000A900320018007800CE08900050179800E4
:10CC8000611798008700370021672A0008007800A4
:10CC9000CC070200000000000000E00002003A00A3
:10CCA000FE0047002300370051672A000800780083
:10CCB000CC070200000000000000E0000C003A0079
:10CCC0007A0447008800780040AE20008E8A020077
:10CCD000000000000000E0008F0032001800780023
:10CCE000EE08900070179800011F98006D00370043
:10CCF00091672A0008007800CC07020000000000BD
:10CD00000000E00003003A00210220008E80400075
:10CD100008003700E1672A0008007800CC0702000D
:10CD2000000000000000E00008003A00610220005E
:10CD30008E80400040AE20008E8A0200000000007D
:10CD40000000E00057003A007300370031682A0005
:10CD500008007800CC070200000000000000E0009E
:10CD600034003A0043AE20000041780007CDB30004
:10CD7000F6CBB300F5C9B30024AC200008C3B30060
:10CD8000010037008301E800934078000104E000CF
:10CD90000A00320007C04000E94F50000E00360084
:10CDA00006C04000E54F50000B00360005C04000B3
:10CDB000E54F5000F3FF3E00070037000280FB0004
:10CDC0007C00400008707A000241E800EB4F5100FF
:10CDD00008003E00F9FF37000280FB007C004000A5
:10CDE00001707A008301E8000241E800EB4F510036
:10CDF000E5FF3600E8AD20003A0420000E054500AE
:10CE0000184078001047980098409000014F780033
:10CE10001E0078003A8C020000000000005D7800DF
:10CE20000884E800A0AE2000800F54001D003200EE
:10CE3000F3FF370071682A0008007800CC07020071
:10CE4000000000000000E0000A003A0040AE2000B0
:10CE50009C8D020000000000200320000E00400016
:10CE600041AE20000F000900315878000001B100E8
:10CE70000C003700C1682A0008007800CC070200C7
:10CE8000000000000000E00006003A0010C3B300FC
:10CE9000E44AE30003003A001E2090000060A00076
:10CEA000102798001056800021568000E00F500097
:10CEB000E08F580055FF3A007604470008007800DC
:10CEC00010A302000000000011692A00E0AD20005C
:10CED000DC070200000000007C04440020AF2000BA
:10CEE0000F000900385878000801B100026BEF000C
:10CEF00020AF200002C2B30021B02000904F1100EB
:10CF000001003A000048EB000000E800810F5000EB
:10CF1000FAFF3A000600370010002000B0508800E9
:10CF2000616A2A00E0AD2000DC070200000000007A
:10CF3000C0002000D05688000002EB0004007800FA
:10CF40004F05BE004F04BE000080FA00000006003E
:10CF50000000FA00881F780010002000705688003A
:10CF6000D02AEF00A8AB2000B8CABF000080FB00A9
:10CF70004200DD000080E80060407C00462A02009C
:10CF800000000000F30F50000A003600CE2AEF0028
:10CF9000D02AEF00B8CABF000080FB004200DD00CD
:10CFA0000080E800A16B2A0060407C000440020081
:10CFB000000000004F0478000080FA000000060026
:10CFC0000000FA00B8CABF000080FB004200DD008C
:10CFD000F16C2A00C2AB20006040790004400200DE
:10CFE000000000000080FA00000006000000FA00C7
:10CFF000881F7800A8AB2000516D2A00E0AD20000A
:10D00000C64102000000000082AB200012417800FF
:10D01000800078000000E000040032000280FB0085
:10D020004200DD000080E800040037000280FB00C1
:10D030004200DD000080E800A16D2A0060407C0015
:10D0400004400200000000004F0478000080FA0055
:10D05000000006000000FA00881F78001000200081
:10D0600070568800D02AEF00A8AB2000B8CABF00D5
:10D070000080FB004200DD000080E80060407C0092
:10D08000462A02000000000091042000810F500099
:10D090000A003600B8CABF000080FB004200DD0075
:10D0A0000080E800216E2A0060407C0004400200FD
:10D0B00000000000CE2AEF00D02AEF004F047800D5
:10D0C0000080FA00000006000800FA00889FBE00F9
:10D0D0000E04780000ACBE000D003700640047006D
:10D0E00000405400E14F400008003200B8CABF00C1
:10D0F0000080FB004200DD000080E800E1C2B300D8
:10D1000060C07C0022400200000000000804E8002B
:10D110001880FB008E007800FC8B020000000000ED
:10D12000A9AB2000B8CABF000080FB004200DD00B0
:10D130000080E8008E00780060C07C00044002009F
:10D140000000000067004700800F5400E3FF3A0032
:10D150004F04BE000080FA00000006000000FA0044
:10D16000B8CABF000080FB004200DD00C1BD200046
:10D17000C2AB2000604079000440020000000000C3
:10D180000080FA00000006000000FA00ECCBAB00C3
:10D1900008003200B8CABF000080FB004200DD007A
:10D1A000716F2A00C2AB2000604079000440020089
:10D1B000000000000080FA00000006000000FA00F5
:10D1C00003BC2000934178008381FB0012BC200047
:10D1D000124178004811DD000300710023BC2000DB
:10D1E000934178008381FB0032BC2000124178001B
:10D1F0004811DD0083007100B3FF07000080FA00D2
:10D20000000006000000FA0083BC20009341780073
:10D210008381FB0092BC2000124178004811DD00A0
:10D2200003007100A3BC2000934178008381FB00C0
:10D23000B2BC2000124178004811DD00830071006B
:10D24000A1FF07000080FA00000006000000FA00BD
:10D2500043BC2000934178008381FB0052BC200036
:10D26000124178004811DD000300710063BC20000A
:10D27000934178008381FB0072BC2000124178004A
:10D280004811DD00830071008FFF07000080FA0065
:10D29000000006000000FA00C3BC200093417800A3
:10D2A0008381FB00D2BC2000124178004811DD00D0
:10D2B00003007100E3BC2000934178008381FB00F0
:10D2C000F2BC2000124178004811DD00830071009B
:10D2D0007DFF07000080FA00000006000000FA0051
:10D2E00003BD2000934178008381FB0012BD200024
:10D2F000124178004811DD000300710023BD2000B9
:10D30000934178008381FB0032BD200012417800F8
:10D310004811DD00830071006BFF07000080FA00F8
:10D32000000006000000FA00889FBE008A1F7800F7
:10D33000B8CABF000080FB004200DD00C1AB200086
:10D3400060C07800462A020000000000F10F500083
:10D35000030036000045EB00D9BE20000F00370067
:10D360001000200070568800D02AEF0027003700F8
:10D370000A04E00008003200B8CABF000080FB00C9
:10D380004200DD000080E800A1C3B30060407C00E3
:10D3900022400200000000008904E80019407800E3
:10D3A0009A8C02000000000080407800A8AB2000AA
:10D3B000B8CABF000080FB004200DD000080E8002A
:10D3C00060407C002240020000000000194078000C
:10D3D000B08C02000000000080407800B8CABF0096
:10D3E0000080FB004200DD000080E80060407C001F
:10D3F00022400200000000000A45E800E64F550008
:10D40000DBFF3A00CE2AEF00D02AEF004F0578006C
:10D410004F04BE000080FA00000006000000FA0081
:10D420000080FA00000006000000FA000080FA0008
:10D43000000006000000FA000000FE000080FA0074
:10D44000000006000000FA00B8CABF000080FB0020
:10D450004200DD00E1AD2000C2AB20006040790059
:10D4600004400200000000000080FA0000000600F6
:10D470000000FA000080FA00000006000000FA0038
:10D480000080FA00000006000000FA000080FA00A8
:10D49000000006000000FA000080FA00000006000C
:10D4A0000000FA00B8CABF000080FB004200DD00A7
:10D4B000F16F2A00C2AB20006040790004400200F6
:10D4C000000000000080FA00000006000000FA00E2
:10D4D000881F7800A8AB2000B8CABF000080FB00FE
:10D4E0004200DD000080E80060407C00462A020027
:10D4F00000000000A1042000810F500004003E0045
:10D500001000200070568800D02AEF000A00370073
:10D51000B8CABF000080FB004200DD000080E800C8
:10D5200041702A0060407C000440020000000000BE
:10D53000CE2AEF00D02AEF004F0478000080FA00D6
:10D54000000006000000FA00B8CABF000080FB001F
:10D550004200DD00B1722A00C2AB200060407900B9
:10D5600004400200000000000080FA0000000600F5
:10D570000000FA00B8CABF000080FB004200DD00D6
:10D5800001732A00C2AB2000604079000440020011
:10D59000000000000080FA00000006000000FA0011
:10D5A000A2AB2000B8CABF00180AE2000500320092
:10D5B0000080FB004200DD000080E80001732A00CB
:10D5C000040037000080FB004200DD000080E8001E
:10D5D000B1722A006040790004400200000000009F
:10D5E000182AEF000080FA00000006000000FA0090
:10D5F000A2AB2000B8CABF00160AE2000500320044
:10D600000080FB004200DD000080E80001732A007A
:10D61000040037000080FB004200DD000080E800CD
:10D62000B1722A006040790004400200000000004E
:10D63000162AEF000080FA00000006000800FA0039
:10D64000CABE02000000000060732A000600090044
:10D65000305F78007E00B100E150800011489000FA
:10D660000018A30008003A00711890000000E000C4
:10D6700005003A00010078005EC0020000000000D2
:10D680006101B800010037006011B8008E00780019
:10D6900002007800FC8B020000000000B8CABF0046
:10D6A0000080FB004200DD008E007800C2AB20004D
:10D6B0006040790004400200000000000080FA0091
:10D6C000000006000600FA00D0732A0005000900D9
:10D6D000305F78006E00B100E0508000407890002C
:10D6E0000080FB008E007800FC8B02000000000030
:10D6F000B8CABF000080FB004200DD008E00780049
:10D70000C2AB20006040790004400200000000002D
:10D710000080FA00000006000000FA00E1508000DE
:10D72000EA804000B8CABF000080FB004200DD0074
:10D73000C2AB2000604079000440020000000000FD
:10D740000080FA00000006000000FA006011B80036
:10D750000288BE0022009800330098009048900094
:10D760000104A10011489800904890000114A10004
:10D7700011489800904890000124A1001148980099
:10D780000080FA00000006000000FA00889FBE003A
:10D790000004780003C5B3002348980052C6B300C4
:10D7A0003248980020C7B300404C980031C7B300FE
:10D7B000514C9800624C980063404000704C9800B7
:10D7C0000154980001C2B3001154980070C4B30012
:10D7D0002054980032549800E0C6B300405498009A
:10D7E00051549800F3C04000615498000040EB0091
:10D7F00070549800181090000080A0001014980039
:10D80000335C9800415C9800B0C4B3002064980079
:10D8100081C0E9000800780040C20200000000005A
:10D8200038289000502498004828900060249800E0
:10D83000582890007024980068289000002C9800C8
:10D84000EF05B00020FA2F00808447002E00090069
:10D85000B81C7800E905B100E805B100C09F0200DE
:10D8600000000000890778004F04BE000080FA0025
:10D87000000006000000FA00881F7800000478000D
:10D88000701890000000E0000C003A0024C0020074
:10D8900000000000487990000281FB00110009009F
:10D8A0000280D8008140E800014C98008180FB0094
:10D8B0000800780098C10200000000004F047800C2
:10D8C0000080FA00000006000000FA00881F7800BF
:10D8D00000047800CAC2BF000048A30010003A004C
:10D8E000184890000018A30021003A001848900042
:10D8F0000028A30004003A00080078007EC102005E
:10D90000000000001A00370008007800D9FF070067
:10D91000184890000054A100104C980014003700E3
:10D92000184890000058A3001100320034BE0200D5
:10D9300000000000528480006384800002005000D8
:10D9400083805800424B2C0043002000820F50007F
:10D95000838F58000600360034BE0200000000002D
:10D96000508488006184880008007800C1FF0700A7
:10D970004F0478000080FA00000006000000FA0062
:10D98000881F780000047800208802000000000052
:10D9900008007800AA860200000000000800780055
:10D9A000C9FF07004F0478000080FA00000006005D
:10D9B0000000FA00881F7800000478000101780058
:10D9C000104890000018A30006003200510020000B
:10D9D0000200780022B40200000000000000EB000A
:10D9E00011003700184890000080FB004500DE0061
:10D9F0000004A200614060004500DD0098489000EE
:10DA00000154A10080C07000114C980034BE020087
:10DA1000000000005084880061848800184890004D
:10DA20004500DE00610060004F0478000080FA00CD
:10DA300000000600C800FA00889FBE008A9FBE0052
:10DA4000000478000105780040D12900C7000900D2
:10DA5000305F78008E0CB1001800BE00809FBE00C1
:10DA6000C1DD2900811F78000E0078004E080200F9
:10DA7000000000001A01900011C0B3000E007800F1
:10DA80000200010028009000B8009000809FBE00B6
:10DA9000F1DE2900811F78000E0078004E08020098
:10DAA000000000001A01900011C0B3000E007800C1
:10DAB00002000100080078005EC0020000000000C3
:10DAC000801F780010E02900801F78000E00780089
:10DAD0004E080200000000001A01900011C0B300BF
:10DAE0000E00780002000100084890000080FB0052
:10DAF000801F780031E12900811F78000E00780036
:10DB00004E080200000000001A01900011C0B3008E
:10DB10000E0078000200010018489000E11F60002C
:10DB200040E22900801F78000E0078004E080200B5
:10DB3000000000001A01900011C0B3000E00780030
:10DB400002000100184890000000D100E11F6000B1
:10DB500031E32900811F78000E0078004E08020092
:10DB6000000000001A01900011C0B3000E00780000
:10DB700002000100184890004200DE00E11F600032
:10DB800020E42900801F78000E0078004E08020073
:10DB9000000000000F02B1001A01900011C0B30094
:10DBA0000E00780002000100C2C2BF000000FB00AE
:10DBB0000080EA004F00DE00801F780001E52900A8
:10DBC000811F78000E0078004E080200000000005F
:10DBD0001A01900011C0B3000E007800020001008D
:10DBE000C3C2BF000080FB004200DE000000A200B4
:10DBF000E11F600040E62900801F78000E007800D9
:10DC00004E080200000000001A01900011C0B3008D
:10DC10000E00780002000100C87D900024C00200C0
:10DC200000000000C8249000382490000000E900A3
:10DC3000010020000801BE001403020000000000E3
:10DC40000B81FB0003002000BC0402000000000068
:10DC50000801BE00DC04020000000000809FBE003E
:10DC600081E72900811F78000E0078004E0802002D
:10DC7000000000001A01900011C0B3000E007800EF
:10DC800002000100EE8757004F05BE004F04BE00A2
:10DC90000080FA0000000600C800FA00889FBE005D
:10DCA0000004BE00E0E82900C7000900305F7800EA
:10DCB0008E0CB100EA1F440061F52900811F780035
:10DCC0000E0078004E0802000000000019019000CC
:10DCD00011C0B3000E00780002000100286090001F
:10DCE0000080FB00801F780040F62900801F78002C
:10DCF0000E0078004E08020000000000190190009C
:10DD000011C0B3000E00780002000100382090001E
:10DD1000C8209000809FBE0081F72900811F7800F5
:10DD20000E0078004E08020000000000190190006B
:10DD300011C0B3000E00780002000100FB1F440078
:10DD400080F82900801F78000E0078004E0802003D
:10DD5000000000001901900011C0B3000E0078000F
:10DD600002000100181090004800DE00E11F600072
:10DD700091F92900811F78000E0078004E080200FA
:10DD8000000000001901900011C0B3000E007800DF
:10DD90000200010058249000881F7800C0FA290072
:10DDA000801F78000E0078004E080200000000007E
:10DDB0001901900011C0B3000E00780002000100AC
:10DDC000FA8757004F04BE000080FA0000000600EA
:10DDD000E400FA00889FBE008A9FBE008C9FBE00B0
:10DDE00000047800C0F92F0000004700A028900030
:10DDF00011B798009028900001B79800E028900093
:10DE000071AF98008028900061AF9800D02E9000EC
:10DE100070269000C02D900060259000B02C9000DE
:10DE200050209000B1FB2900DB000900315F780031
:10DE3000CE0DB100801F780070092A00801F780085
:10DE40000E0078004E08020000000000180190004B
:10DE500011C0B3000E00780002000100891F780095
:10DE6000710A2A00811F78000E0078004E08020017
:10DE7000000000001801900011C0B3000E007800EF
:10DE8000020001008A1F7800F00B2A00801F780032
:10DE90000E0078004E0802000000000018019000FB
:10DEA00011C0B3000E007800020001008B1F780043
:10DEB000E10C2A00811F78000E0078004E08020055
:10DEC000000000001801900011C0B3000E0078009F
:10DED000020001008C1F7800500E2A00801F78007D
:10DEE0000E0078004E0802000000000018019000AB
:10DEF00011C0B3000E007800020001008D1F7800F1
:10DF0000910F2A00811F78000E0078004E08020051
:10DF1000000000001801900011C0B3000E0078004E
:10DF2000020001006EA89000801F780051112A00A5
:10DF3000811F78000E0078004E08020000000000EB
:10DF40001801900011C0B3000E007800020001001B
:10DF50007EA89000801F7800A1122A00811F7800FF
:10DF60000E0078004E080200000000000F02B10011
:10DF70001801900011C0B3000E00780002000100EB
:10DF80000EB09000801F7800C1FA2900811F780030
:10DF90000E0078004E0802000000000018019000FA
:10DFA00011C0B3000E007800020001001EB0900006
:10DFB000801F780071142A00811F78000E007800FD
:10DFC0004E080200000000001801900011C0B300CC
:10DFD0000E00780002000100E88757004F06BE00DF
:10DFE0004F05BE004F04BE000080FA00000006008E
:10DFF0000000FA0001017800104890001100200094
:10E000000018A30005003200510020000200780033
:10E0100022B40200000000008000EB000100780044
:10E020000080FA00000006000000FA000001BE00B7
:10E0300010489000510020000018A30009003A0089
:10E0400012489000810020000028A3000500320043
:10E0500012489000110020000008A30005003200C3
:10E06000910020000300780022B4020000000000AC
:10E070008000EB00010078000080FA00000006003C
:10E080000000FA0001017800104890001100200003
:10E090000008A300050032002100200002007800E3
:10E0A00022B40200000000008000EB0001007800B4
:10E0B0000080FA00000006000000FA00889FBE0001
:10E0C0008A1F780000057800810478000204780037
:10E0D000010120000200780012C4020000000000CC
:10E0E0000004E00005003A0021002000090078004B
:10E0F00022B40200000000000E0037006A00450054
:10E1000088007800DC07020000000000EF05B00086
:10E1100020FA2F00008447002E0009003A1C7800E6
:10E12000E805B100EA05B100C09F02000000000050
:10E13000880778004F0578004F04BE000080FA0081
:10E14000000006000000FA00889FBE008A1F7800C9
:10E1500080047800810178000204780002CDB300C9
:10E1600018404100A1C2B300814F500004003E009E
:10E170000805E8001A404100814F500005003600B4
:10E18000110020000300780022B40200000000000B
:10E190001F0037000040EB008EB4020000000000BA
:10E1A00018447800B85C98001A457800CA5C98005A
:10E1B0000900780064FD070011C3B300090078006E
:10E1C00040C202000000000039289000D0249800CE
:10E1D00049289000E024980059289000F0249800E5
:10E1E00069289000802C9800EF05B00020FA2F00DD
:10E1F000008447002E000900391C7800E805B100B2
:10E20000E905B100C09F0200000000008807780007
:10E210004F0578004F04BE000080FA0000000600A1
:10E220000000FA00881F78008180FB008100EA006E
:10E23000CF08DE00C808DD00101190000280A100A8
:10E240000101710012109800EF05B00021FA2F00B3
:10E25000018447002E000900301C7800E805B10059
:10E26000E005B100C09F02000000000088077800B0
:10E270004F0478000080FA00000006000000FA0059
:10E28000881F7800800178000102780050209000FB
:10E29000800F51000300310013289000800F5100BF
:10E2A00005003600210020000400780022B402009E
:10E2B000000000000B003700E2219800EF05B000DD
:10E2C00020FA2F00008447002E000900331C78003C
:10E2D000E805B100E305B100C09F020000000000A6
:10E2E000880778004F0478000080FA0000000600DC
:10E2F0000000FA00881F7800800178000102780091
:10E3000060209000800F5100030036001328900019
:10E31000800F510005003600210020000400780025
:10E3200022B40200000000000B003700D221980048
:10E33000EF05B00020FA2F00008447002E000900EE
:10E34000331C7800E805B100E305B100C09F02006E
:10E3500000000000880778004F0478000080FA0071
:10E36000000006000000FA00881F78008001780095
:10E370000102780020289000800F5100050039002C
:10E38000210020000400780022B4020000000000F8
:10E390000B00370082299800EF05B00020FA2F000B
:10E3A000008447002E000900331C7800E805B10006
:10E3B000E305B100C09F020000000000880778005C
:10E3C0004F0478000080FA00000006000000FA0008
:10E3D000881F7800800178000102780020289000D2
:10E3E000800F510005003900210020000400780052
:10E3F00022B40200000000000B003700F221980058
:10E40000EF05B00020FA2F00008447002E0009001D
:10E41000331C7800E805B100E305B100C09F02009D
:10E4200000000000880778004F0478000080FA00A0
:10E43000000006000000FA00889FBE0080047800FB
:10E4400021609800EF05B00020FA2F0000844700FB
:10E450002E000900391C7800E805B100E905B1007B
:10E46000C09F020000000000880778002964900027
:10E470000804E0000500320024C002000000000093
:10E480008040780010C0B3000400370024C00200B0
:10E49000000000008040780008407800FEC00200C4
:10E4A000000000004F04BE000080FA0000000600DB
:10E4B0000000FA00E0F5200000C1EB0041F9200067
:10E4C0000008EB006248980072004000810F500085
:10E4D000FBFF3A000080FA00000006000000FA008E
:10E4E000E20F500026003A000200E0000A003A0065
:10E4F00040062000808F5000040032006A00400077
:10E50000808F500004003A000200370062002000B3
:10E510000100370012012000C4F520008001EB004B
:10E520001600200083427800140090000000E000F4
:10E530000F003A00010A7800E0062000808F5000AA
:10E5400003003A00F10F51000D003A0005003700BA
:10E5500040062000808F500009003A00E60F51006D
:10E5600007003A00160298000580FB0005003700FE
:10E57000720242008301E800E38F5100E9FF3A0094
:10E58000E00F20000080FA00000006000000FA0002
:10E59000889FBE008101780082007800E24F500021
:10E5A00028003E0022C1B3000440BC00C0F520009A
:10E5B0008004410019009000E10F500021003A0052
:10E5C000EF8F50001F003600A34090008180FB00B9
:10E5D000334090004800DD000104700008003A005C
:10E5E000C88580008800E800C18588008038210047
:10E5F000808F50000200360000402000C085880057
:10E60000E0062000990F100009003A000002EB001C
:10E6100088017800044178006000B800828E020012
:10E620000000000080549800E14F400005003200D7
:10E63000A804980020002000900498000000EB003F
:10E64000010037000080EB004F04BE000080FA009C
:10E65000000006000200FA00889FBE008A9FBE00EC
:10E660008C9FBE00010F7800E24F500041003E0039
:10E6700022C1B3000440BC00C0F52000800441006A
:10E6800040062000990F10003A003A00190090004F
:10E69000E30F500002003A00E9009000010F7800FB
:10E6A0000080E900E10F500032003E0029003700F1
:10E6B0000005EB00E0F52000CDF620001000E000A2
:10E6C0001E003A00A4C0B300A90190000041EB0075
:10E6D0006000B800A431020000000000004478008F
:10E6E0008B05E800E24F4000220032000C2A0200B5
:10E6F000000000003000200090049800EC04980016
:10E700007250B900C4F52000884E78008081E8007E
:10E710004200200082317A00EE0140001200200009
:10E7200082317A0064014000A900900001317A0032
:10E730004206200002307A00080037000A05E8008F
:10E74000F286460072004000E30F550009003200D7
:10E75000DAFF37001E0678008005EB000C06E900A2
:10E760001E007800808F5500D1FF3A000000EB00BA
:10E77000010037000080EB004F06BE004F05BE00D1
:10E780004F04BE000080FA00000006000200FA00FC
:10E79000889FBE008A9FBE008C9FBE0081047800C7
:10E7A00002067800E24F50004B003E0022C1B30049
:10E7B0000440BC00C0F52000000541001A00900094
:10E7C000E30F500044003A00400620009A0F10006A
:10E7D00041003A008006EB00EBF5200040F62000F7
:10E7E000000F7800410020009B8F100033003A009A
:10E7F0009B0090002A009000808F50002F003A006C
:10E800006B4C9000084078000C2A020000000000C9
:10E81000084078002C2A0200000000000000E00000
:10E820002600320008407800BA2C020000000000E8
:10E83000000278000900E000130032000C00E00044
:10E8400011003200F60020009C0F13002200360059
:10E8500090437800C744980010409000D04498003E
:10E86000A4409000E144980034439000F64498009E
:10E87000A44B9000A744980034489000B0449800FE
:10E8800000012000000E78007268B90066014000A7
:10E89000C3F52000D400900001B179001403BE003C
:10E8A0009E0078008688BE000080E800620020009C
:10E8B00002B079000D80FB00080037008D06E800EB
:10E8C0001E03780072034300060F7800F2854500AE
:10E8D000E38F5600C3FF3A00E00F20004F06BE0052
:10E8E0004F05BE004F04BE000080FA000000060085
:10E8F0000000FA00889FBE00800478000004EB004E
:10E90000C3BD200002C2B30068C07900824F50002E
:10E91000050032000004E000030032000804E800B3
:10E92000F00F5400F8FF3A000800E8000081EB0007
:10E93000808F50000800350008017800C1BD20001C
:10E9400009007800FA080200000000000040EB0017
:10E9500000F47C000001EB00020078004F04BE00D0
:10E960000080FA00000006000000FA00881F78000E
:10E9700022C1B3000440BC00C0F5200000044100E7
:10E980001800900011002000E70F50002100320015
:10E99000085090000C2A020000000000800178005E
:10E9A000780090000000E00010003200E2F5200046
:10E9B00044F9200030002000920F100008003A00B7
:10E9C0009200900028009000808F500004003A00D0
:10E9D000400020000300E0000A003A000C0037006D
:10E9E00072014100840F5100F2FF3A000300E00081
:10E9F00007003200085090008C3102000000000037
:10EA00007000200010049800110020000100370061
:10EA10008000EB00010078004F0478000080FA00CD
:10EA2000000006000000FA00889FBE008A1F7800E0
:10EA3000804178000105780082047800E24F5000A0
:10EA400025003E0022C1B3000440BC00C0F52000F8
:10EA5000000441009800780040062000808F50009C
:10EA60000D003A0018009000E60F50001A003A001E
:10EA700003407800BCFF07000000E00016003A00E9
:10EA800008509000090178008A007800863E020054
:10EA90000000000013003700E0062000808F5000C7
:10EAA0000F003A0018009000E20F50000A003A00F0
:10EAB000085090004C910200000000000000E000AF
:10EAC00007003200890078000A0078009491020063
:10EAD00000000000030037000080EB000100370059
:10EAE0000000EB004F0578004F04BE000080FA00E4
:10EAF000000006000000FA00889FBE008A9FBE004A
:10EB00008C9FBE0080457800810678000206780060
:10EB1000040478000505780022C1B3000440BC005D
:10EB2000C0F5200080044100E0062000990F10008D
:10EB30002C003A0019009000E20F500047003A0004
:10EB4000095090004C910200000000000000E0001D
:10EB5000420032000800E0001D0032000A00E00020
:10EB60001B003200F00020009A0F10001800360041
:10EB70000950900082C1B3000440BC00C1EA2000EB
:10EB8000010141001240780040449800124090007A
:10EB90005044980022409000604498003241900018
:10EBA000724498000950900082C1B3000440BC0038
:10EBB0006A01410062C078002044980001014100D0
:10EBC000124190003244980000012000000D7800AE
:10EBD0008C0078000D007800949102000000000085
:10EBE0001F0037000400E000160032000500E000BE
:10EBF00014003200F1002000958F10001100360043
:10EC000009509000BA2C02000000000090407800EB
:10EC1000414498009040900051449800A0409000DA
:10EC200061449800B040900071449800A048900062
:10EC300021449800304890003044980000012000A2
:10EC4000000D78008001EB000C0178008D00780049
:10EC50000B40780073FF0700010037000000EB0055
:10EC60004F06BE004F05BE004F04BE000080FA00F4
:10EC7000000006001C00FA00889FBE008A9FBE00AC
:10EC80008C9FBE0080457800510F980002067800E6
:10EC900005057800E24F50008C003E0022C1B30011
:10ECA0000440BC00C0F5200080044100990290009F
:10ECB0000500E0008500320099007800E0062000A1
:10ECC000808F50006C003A0049009000D9009000FD
:10ECD000008FBE00B90690000400E0002000320062
:10ECE000F00F550079003A00A44090008180FB00AD
:10ECF000344090004800DD0081067000C440900060
:10ED00008180FB00544090004800DD00010170004C
:10ED1000E44090008180FB00744090004800DD00DA
:10ED200081017000028FBE00E18F52000C003A009A
:10ED30006A0447000A0178008000EB0008007800B0
:10ED4000EC070200000000000A017800880078004B
:10ED50000B4078000DFE0700E10F40005B00320021
:10ED60001E0078009E009000E00F5000E08F5800D9
:10ED700002003A00009FEB000097EB000950900062
:10ED800082C1B3000440BC00C8EA20000801410071
:10ED90001E0078009E009000B20F1000A28F180095
:10EDA00022003200E40047000E007800A2A4020016
:10EDB000000000000000E00009003200095090004F
:10EDC00082C1B3000440BC000801410009000900F1
:10EDD0003E597800A200B100AE00B1001300370028
:10EDE00034BE020000000000C27A8000D37A8000A6
:10EDF0000200500083805800A22526002300200036
:10EE0000820F5000838F5800300036000E007800CB
:10EE1000D6A502000000000034BE02000000000081
:10EE2000C07A8800D17A8800280037000950900005
:10EE300052900200000000000000E00023003200B9
:10EE40000950900082C1B3000440BC006A01410037
:10EE5000C0EA20000D3178008C0078005E08900038
:10EE6000AA9002000000000000047800F490020064
:10EE7000000000001600370040062000808F500080
:10EE800012003A00E68F520010003A000B40780062
:10EE9000B5FE07000000E0000C003A000C00E000A6
:10EEA00002003A000C047800090037000950900075
:10EEB0000C017800DE089000623F020000000000B4
:10EEC000000478000000E00001003A000084EB003C
:10EED000080078004F06BE004F05BE004F04BE007C
:10EEE0000080FA00000006000000FA008002EB003B
:10EEF000050278005FFF07000080FA0000000600AE
:10EF00000000FA00889FBE008A9FBE008041780002
:10EF10008102780082007800E24F500067003E00D6
:10EF200022C1B3000440BC00C0F520000005410030
:10EF30001A0190000200E00060003200EF8F5000E4
:10EF40005E003600A54090008180FB0035409000B7
:10EF50004800DD0081057000C54090008180FB0005
:10EF6000554090004800DD0001047000E54090002D
:10EF70008180FB00754090004800DD008104700036
:10EF8000E00F5400E08F5C004C0032000B00E0000A
:10EF90004A003200400620009A0F10002B003A0071
:10EFA000E50F51000900320004003E000200E900B4
:10EFB000E10F500041003E00130037008000EB00DD
:10EFC000E60F51003E0032003C003700034078005D
:10EFD00065FE0700000478000000E00037003A00FA
:10EFE0000A5090002C2A020000000000E1FF2F00D0
:10EFF0000000E000320032006000200010059800A0
:10F00000880078002E003700B4C0B3008B01780070
:10F0100032C0B3000800BE00A431020000000000AE
:10F0200000559800E24F4000240032000C2A0200F4
:10F03000000000000000EB00700598005000200068
:10F0400010059800E1FF2F001D003700E10F51006F
:10F0500012003A00C38580008300E800C185880063
:10F0600080382100808F50000200360000402000D0
:10F07000C08588000B0278000041EB006000B800FA
:10F08000828E02000000000000559800E14F400011
:10F090000A00320020002000100598001A0090009D
:10F0A000E20F500005003A003B0598004805980023
:10F0B000590598008000EB00010037008080EB00CC
:10F0C000010078004F05BE004F04BE000080FA002A
:10F0D000000006000000FA00889FBE008080EB0060
:10F0E000E24F500044003E0022C1B3000440BC0087
:10F0F000C0F5200080044100990090000100E0006C
:10F100003D00320040062000990F100032003A0006
:10F11000E38F500011003A00E8F520004000200085
:10F12000980F100008003A00980090002900900005
:10F13000808F500004003A00684890008C31020033
:10F1400000000000000CEB007204440040F92000B5
:10F15000800F540025003200F0FF3700E38F50008D
:10F1600022003600790090000000E0000D0032001F
:10F17000E2F5200043F9200030002000920F10003B
:10F1800004003A009200900029009000808F500007
:10F190000A00320072014100830F5100F6FF3A006D
:10F1A00002003700E78F5000100032000950900035
:10F1B0008C310200000000000C0037000950900064
:10F1C000163102000000000040002000900498006A
:10F1D0008000EB0008003700E28F500003003A0087
:10F1E00009509000488E0200000000000000EB0073
:10F1F0009004980080007800010078004F04BE0061
:10F200000080FA00000006000000FA00804078004C
:10F210000040E900E64F500007003E000140780042
:10F22000A2C0B3000440BC0060E520000001410022
:10F230000099EB000091EB000080FA00000006004E
:10F240000000FA00889FBE008A1F78000105780040
:10F25000E74F500036003E00A2C0B3000440BC009F
:10F260000200780061E52000810441001901BE0020
:10F27000E10F4100E08F49002D00320064004000A2
:10F28000010440001800BE00E00F5000E08F58005D
:10F29000270032000A00E00009003A0014002000B4
:10F2A00005002000841C4100859449000080EB008B
:10F2B0008080EB00180C4000589448001A0037007A
:10F2C000B4718000C571800061004200E0804A0096
:10F2D000800F5100818F5900050032009208B00064
:10F2E0000380B0000200BE009CA7020000000000E6
:10F2F00052A8020000000000004D78001900BE0076
:10F30000B0718800C1718800120020000300200045
:10F31000821C4000839448000082EB008082EB0056
:10F32000180C420058944A001000200001003700D9
:10F330000000EB004F0578004F04BE000080FA008B
:10F34000000006000000FA00889FBE008A9FBE00F1
:10F350008C1F78000103780002057800E74F500009
:10F3600029003E00A2C0B3000440BC0002027800A5
:10F370006400410065E52000050640001C01BE0058
:10F380006150B800820F5000838F58000100360092
:10F3900002057800850542001B00BE00E10F400019
:10F3A000E08F4800180032000A00E000160032002A
:10F3B0006154B8000600E00005003A00881D4000D6
:10F3C000899548001C1E14001C961C000C00370078
:10F3D0009008B0000180B0008A0178000601780032
:10F3E000C0A70200000000009B0D4400DB954C000C
:10F3F0001C1E14001C961C0036AEEF0038AEEF0049
:10F400000A017800010037000001EB0002007800DB
:10F410004F0678004F05BE004F04BE000080FA0082
:10F42000000006000000FA00881F78000004780041
:10F43000E0718000800F540012003200D271800011
:10F44000820F54000F00310060012000D07288004C
:10F450005C2EEF006B40B90000004100000040004E
:10F460006800400001002000B0728800C17288006E
:10F4700062012000E1E320000040EB00B1FF070043
:10F48000E87188004F0478000080FA000000060050
:10F490000000FA00889FBE0080047800A0728000FF
:10F4A000E10F500024003200D0718000808F5400A2
:10F4B00021003E0018C0B30000E620000081EB00F0
:10F4C0008081EB00B00F1100A08F19000500320001
:10F4D0000844E8006A004000E84F5400030032008E
:10F4E000F8FF3700E74F540013003200090078009E
:10F4F000CCFF07008881FB0008407800A2C0B30061
:10F500000440BC00E800410060E52000893078003C
:10F510008000410014728000257280008488BE0043
:10F520000101780030728000417280002001980053
:10F530003101980001003700F30F2000030078002C
:10F540004F04BE000080FA00000006001200FA001E
:10F55000889FBE008A9FBE008C9FBE000006780078
:10F56000004FEB001004E00060003200A072800049
:10F57000E10F50005D0032008C0078008006EB0047
:10F58000040037000080FB00008046008006400039
:10F590008100E800114078000004E000F9FF3A0023
:10F5A0001BC0B30000E620000081EB008081EB006F
:10F5B000B00F1100A08F1900050032008B45E80044
:10F5C0006A004000E8CF550043003200F8FF3700E2
:10F5D000E7CF550040003A00440037008B81FB0024
:10F5E0000B407800A2C0B3000440BC0061E52000DD
:10F5F0000100410014728000257280000488BE0062
:10F600003472800045728000240098003500980014
:10F610006801410009B17800350037006784640053
:10F620000A003A006150B800B0728800C1728800C8
:10F6300005012000D57288005C2EEF000201200039
:10F640008E80E800084078003EFF07000800440074
:10F650008E80E800608078008D0F50001B003A001B
:10F66000090078006FFF0700F071800001728000D0
:10F67000B0728800C1728800F10F2000D17288003A
:10F680005C2EEF000C047800070037008E00780035
:10F690000040EB00EAFE0700184278009E4F52003F
:10F6A00003003A000804E8001804E000F7FF3A00FD
:10F6B0008E0078000040EB00E1FE07001E04E00031
:10F6C00002003A001804E000C4FF32008904E80098
:10F6D0000A85E800020037008004EB008A00200061
:10F6E000D0718000808F5400CCFF3900F30F2000D0
:10F6F000030078004F06BE004F05BE004F04BE0059
:10F700000080FA00000006000000FA00420020001D
:10F710000CFF0700800078000120A2000100EA0031
:10F72000010070004F00DE00610010000080FA0050
:10F73000000006000000FA00E74F500010003E00F5
:10F74000A2C0B3000440BC008201780064E5200040
:10F75000040141000080EB008080EB00B20F10003C
:10F76000A28F1800060032006880410060007A0015
:10F770002CFF0700307280004172800001003700CA
:10F780006000B8000080FA00000006000000FA00E7
:10F79000004178006000B800E74F510012003E00C1
:10F7A00002407800A2C0B3000440BC008200780090
:10F7B00064E52000040041000081EB008081EB0043
:10F7C000B00F1100A08F190002003A000200BE0025
:10F7D000050037006880400060007A0011FF0700D4
:10F7E00010728000217280000080FA000000060084
:10F7F0000000FA00E74F500014003E00A2C0B30022
:10F800000440BC008201780064E52000040141004E
:10F810000080EB008080EB00B20F1000A28F180078
:10F820000A0032006880410060007A00FDFE070097
:10F83000307280004172800012728000237280005A
:10F840000200400083804800020037000080EB0087
:10F850008080EB000080FA00000006000200FA0041
:10F86000889FBE008A9FBE008C9FBE000045780026
:10F870000204BE0001067800E74F500050003E0031
:10F88000A2C0B3000440BC00020F780060E5200075
:10F89000800541001B01BE00E10F4100E08F4900DF
:10F8A00047003200E18F500035003200050039007A
:10F8B000E28F500014003200E38F500040003A0005
:10F8C0001E0037000A4078009AFF07000006BE00BD
:10F8D000800F5400818F5C0039003E000A407800A0
:10F8E000AAFF0700881D4000899548009E00780007
:10F8F0006480400062E520000200400008185600C5
:10F9000009905E000B0037009E0078006480400084
:10F9100061E5200001004000B00F5400A08F5C00A2
:10F9200027003E00881D41008995490010181400E9
:10F9300010901C0011002000220037000A407800BF
:10F9400092FF07001B01BE000000440081804C00B4
:10F95000800F5100818F590019003900881D510016
:10F96000899559001E0178006400410061E520007E
:10F97000010040001008440050904C00EDFF37009B
:10F980000A4078006BFF0700800F5400818F5C00F5
:10F990000B003E000A40780095FF0700881D5000CC
:10F9A000899558001E01780061E5200001004100A2
:10F9B00028009800390098008C007800010037007A
:10F9C0008000EB00010078004F06BE004F05BE002E
:10F9D0004F04BE000080FA00000006000000FA009C
:10F9E00060E52000C1E920000098EB000090EB00EA
:10F9F0006A004000810F5000FBFF3A001000200019
:10FA0000A0728800562EEF00582EEF005EAEEF0079
:10FA100062E520001241780069014100F203B20062
:10FA2000000420000100200002005000E080580087
:10FA3000D0728800E1728800900820000100200048
:10FA4000B2A7020000000000F10F20000000E0005B
:10FA500001003A0080007800010078000080FA0080
:10FA6000000006000000FA00E74F500010003E00C2
:10FA7000A2C0B3000440BC008201780064E520000D
:10FA8000040141000080EB008080EB00B20F100009
:10FA9000A28F1800060032006880410060007A00E2
:10FAA00060FE070050728000617280000100370024
:10FAB0006000B8000080FA00000006000000FA00B4
:10FAC000E74F500010003E00A2C0B3000440BC004D
:10FAD0008201780064E52000040141000080EB0011
:10FAE0008080EB00B20F1000A28F180006003200D9
:10FAF0006880410060007A004AFE07007072800052
:10FB000081728000010037006000B8000080FA00B8
:10FB1000000006000000FA00E74F50000F003E0012
:10FB2000A2C0B3000440BC008201780064E520005C
:10FB3000040141000080EB008080EB00B20F100058
:10FB4000A28F1800050032006880410060007A0032
:10FB500034FE070090728000010037000000EB00C7
:10FB60000080FA00000006000000FA00E74F500095
:10FB70000C003E00A2C0B3000440BC0064E52000BD
:10FB8000040141000080EB008080EB00B20F100008
:10FB9000A28F18000300320022009000B2009000F3
:10FBA000010037006000B8000080FA000000060085
:10FBB0000000FA00889FBE008104780002047800EB
:10FBC000E74F50001A003E00A2C0B3000440BC0042
:10FBD0008201780064E52000040141000080EB0010
:10FBE0008080EB00B20F1000A28F180010003200CE
:10FBF0006880410060007A000AFE0700F071800012
:10FC000001728000B0728800C1728800F10F20007C
:10FC1000D17288005C2EEF0008017800890078001E
:10FC20000040EB00C7FD0700100020000100370076
:10FC30000000EB004F04BE000080FA000000060048
:10FC40000000FA00889FBE00A2C0B3000440BC00C0
:10FC500061E52000010141001204BE00CBFE070057
:10FC60000004540081845C000800BE004F04BE0004
:10FC70000080FA00000006000000FA00A2C0B300F5
:10FC80000440BC006801410060E52000620078008B
:10FC90000080FA00000006000000FA00562EEF0077
:10FCA000582EEF0080002000D07288005C2EEF00FC
:10FCB00062002000E1E320000040EB00A1FD07000E
:10FCC00062002000819C2A00E0E3200098070200E7
:10FCD000000000000000E00004003A0022002000C4
:10FCE000A1E3200097FD0700010037003A2EEF0046
:10FCF0003CAEEF000080FA00000006000000FA00B1
:10FD0000881F780000047800542EEF00A4A9020098
:10FD1000000000008EA80200000000000000E000CB
:10FD2000FCFF3A000800E00001003200DAFF0700A3
:10FD30004F0478000080FA00000006000000FA007E
:10FD4000889FBE008A9FBE008C9FBE0080467800C0
:10FD500001067800820578000005EB0024003700DA
:10FD60006C407D00B2A90200000000000D40780048
:10FD7000A2C0B3000440BC0060E5200000044100C4
:10FD80001400200005002000180C420058944A007E
:10FD900064014100800441000081EB008081EB00A0
:10FDA00039004100A9804900808CBE00E00F50005E
:10FDB000E08F58000D003A000000EB00CFFF070075
:10FDC00010002000A0728800940820000500200088
:10FDD00038004200A8804A00B2A7020000000000DC
:10FDE0000004200001002000808CBE000A05E8000D
:10FDF0008B0F5500DAFF39000A0078004F06BE006D
:10FE00004F05BE004F04BE000080FA00000006004F
:10FE10000000FA0000E6200061EA20000098EB00F4
:10FE20000090EB006A004000810F5000FBFF3A0099
:10FE300080A702000000000036AEEF0038AEEF00F1
:10FE400095FF0700542EEF000080FA000000060026
:10FE50000000FA000000EB001410AB0002003A00B2
:10FE60001410A800100020000080FA000000060016
:10FE70000000FA0096D0BF00E14F400003003200BE
:10FE8000488E02000000000096F0EF007000200095
:10FE9000C08488001410A90014D0BF000000D10055
:10FEA000610060000080FA00000006000000FA0017
:10FEB000889FBE000004780081447800C1012100C1
:10FEC0008E8A0200000000000000E0000400320002
:10FED0001430A80070002000C0848800060037009D
:10FEE0005881880040818800C0848800090078001B
:10FEF00026F0B7001430A9004F04BE000080FA00BD
:10FF0000000006000000FA00889FBE008A9FBE0025
:10FF10008C1F7800000578008045E8000006780016
:10FF2000010037008B45E8003C4478000804E000FD
:10FF30000C003200E0C2B300804F540009003200D0
:10FF40000040E800804F540006003200634050003B
:10FF5000804F54000300320072404000804F540034
:10FF6000F0FF3A000AC055008044E90009407800DB
:10FF700080900200000000008980FB000A007800E9
:10FF8000AA90020000000000000045000005E80003
:10FF90000804E00009003200F0C2B300804F5400B2
:10FFA0000600320063405000804F540003003200CE
:10FFB00072404000804F5400DAFF3A000040EB00EE
:10FFC00080900200000000004F0678004F05BE0040
:10FFD0004F04BE000080FA00000006000200FA0094
:10FFE0000E0078006C910200000000000000E000AC
:10FFF000120032001E4178008281FB0083007800ED
:020000040001F9
:10000000010CB200000C2000808F500004003A0068
:100010000E0078006C91020000000000070037001D
:100020000204E00005003200830078000000EB00CD
:100030009491020000000000E9FF37000080FA0000
:10004000000006001A00FA00889FBE008A9FBE00CA
:1000500080057800C0848000E30F50004800320023
:1000600004003E00E10F50000C00320015003E007D
:1000700008003700E50F5000900032004C003900B6
:10008000E60F5000B5013200E70F500002023A00BF
:100090009D0137001670EF001570EF00C0BC200006
:1000A000D6A50200000000001670EC0034BE02006D
:1000B00000000000C0808800D1808800200020005F
:1000C000F401370001022100C0BC2000A2A40200FC
:1000D000000000000000E00013003A0034BE0200FF
:1000E00000000000C2808000D38080000200500029
:1000F00083805800A225260023002000820F500094
:10010000838F5800E4013600610020006001210067
:1001100022C0B300904F110001003E0011002000EA
:10012000C1848800DC013700C1BC20009140780008
:100130008180FB00CDCBBF004800DD0001017000D5
:10014000E1BC2000914078008180FB00CFCBBF0054
:100150004800DD0081017000020078001CF0B7004B
:100160004810DE001DF0B700030078001EF0B70055
:100170004818DE001FF0B70030002000C08488005F
:10018000540320008001EB0042C0B300C0012100F5
:1001900001002000828E02000000000096F0B700EF
:1001A000E14F4000BC01320040002000C0848800C4
:1001B00096D0BF0052900200000000000000E00056
:1001C000B5013200BC30EC00BDD0BF008090020011
:1001D00000000000BCD0BF008090020000000000C2
:1001E00010C0B30080900200000000000040EB004F
:1001F00080900200000000000040EB0080900200B0
:100200000000000010C0B300809002000000000059
:100210000040EB0080900200000000000040EB0076
:1002200080900200000000000040EB00809002007F
:10023000000000000040EB00809002000000000081
:100240000040EB0080900200000000000040EB0046
:100250008090020000000000508180000000E0005B
:1002600001003A004081800026FF07000040EB00BB
:10027000809002000000000026D0BF0080900200A5
:10028000000000000040EB00809002000000000031
:1002900010C0B3008090020000000000F490020043
:1002A0000000000034BE020000000000C080880092
:1002B000D1808800500020007601370096D0BF0022
:1002C0004C91020000000000000478000000E000F3
:1002D0000F003A0034BE020000000000C28080001F
:1002E000D38080000200500083805800A2252600A1
:1002F00023002000820F5000838F580066013600D3
:1003000060002000C0848800080078006301370086
:100310006E0447006F0047006C910200000000006F
:10032000080078006C91020000000000E085800069
:10033000980F100003003200C2910200000000007C
:1003400055013700710047006C9102000000000069
:10035000700047006C91020000000000730047002D
:100360006C91020000000000720047006C910200D6
:1003700000000000750047006C91020000000000C2
:10038000740047006C9102000000000077004700F5
:100390006C91020000000000760047006C910200A2
:1003A00000000000790047006C910200000000008E
:1003B000780047000D00370008FF07008E84E80032
:1003C00063044700080078006C9102000000000000
:1003D000090078006C91020000000000080078001D
:1003E0006C91020000000000090078006C9102008E
:1003F000000000001E0890000000E900100F9800A7
:10040000E10F4000ECFF3A0033003700F3FE070035
:1004100064044700650047006C9102000000000082
:10042000080078006C91020000000000670047009F
:100430006C91020000000000660547000A00780089
:100440006C910200000000006B0047006C910200FC
:10045000000000006A0047006C91020000000000EC
:10046000690047006C910200000000006400440035
:100470006C910200000000006D0047006C910200CA
:1004800000000000EC044700090078006C910200B5
:100490000000000010002000980F100009003A0032
:1004A0009A0F100007003A0042002000990F110037
:1004B00004003A00710037000E0078006C910200D1
:1004C000000000006E0090000000E9006007980046
:1004D000E10F4000F8FF3A002E0890000000E9000C
:1004E000200F9800E10F4000C8FF3A0033003700AA
:1004F000BAFE070064044700650047006C910200E3
:1005000000000000080078006C910200000000006C
:10051000670047006C91020000000000660547007C
:100520000A0078006C910200000000006B00470098
:100530006C910200000000006A0047006C9102000C
:1005400000000000690047006C91020000000000FC
:10055000640044006C910200000000006D00470040
:100560006C91020000000000EC04470009007800D4
:100570006C9102000000000010002000980F100095
:1005800009003A009A0F100007003A0042002000CC
:10059000990F110004003A00380037000E0078006F
:1005A0006C910200000000006E0090000000E90065
:1005B00060079800E10F4000F8FF3A003E08900005
:1005C0000000E900300F9800E10F4000C8FF3A003A
:1005D0004000370081FE07006404470065004700C3
:1005E0006C91020000000000080078006C9102008D
:1005F00000000000670047006C910200000000004E
:10060000660547000A0078006C91020000000000B7
:100610006B0047006C910200000000006A00470078
:100620006C91020000000000690047006C9102001C
:1006300000000000640044006C9102000000000013
:100640006D0047006C91020000000000EC044700C0
:10065000090078006C9102000000000010002000EA
:10066000980F100016003A009A0F100014003A007C
:1006700042002000990F110011003A001430A80028
:10068000C00121006C91020000000000D001210097
:100690006C91020000000000E00121006C9102005A
:1006A00000000000F00121006C9102000000000039
:1006B0000D0037000E0078006C9102000000000071
:1006C0006E0090000000E90060079800E10F400014
:1006D000F8FF3A004E0890000000E900400F980033
:1006E000E10F4000BBFF3A00C29102000000000091
:1006F00096D0BF00488E02000000000096F0EF0088
:1007000070002000C084880014D0BF0062406000E8
:1007100004003A001CF0B7001DF0B7001EF0B7004F
:100720001FF0B700C1012100914078008180FB00DB
:100730001DD0BF004800DD0001017000E101210073
:10074000914078008180FB001FD0BF004800DD0091
:1007500081017000828DBE000500370015D0BF00FA
:10076000E14F500004003600800DEB00BB1578000F
:1007700010002000490037000040E80015F0B700E5
:1007800001BD2000914078008180FB00D1CBBF00EB
:100790004800DD00810470000901780021BD2000BF
:1007A000914078008180FB00D3CBBF004800DD0082
:1007B0000104700088017800E00F5100E08F5900BB
:1007C00035003200C1BC2000914078008180FB00E0
:1007D000CDCBBF004800DD0001037000E1BC20006C
:1007E000914078008180FB00CFCBBF004800DD0046
:1007F0008103700002036B0083836B0009027800A1
:100800008802780006026A0087826A000400780085
:10081000D0EBB7004820DE00D1EBB7000500780030
:10082000D2EBB7004828DE00D3EBB7008681FB008F
:100830004831DE004811DD00030071008781FB00B4
:100840004839DE004811DD008300710004006800B3
:1008500085806800CCEBB7004801DE00020078001C
:10086000CDEBB70001007800CEEBB7004808DE0002
:10087000CFEBB7001670EF0096D0BF00E14F4000FD
:1008800003003200488E02000000000096F0EF00E6
:1008900010002000C08488000000EB004F05BE005F
:1008A0004F04BE000080FA00000006000000FA00BD
:1008B0008040EB0001789800D07890000104A000FF
:1008C000517898008000EB00511898000080FA00E1
:1008D000000006000000FA00889FBE0000047800B7
:1008E00010C0B3008EB40200000000001848900051
:1008F000E1CFB30001406000104C98001848900010
:100900000014A100104C9800184890000024A10089
:10091000104C98008004EB00591C98005878900007
:1009200001406000507C9800E820900010C0B300A7
:10093000FAB40200000000008828900010C0B30044
:1009400096B40200000000001800BE0020049800C9
:1009500031049800791C980010C0B30086B40200DE
:10096000000000004F04BE000080FA0000000600F6
:100970000000FA00881F78000004780010489000FA
:100980000054A100104C9800082090000000E000E6
:1009900004003A0008007800CEFF07001000200095
:1009A000002498004F0478000080FA000000060040
:1009B0000000FA00889FBE008A1F7800407D9000EA
:1009C00030249000C02490000180FB000000E9006A
:1009D000CF80DE000801BE0014030200000000000A
:1009E0000A81FB0003002000BC040200000000009C
:1009F0000801BE00DC040200000000004F05780082
:100A00004F04BE000080FA00000006000000FA005B
:100A1000889FBE008A1F78000004780010C0B300D1
:100A20008EB402000000000024C00200000000009C
:100A30008040780008007800DDFF0700008CBE00D1
:100A40002004980031049800184890000024A00069
:100A5000104C9800184890000014A100104C980009
:100A600018489000EACFB3000A406000104C98008C
:100A7000EF05B00020FA2F00808447002E00090007
:100A8000B81C7800E905B100E805B100C09F02007C
:100A900000000000587890000A406000507C9800E8
:100AA0000005EB005A1C980089077800E8209000A8
:100AB00010C0B300FAB402000000000088289000C3
:100AC00010C0B30096B402000000000024C0020071
:100AD000000000008040780010C0B300FEC002009B
:100AE000000000000A2498004F0578004F04BE0063
:100AF0000080FA00000006000000FA000008EB0089
:100B00003010780082BB20000300200022009800F3
:100B100033009800D07890000104A000517898002C
:100B20000080FA00000006000000FA00881F78002C
:100B300002447800823E200003002000DC04020012
:100B400000000000421F2000820F5000E08F58007C
:100B500003003600884078000040EB0002003700B8
:100B60008840780010C0B300FEC002000000000002
:100B70004F0478000080FA00000006000000FA0030
:100B8000201890000080FA00000006000000FA0023
:100B9000889FBE008A1F7800000478000105780055
:100BA00010C0B3008EB4020000000000184890008E
:100BB0000004A000104C9800184890000014A000F9
:100BC000104C9800184890000024A100104C980088
:100BD000EF05B00020FA2F00808447002E000900A6
:100BE000B81C7800E905B100E805B100C09F02001B
:100BF0000000000089077800F820900010C0B300C2
:100C000096B4020000000000587890000004A00094
:100C1000507C98000000EB00501C98001A1C9800B3
:100C2000000CEB003814780038209000C8209000A9
:100C300061005000E08058002004980031049800C2
:100C40001A1C980010C0B30086B402000000000017
:100C50004F0578004F04BE000080FA000000060037
:100C60000000FA00889FBE000004BE00E020900053
:100C700010C0B300FAB402000000000058789000E1
:100C80000004A000507C98000000EB00501C98006D
:100C9000191C98006000B8002004980031049800E6
:100CA000191C98004F04BE000080FA0000000600E6
:100CB0000000FA00881F78000004780010489000B7
:100CC0000004A100104C9800E820900010C0B30070
:100CD000FAB40200000000008828900010C0B300A1
:100CE00096B4020000000000587890000004A100B3
:100CF000507C98000000EB00501C9800701C98007D
:100D000024C0020000000000800078000848900025
:100D1000814F500003003200184890000024A100C9
:100D2000104C9800014C980010C0B300FEC00200A7
:100D300000000000D2C2BF000068A3000200320021
:100D400076AC0200000000004F0478000080FA003A
:100D5000000006000000FA00889FBE000004780032
:100D6000F01C9000E28F54002C00320003003E0083
:100D7000E18F540091003A0005003700E38F5400E2
:100D800055003200E48F54008C003A0070003700A8
:100D9000094078008EB4020000000000F8209000A6
:100DA0000940780096B402000000000058789000D6
:100DB0000004A000507C98000000EB00501C98003C
:100DC000281A9000141C9800780890007284800003
:100DD0008384800000004100E0804900141C9800DA
:100DE00038219000C8219000DC04020000000000BF
:100DF000200498003104980020002000701C980006
:100E0000184890000004A000104C98000940780099
:100E100086B4020000000000680037001001BE0028
:100E2000B000900020009000800F5100818F590089
:100E300022003A0038189000101C9800748480003A
:100E400085848000081090006101B800820F520074
:100E5000838F5A000500310038209000C820900090
:100E60000200500083805800020037000200520048
:100E700083805A002004980031049800300020003C
:100E8000701C9800587890000004A100507C9800D5
:100E90000000EB00501C9800F820900010C0B30038
:100EA00096B4020000000000E820900010C0B300DB
:100EB000FAB40200000000004000370058789000AB
:100EC0000004A000507C9800084990001800BE0063
:100ED00015FF0700390037001001BE00B000900078
:100EE00020009000800F5100818F590010003A00BF
:100EF0008828900010C0B30096B4020000000000E3
:100F00007084800081848000D002B0000180B00035
:100F100038219000C8219000DC040200000000008D
:100F2000008CBE0040002000701C98002300370099
:100F3000B8189000111C9800587890000004A00088
:100F4000507C98000000EB00501C98001B003700FC
:100F50001001BE00B000900020009000800F5100F2
:100F6000818F59000A003A007084800081848000DB
:100F7000200498003104980028009000B8009000E8
:100F8000008CBE000800780049FF07000B00370006
:100F9000B8189000111C9800587890000004A00028
:100FA000507C9800A0502000501C98008828900089
:100FB00010C0B30096B40200000000004F04BE0051
:100FC0000080FA00000006000000FA0080007800AF
:100FD000B00F5100A08F59000400320072848800C5
:100FE0008384880010002000F01898000080FA0028
:100FF000000006000000FA00881F78000004780056
:10100000002090000000E0000A003A00014C980027
:101010000800780066FE0700B80F5000A88F58003F
:101020000400320070848800818488001000200051
:10103000701C98004F0478000080FA000000060041
:101040000000FA00889FBE008A1F78000005780023
:1010500000249000E30F54002100320005003E0000
:101060000800E000A0003200E10F540006003A0042
:1010700007003700E50F54004C0032003B003900F8
:10108000E60F5400590032000000EB003100370039
:10109000884178000841780088407800084078004E
:1010A000BEC00200000000002A189000101D980029
:1010B0000000EB00501D9800EA20900008407800E6
:1010C000FAB4020000000000AA1890000A0078009C
:1010D000AEFE070030002000002598004F003700CA
:1010E000C242E20003003D00C3C2BF000028A300CB
:1010F0001A003A001A04BE004A7990000281FB00EF
:101100000281E800CF91DE001A209000AA20900012
:10111000BC04020000000000800F5400818F5C00BE
:101120003E003600000DEB003A15780080BB200031
:101130000100200020059800310598005A789000A1
:101140000004A000507D98002A199000121D9800FC
:101150004000200000259800630037005A78900076
:101160000004A000507D98002C003700C242E2002D
:101170002A003D00C3C2BF000028A30027003200A0
:101180001A00BE0042062000820F5000E08F580077
:10119000220036005000200000259800BA18900068
:1011A0000A007800AEFE07004F0037001001BE00B5
:1011B000B000900020009000800F5100818F5900F6
:1011C00049003A000A00780010FE070024C002001F
:1011D00000000000E10F50004300320011C0B300D6
:1011E0000A00780083FF07003F00370024C0020098
:1011F00000000000E40F50003B003A001A48900045
:101200000008A30038003A000000EB000025980019
:101210000A007800D6FD0700330037001A01BE002F
:101220002A009000BA009000800F5100818F590071
:101230002D003A0010C0B3008EB402000000000080
:101240001A4890000024A100104D98001A48900000
:101250000014A100104D98001A4890000004A1004D
:10126000104D9800EA20900010C0B300FAB40200BC
:10127000000000008A28900010C0B30096B402005D
:10128000000000000004EB00082598008841780069
:1012900012C0B3008840780002407800BEC002004F
:1012A00000000000EF05B00020FA2F008084470006
:1012B0002E000900BA1C7800E905B100EA05B1006A
:1012C000C09F0200000000005A7890000004A100B6
:1012D000507D9800581D98008907780010C0B30011
:1012E00086B40200000000004F0578004F04BE00E5
:1012F0000080FA00000006000000FA00889FBE008F
:10130000D0848000E18480000044EB0009002D00BF
:101310008102D1000082D30061016000030020003F
:1013200060011100E0811900038064006103B800CE
:10133000C030DD000000200060031100E0831900D0
:10134000060070008780700000006A0081806A00DB
:101350000844E800EF4F5400EDFF3A00D0848800C5
:10136000E18488004F04BE000080FA0000000600FF
:101370000000FA00881F78008A9FBE00DA8480008F
:10138000EB848000E00F5000E08F580002003A002C
:101390001000200001002000D0848800E184880033
:1013A00008C1B300D4FF07000844E900FDFF3A007C
:1013B0000A00BE004F05BE004F0478000080FA000E
:1013C000000006000C00FA00889FBE008A9FBE0045
:1013D0008C9FBE0000198000400798001019800003
:1013E000300798002019800020079800200880000E
:1013F0001007980010088000000F78002023EF00ED
:1014000000F0290020198800F0032000101988003E
:10141000400E2800001988000000280020088800DD
:1014200002A1EF00B4FF07006105B8000040EB0027
:10143000204F98006066B8008004EB000100370080
:10144000880478000060FE0085C0BF000058A3003B
:10145000FDFF3200080880000021EF0085A0A900F0
:10146000A5FF07000001780008064600E0864E0050
:10147000F09F250021262000800F5600818F5E00FE
:10148000050036009CFF070000056D009AFF07006D
:1014900080856D0010003700888F5400E9FF32000E
:1014A000088054000000410001002000B0FF070048
:1014B0000A0545008B854D008FFF07000078A300CB
:1014C000010032000A00A0002E4890000040E80011
:1014D000204F9800DAFF3A002023EF002E00900002
:1014E000201988003E009000101988004E009000DE
:1014F000001988001E009000200888001E00780057
:10150000100888000A00BE004F06BE004F05BE004E
:101510004F04BE000080FA00000006000000FA0040
:10152000889FBE008A9FBE008C9FBE000006780088
:10153000810478006033B8000041EB000244780079
:101540005A5020002B0020004D06200027003700B5
:10155000E34F540029003E0000CDB30000C040001E
:101560000204E00016003200E34F510003003A008D
:10157000E24F40003F003A0002003700E24F4000D7
:101580000F003A008A0F53008B8F5B0039003E003A
:101590000880FB000781FB000D91B9004832DE0096
:1015A0006A22B900044141000641410002F07C007A
:1015B0000844E8006033B8000041EB000B0037003E
:1015C000E94F50002B003E000241E800C83BDD001F
:1015D0000680FD00864378000043EB008080FB001E
:1015E00000F02F000003630001037300BC4078008B
:1015F0000104E000D6FF3A000F003700F0C2B3004C
:1016000080CF50000C003200EDCF50000A003200B5
:10161000EACF5000080032006F40500080CF5000E9
:1016200005003200E9CF5000030032007A4040004C
:1016300080CF50000F003A005050200021002000C1
:10164000800F5300818F5B000A003E000780FB0083
:10165000420620000280B9004831DE006A11B9005C
:101660000240400006404000B044980010002000B6
:10167000010037000000EB004F06BE004F05BE0022
:101680004F04BE000080FA00000006000000FA00CF
:10169000889FBE00800478000104780082027800F0
:1016A0000043EB008003EB00870078004C0037001C
:1016B00069C27800F0CBB30000404200F94F5000FF
:1016C00002003E00004278001D003700F0C9B30060
:1016D00000404200F94F500003003E0090CBB300A1
:1016E000004242001600370000CDB3000040420027
:1016F000E94F500002003E006442420010003700F3
:10170000B0C2B300804F52000A00320000C0E800AF
:10171000804F52000700320000C0E800804F5200A6
:1017200006003200F0C5B300804F52002B003A0093
:1017300002003700E4C3B30001003700F4C3B30074
:101740000604E00007003A00838F530026003100B2
:101750008703E8004220DD00804A780016C0B3000D
:101760001E003700E14F53000B003A000480FB00DD
:101770004400DE0015407000805A7800838F5300CB
:10178000190031008703E8004420DD00804A78001A
:1017900026C0B300110037000501E800E24F5300F6
:1017A0000B003A000480FB004200DE00954A700006
:1017B00082027800838F53000B0031008703E8001A
:1017C0004620DD000049780036C0B3000300370032
:1017D000954A7200820278000043EB008100E80025
:1017E000888F5000B2FF3A00070078004F04BE0017
:1017F0000080FA00000006000000FA000001BE00B0
:101800000000E000160032000003EB00047122002B
:1018100055C0B300A7002000110009000481D800C2
:101820008000FD000100E00002003A000600E00038
:101830000500320000C3B30080D940000488B9001D
:101840000001510016002000110009000782D80095
:10185000000278008542E90003003200EEFF370005
:1018600000C3B300805978008049EB000080FA0083
:10187000000006000000FA0000017800C800DE0049
:1018800063C4B30083CF50000500360000CEB30020
:1018900000C040004800DD00F20FB20000017100FE
:1018A000834F51000600360000CEB30000404100D7
:1018B0000080FB0001F02F000101610000017100B8
:1018C000C810DE00F20FB20090C3B30080CF50000A
:1018D0000200360090CCB3000100370000CDB30009
:1018E00000C040004800DD00000171008240780027
:1018F00090C3B300804F51000200360090CCB3007B
:101900000100370000CDB30000C040000080FB00A4
:1019100001F02F0001016100000171004810DE009C
:101920004400DD00024070000080FB000080FA00EF
:10193000000006000000FA000080FB004400DE000A
:10194000E94F5000020036007043B000010037003C
:101950000043B0000080FB000080FA000000060099
:101960000000FA006F406000E94F500002003600AE
:101970007043B000010037000043B0000080FB005E
:101980000080FA00000006000000FA000002780063
:10199000904178001141780006CEB3000E00370068
:1019A000F5C9B30005C04100F94F500001003E00E9
:1019B00086C1410005404100F94F500001003E0042
:1019C0000641410082CF51000E003E000F00390059
:1019D000D4417800514178000304E0000500320052
:1019E0000204E000EEFF3A000304E00005003E00C0
:1019F0000200370082CF5100040039000000EB00E4
:101A00000300370010002000010037000080EB00C9
:101A10000080FA00000006000000FA0000017800D3
:101A2000C800DD000080FB00010070004811DE00EE
:101A300001F02F0001006000020070000080FA0039
:101A4000000006000400FA00008FBE00BE409000B7
:101A50001EC06800004F78000140680030479800C1
:101A60001E4F68002E4090009E40900080C068008D
:101A700000C06800204798000140680010479800A7
:101A80001E00BE000080FA00000006000000FA0000
:101A90000103D100000278006011B8008002EB0061
:101AA000040037003400780000014100E081490063
:101AB0008502E800868F5200FAFF3A000108A30071
:101AC00005003200144078000080FB000100200077
:101AD00002014000838148006118B8000200400004
:101AE000E0804800010040000080EA000080FA0029
:101AF000000006000000FA00800178000001780074
:101B0000F5C9B30004CEB3000500370005C040009E
:101B1000F94F500001003E0004C940000201E800F6
:101B2000924078000104E000F8FF3A0003007800DA
:101B30000080FA00000006000000FA00881F78000C
:101B4000000478000040EB00704C9800080078001A
:101B5000E8FF07000001EB00824078006840790050
:101B60000004E00008003A0002C2B3000180FB005C
:101B700008004000025878008140E800EECF500095
:101B800004003E00FBFF37000201E800EF0F5100A8
:101B9000F1FF3A004F0478000080FA0000000600D0
:101BA0000000FA00000278008002EB000A00370013
